:020000040800F2
:1000000000060020E1010008E3010008E301000808
:10001000E3010008E3010008E3010008E301000830
:10002000E3010008E3010008E30100086D2F000868
:10003000E3010008E3010008E3010008E301000810
:10004000E3010008E3010008E3010008E301000800
:10005000E3010008E3010008153200083D32000802
:10006000653200088D320008B5320008E30100084F
:10007000E3010008E3010008E3010008E3010008D0
:10008000E3010008E3010008E3010008E3010008C0
:10009000E3010008E3010008E3010008DD32000885
:1000A000E3010008E3010008E3010008E3010008A0
:1000B000B1330008E3010008E3010008E301000890
:1000C000E3010008E3010008E3010008E301000880
:1000D000E3010008E3010008E3010008E301000870
:1000E00041330008E3010008E3010008E3010008D0
:1000F000E3010008E3010008E3010008E301000850
:10010000E3010008E3010008E3010008E30100083F
:10011000E3010008E3010008E3010008E30100082F
:10012000E3010008E3010008E3010008E30100081F
:10013000E3010008E3010008E3010008E30100080F
:10014000E3010008E3010008E3010008212700089B
:10015000E3010008E3010008E3010008E3010008EF
:10016000E3010008E3010008E3010008E3010008DF
:10017000E3010008E3010008E3010008E3010008CF
:10018000E3010008E3010008E3010008E3010008BF
:10019000E3010008E3010008E3010008E3010008AF
:1001A000E3010008E3010008E3010008E30100089F
:1001B000E3010008E3010008E3010008E30100088F
:1001C000E3010008E3010008E3010008E30100087F
:1001D000E3010008E3010008E3010008E30100086F
:1001E00002E000F000F8FEE772B6374880F30888B6
:1001F000364880F3098836483649086040F20000E6
:10020000CCF200004EF63471CEF200010860BFF36C
:100210004F8FBFF36F8F40F20000C0F2F0004EF638
:100220008851CEF200010860BFF34F8FBFF36F8F8C
:100230004FF00000E1EE100A4EF63C71CEF20001E4
:100240000860062080F31488BFF36F8F01F030FF41
:1002500002F02AFE4FF055301F491B4A91423CBF25
:1002600041F8040BFAE71D49184A91423CBF41F896
:10027000040BFAE71A491B4A1B4B9A423EBF51F83E
:10028000040B42F8040BF8E700201849184A914281
:100290003CBF41F8040BFAE701F00EFF02F058FEF4
:1002A000144C154DAC4203DA54F8041B8847F9E7A7
:1002B00000F042F8114C124DAC4203DA54F8041B22
:1002C0008847F9E701F0F6BE000600200022002072
:1002D0000000000808ED00E00000002000060020FB
:1002E0007837000800220020402200204022002011
:1002F000602E0020E0010008E0010008E001000895
:10030000E00100082DE9F04F2DED108AC1F80CD066
:10031000C3689D46BDEC108ABDE8F08F002383F3CF
:1003200011882846A047002001F072FAFEE701F08C
:1003300001FA00DFFEE7000038B500F0BBFB01F07A
:1003400087FE054601F0AAFE0446C8B90E4B9D4241
:1003500018D001339D4218BF044641F2883504BFCE
:1003600001240025002001F07DFE0CB100F074F89E
:1003700000F000FD284600F0BFF800F06DF8F9E746
:100380000025EFE70546EDE7010007B008B500F0EE
:1003900063FBA0F120035842584108BD07B541F264
:1003A0001203022101A8ADF8043000F073FB03B082
:1003B0005DF804FB38B5302383F3118817480368D0
:1003C0000BB101F0F1FA164A144800234FF47A7188
:1003D00001F0E0FA002383F31188124C236813B173
:1003E0002368013B2360636813B16368013B63606A
:1003F0000D4D2B7833B963687BB9022000F024FCE3
:10040000322363602B78032B07D163682BB902205A
:1004100000F01AFC4FF47A73636038BD402200206C
:10042000B50300086023002058220020084B1870F4
:1004300003280CD8DFE800F008050208022000F0CD
:10044000F9BB022000F0ECBB024B00225A6070475F
:100450005822002060230020234B244A10B51C465C
:10046000196801313FD004339342F9D16268A24246
:1004700039D31F4B9B6803F1006303F540439A4255
:1004800031D2002000F030FB0220FFF7CFFF194BE4
:100490001A6C00221A64196E1A66196E596C5A6425
:1004A000596E5A665A6E5A6942F080025A615A6908
:1004B00022F080025A615A691A6942F000521A61A8
:1004C0001A6922F000521A611B6972B64FF0E023DC
:1004D0003021C3F8084DD4E9003281F311889D46DC
:1004E00083F30888104710BD00C0000820C0000832
:1004F00000220020003802402DE9F04F93B0AA4BB3
:1005000000902022FF210AA89D6800F0DDFBA74A89
:100510001378A3B9A648012103601170302383F337
:10052000118803680BB101F03FFAA24AA0480023EA
:100530004FF47A7101F02EFA002383F31188009BA7
:1005400013B19D4B009A1A609C4A009C1378032BB0
:100550001EBF00231370984A4FF0000A18BF536063
:10056000D3465646D146012000F064FB24B1924B9D
:100570001B68002B00F01182002000F06DFA039040
:10058000039B002BF2DB012000F04AFB039B213B85
:10059000162BE8D801A252F823F000BFF905000895
:1005A00021060008B5060008670500086705000871
:1005B000670500083F0700080F0900082908000820
:1005C0008B080008B3080008D90800086705000870
:1005D000EB080008670500085D0900089906000897
:1005E00067050008A109000805060008990600082B
:1005F000670500088B0800080220FFF7C7FE0028E7
:1006000040F0F581009B0221BAF1000F08BF1C46A3
:1006100005A841F21233ADF8143000F03BFAA2E71E
:100620004FF47A7000F018FA071EEBDB0220FFF798
:10063000ADFE0028E6D0013F052F00F2DA81DFE8A9
:1006400007F0030A0D10133605230593042105A8AE
:1006500000F020FA17E054480421F9E75848042133
:10066000F6E758480421F3E74FF01C08404600F035
:100670003DFA08F104080590042105A800F00AFAE3
:10068000B8F12C0FF2D1012000FA07F747EA0B0B63
:100690005FFA8BFB4FF0000900F062FB26B10BF014
:1006A0000B030B2B08BF0024FFF778FE5BE74648DF
:1006B0000421CDE7002EA5D00BF00B030B2BA1D10D
:1006C0000220FFF763FE074600289BD0012000F0C0
:1006D0000BFA0220FFF7AAFE00261FFA86F8404612
:1006E00000F012FA044690B10021404600F01CFAD6
:1006F00001360028F1D1BA46044641F21213022114
:1007000005A8ADF814303E4600F0C4F92BE70120EF
:10071000FFF78CFE2546244B9B68AB4207D9284641
:1007200000F0E4F9013040F067810435F3E7234B32
:1007300000251D70204BBA465D603E46ACE7002E9A
:100740003FF460AF0BF00B030B2B7FF45BAF022089
:10075000FFF76CFE322000F07FF9B0F10008FFF6E1
:1007600051AF18F003077FF44DAF0F4A926808EBC2
:10077000050393423FF646AFB8F5807F3FF742AF9F
:10078000124B0193B84523DD4FF47A7000F064F901
:100790000390039A002AFFF635AF019B039A03F8F2
:1007A000012B0137EDE700BF002200205C23002071
:1007B00040220020B50300086023002058220020BA
:1007C00004220020082200200C2200205C220020AD
:1007D000C820FFF7DBFD074600283FF413AF1F2DAD
:1007E00011D8C5F1200242450AAB25F0030028BF0D
:1007F000424683490192184400F040FA019A804829
:10080000FF2100F061FA4FEAA8037D490193C8F384
:100810008702284600F060FA064600283FF46DAFD4
:10082000019B05EB830537E70220FFF7AFFD0028AA
:100830003FF4E8AE00F0A4F900283FF4E3AE00274F
:10084000B846704B9B68BB4218D91F2F11D80A9B22
:1008500001330ED027F0030312AA134453F8203CAF
:1008600005934046042205A900F0AEFA04378046FD
:10087000E7E7384600F03AF90590F2E7CDF8148042
:10088000042105A800F006F906E70023642104A866
:10089000049300F0F5F800287FF4B4AE0220FFF7CF
:1008A00075FD00283FF4AEAE049800F051F90590B4
:1008B000E6E70023642104A8049300F0E1F800288F
:1008C0007FF4A0AE0220FFF761FD00283FF49AAE4E
:1008D000049800F04DF9EAE70220FFF757FD0028E1
:1008E0003FF490AE00F05CF9E1E70220FFF74EFD27
:1008F00000283FF487AE05A9142000F057F9042121
:100900000746049004A800F0C5F83946B9E732203C
:1009100000F0A2F8071EFFF675AEBB077FF472AEBB
:10092000384A926807EB090393423FF66BAE022008
:10093000FFF72CFD00283FF465AE27F003074F4476
:10094000B9453FF4A9AE484600F0D0F8042105901F
:1009500005A800F09FF809F10409F1E74FF47A7057
:10096000FFF714FD00283FF44DAE00F009F9002810
:1009700044D00A9B01330BD008220AA9002000F0C2
:10098000ABF900283AD02022FF210AA800F09CF9F8
:10099000FFF704FD1C4800F041FF13B0BDE8F08FE5
:1009A000002E3FF42FAE0BF00B030B2B7FF42AAE7F
:1009B0000023642105A8059300F062F8074600288B
:1009C0007FF420AE0220FFF7E1FC804600283FF4D0
:1009D00019AEFFF7E3FC41F2883000F01FFF0598E5
:1009E00000F0F0F9464600F0BBF93C46BBE5064690
:1009F00052E64FF0000905E6BA467EE637467CE649
:100A00005C22002000220020A086010070B50F4B60
:100A10001B780133DBB2012B0C4611D80C4D296831
:100A20004FF47A730E6AA2FB03320146224628462F
:100A3000B047844204D1074B00221A70012070BDD8
:100A40004FF4FA7000F0EAFE0020F8E710220020D0
:100A5000082600209423002007B500230246012128
:100A60000DF107008DF80730FFF7D0FF20B19DF89A
:100A7000070003B05DF804FB4FF0FF30F9E700001A
:100A80000A4608B50421FFF7C1FF80F00100C0B29B
:100A9000404208BD30B4054C2368DD69044B0A466A
:100AA000AC460146204630BC604700BF0826002007
:100AB000A086010070B501F0D1F9094E094D3080D2
:100AC000002428683388834208D901F0C1F92B68D3
:100AD00004440133B4F5404F2B60F2D370BD00BF26
:100AE000962300206823002001F066BA00F1006020
:100AF00000F540400068704700F10060920000F58A
:100B0000404001F0F1B90000054B1A68054B1B8805
:100B10009B1A834202D9104401F09AB90020704711
:100B2000682300209623002038B5084D044629B1DB
:100B300028682044BDE8384001F0AAB9286820445C
:100B400001F08EF90028F3D038BD00BF68230020E3
:100B500010F003030AD1B0F5047F05D200F1005074
:100B6000A0F51040D0F80038184670470023FBE786
:100B700000F10050A0F51040D0F8100A70470000B6
:100B8000064991F8243033B10023086A81F82430F3
:100B90000822FFF7B1BF0120704700BF6C2300207F
:100BA000014B1868704700BF002004E070B5194B76
:100BB0001D68194B0138C5F30B0408442D0C0422A1
:100BC0001E88A6420BD15C680A46013C824213464D
:100BD0000FD214F9016F4EB102F8016BF6E7013A3A
:100BE00003F10803ECD181420B4602D22C2203F818
:100BF000012B0A4A05241688AE4204D1984284BFCC
:100C0000967803F8016B013C02F10402F3D1581A03
:100C100070BD00BF002004E0943400088034000858
:100C2000022802BF024B4FF000529A61704700BF8A
:100C300000000240022802BF024B4FF400529A61AA
:100C4000704700BF00000240022801BF024A5369FA
:100C500083F40053536170470000024070B50446AE
:100C60004FF47A764CB1412C254628BF412506FB2E
:100C700005F000F0D3FD641BF4E770BD10B5002350
:100C8000934203D0CC5CC4540133F9E710BD00009B
:100C900010B5013810F9013F3BB191F900409C4279
:100CA00003D11AB10131013AF4E71AB191F90020E8
:100CB000981A10BD1046FCE703460246D01A12F9F6
:100CC000011B0029FAD1704702440346934202D027
:100CD00003F8011BFAE770472DE9F8431F4D14464E
:100CE00095F824200746884652BBDFF870909CB3E5
:100CF00095F824302BB92022FF2148462F62FFF7B8
:100D0000E3FF95F82400C0F10802A24228BF224662
:100D1000D6B24146920005EB8000FFF7AFFF95F891
:100D20002430A41B1E44F6B2082E17449044E4B2AB
:100D300085F82460DBD1FFF723FF0028D7D108E036
:100D40002B6A03EB82038342CFD0FFF719FF002801
:100D5000CBD10020BDE8F8830120FBE76C23002005
:100D6000024B1A78024B1A70704700BF9423002080
:100D70001022002010B5104C104800F0B5F82146A4
:100D80000E4800F0DDF82468626DD2F8043843F0B4
:100D90000203C2F804384FF47A70FFF75FFF084986
:100DA000204600F0D3F9626DD2F8043823F0020334
:100DB000C2F8043810BD00BF6035000808260020C6
:100DC000683500087047000030B5094D0A4491426B
:100DD0000DD011F8013B5840082340F30004013BBB
:100DE0002C4013F0FF0384EA5000F6D1EFE730BD4A
:100DF0002083B8ED026843681143016003B11847CE
:100E00007047000013B5446BD4F894341A68117815
:100E1000042915D1217C022912D1197912890123C3
:100E20008B4013420CD101A904F14C0001F0F8FEF3
:100E3000D4F89444019B21790246206800F0D0F94F
:100E400002B010BD143001F07BBE00004FF0FF3344
:100E5000143001F075BE00004C3001F04DBF0000B1
:100E60004FF0FF334C3001F047BF0000143001F069
:100E700049BE00004FF0FF31143001F043BE0000C6
:100E80004C3001F019BF00004FF0FF324C3001F040
:100E900013BF00000020704710B5D0F894341A68D2
:100EA00011780429044617D1017C022914D15979FB
:100EB000528901238B4013420ED1143001F0DCFD26
:100EC000024648B1D4F894444FF4807361792068A5
:100ED000BDE8104000F072B910BD0000406BFFF794
:100EE000DBBF0000704700007FB5124B036000239A
:100EF0004360C0E90233012502260F4B0574044606
:100F00000290019300F18402294600964FF4807309
:100F1000143001F08DFD094B0294CDE9006304F516
:100F200023724FF48073294604F14C0001F054FE03
:100F300004B070BDB4340008DD0E0008050E0008D2
:100F40000B68302282F311880A7903EB82029061E8
:100F50004A79093243F822008A7912B103EB8203FD
:100F600098610223C0F894140374002080F3118860
:100F70007047000038B5037F044613B190F8543031
:100F8000ABB9201D01250221FFF734FF04F1140045
:100F900025776FF0010100F069FC84F8545004F1EA
:100FA0004C006FF00101BDE8384000F05FBC38BD77
:100FB00010B5012104460430FFF71CFF00232377FE
:100FC00084F8543010BD000038B5044600251430B4
:100FD00001F046FD04F14C00257701F015FE201DBF
:100FE00084F854500121FFF705FF2046BDE8384042
:100FF000FFF752BF90F8443003F06003202B07D175
:1010000090F84520212A4FF0000303D81F2A06D864
:1010100000207047222AFBD1C0E90E3303E0034AC7
:1010200082630722C26303640120704711220020FB
:1010300037B5D0F894341A681178042904461AD1C7
:10104000017C022917D11979128901238B4013429F
:1010500011D100F14C05284601F096FE58B101A9C6
:10106000284601F0DDFDD4F89444019B2179024625
:10107000206800F0B5F803B030BD0000F0B500EB1B
:10108000810385B09E6904460D46FEB1302383F38B
:10109000118804EB8507301D0821FFF7ABFEFB68C4
:1010A0005B691B6806F14C001BB1019001F0C6FDA5
:1010B000019803A901F0B4FD024648B1039B2946FB
:1010C000204600F08DF8002383F3118805B0F0BDB1
:1010D000FB685A691268002AF5D01B8A013B13404D
:1010E000F1D104F14402EAE7093138B550F8214062
:1010F000DCB1302383F31188D4F894241368527937
:1011000003EB8203DB689B695D6845B104216018CD
:10111000FFF770FE294604F1140001F0B7FC2046E9
:10112000FFF7BAFE002383F3118838BD7047000033
:1011300001F016B8012303700023C0E90133C36135
:1011400083620362C36243620363704738B5044637
:10115000302383F311880025C0E90355C0E9055504
:10116000416001F00DF80223237085F311882846B1
:1011700038BD000070B500EB810305465069DA60A8
:101180000E46144618B110220021FFF79DFDA069FC
:1011900018B110220021FFF797FD31462846BDE81F
:1011A000704001F0B7B80000826802F0011282605E
:1011B0000022C0E90422826101F038B9F0B400EBEA
:1011C00081044789E4680125A4698D403D43458138
:1011D00023600023A2606360F0BC01F053B90000FB
:1011E000F0B400EB81040789E468012564698D404F
:1011F0003D43058123600023A2606360F0BC01F0E1
:10120000CDB9000070B50223002504460370C0E983
:101210000255C0E90455C564856180F8345001F079
:1012200015F863681B6823B129462046BDE8704065
:10123000184770BD0378052B10B504460AD080F816
:1012400050300523037043681B680BB10421984795
:101250000023A36010BD00000178052906D190F895
:101260005020436802701B6803B1184770470000A4
:1012700070B590F83430044613B1002380F8343050
:1012800004F14402204601F0F3F863689B68B3B9A7
:1012900094F8443013F0600535D00021204601F069
:1012A00093FB0021204601F085FB63681B6813B1A6
:1012B000062120469847062384F8343070BD204626
:1012C00098470028E4D0B4F84A30E26B9A4288BFCD
:1012D000E36394F94430E56B002B4FF0300380F268
:1012E0000381002D00F0F280092284F8342083F37A
:1012F00011880021D4E90E232046FFF771FF002357
:1013000083F31188DAE794F8452003F07F0343EA7A
:10131000022340F20232934200F0C58021D8B3F597
:10132000807F48D00DD8012B3FD0022B00F0938056
:10133000002BB2D104F14C02A2630222E2632364C7
:10134000C1E7B3F5817F00F09B80B3F5407FA4D166
:1013500094F84630012BA0D1B4F84C3043F002038E
:1013600032E0B3F5006F4DD017D8B3F5A06F31D090
:10137000A3F5C063012B90D8636894F846205E689B
:1013800094F84710B4F848302046B047002884D07D
:101390004368A3630368E3631AE0B3F5106F36D0C4
:1013A00040F6024293427FF478AF5C4BA363022382
:1013B000E3630023C3E794F84630012B7FF46DAF5D
:1013C000B4F84C3023F00203C4E90E55A4F84C30B5
:1013D000256478E7B4F84430B3F5A06F0ED194F8E3
:1013E000463084F84E30204600F088FF63681B6862
:1013F00013B1012120469847032323700023C4E939
:101400000E339CE704F14F03A3630123C3E7237862
:10141000042B10D1302383F311882046FFF7C4FE3C
:1014200085F311880321636884F84F5021701B688D
:101430000BB12046984794F84630002BDED084F854
:101440004F300423237063681B68002BD6D0022121
:1014500020469847D2E794F848301D0603F00F0164
:1014600020460AD500F0F6FF012804D002287FF4B8
:1014700014AF2B4B9AE72B4B98E700F0DDFFF3E717
:1014800094F84630002B7FF408AF94F8483013F0FE
:101490000F01B3D01A06204602D501F0A9FAADE734
:1014A00001F09CFAAAE794F84630002B7FF4F5AEE1
:1014B00094F8483013F00F01A0D01B06204602D547
:1014C00001F082FA9AE701F075FA97E7142284F89E
:1014D000342083F311882B462A4629462046FFF7FD
:1014E0006DFE85F31188E9E65DB1152284F834209C
:1014F00083F311880021D4E90E232046FFF75EFE16
:10150000FDE60B2284F8342083F311882B462A460B
:1015100029462046FFF764FEE3E700BFE4340008F5
:10152000DC340008E034000838B590F83430044664
:10153000002B3ED0063BDAB20F2A34D80F2B32D81C
:10154000DFE803F0373131082232313131313131C6
:1015500031313737C56BB0F84A309D4214D2C36879
:101560001B8AB5FBF3F203FB12556DB9302383F3ED
:1015700011882B462A462946FFF732FE85F311884B
:101580000A2384F834300EE0142384F834303023F6
:1015900083F3118800231A4619462046FFF70EFEF2
:1015A000002383F3118838BD036C03B198470023EF
:1015B000E7E70021204601F007FA0021204601F06C
:1015C000F9F963681B6813B1062120469847062382
:1015D000D7E7000010B590F83430142B044629D01A
:1015E00017D8062B05D001D81BB110BD093B022B23
:1015F000FBD80021204601F0E7F90021204601F048
:10160000D9F963681B6813B1062120469847062361
:1016100019E0152BE9D10B2380F83430302383F304
:10162000118800231A461946FFF7DAFD002383F3D9
:101630001188DAE7C3689B695B68002BD5D1036C1E
:1016400003B19847002384F83430CEE700230375B4
:10165000826803691B6899689142FBD25A680360EB
:101660004260106058607047002303758268036908
:101670001B6899689142FBD85A6803604260106009
:101680005860704708B50846302383F311880B7DF6
:10169000032B05D0042B0DD02BB983F3118808BD83
:1016A0008B6900221A604FF0FF338361FFF7CEFF92
:1016B0000023F2E7D1E9003213605A60F3E700003B
:1016C000FFF7C4BF054BD9680875186802681A602F
:1016D000536001220275D860FEF714BE98230020E3
:1016E00030B50C4BDD684B1C87B004460FD02B4641
:1016F000094A684600F04EF92046FFF7E3FF009BD9
:1017000013B1684600F050F9A86907B030BDFFF783
:10171000D9FFF9E79823002085160008044B1A68C2
:10172000DB6890689B68984294BF00200120704756
:1017300098230020084B10B51C68D86822681A60EE
:10174000536001222275DC60FFF78EFF01462046C0
:10175000BDE81040FEF7D6BD9823002038B5074CF1
:1017600007490848012300252370656001F044FB08
:101770000223237085F3118838BD00BF00260020A6
:10178000EC3400089823002000F044B9034A516863
:1017900053685B1A9842FBD8704700BF001000E006
:1017A0008B60022308618B82084670478368A3F12F
:1017B000840243F8142C026943F8442C426943F82C
:1017C000402C094A43F8242CC26843F8182C022202
:1017D00003F80C2C002203F80B2C044A43F8102CBD
:1017E000A3F12000704700BF1D03000898230020CC
:1017F00008B5FFF7DBFFBDE80840FFF761BF000059
:10180000024BDB6898610F20FFF75CBF9823002034
:10181000302383F31188FFF7F3BF000008B50146BA
:10182000302383F311880820FFF75AFF002383F346
:10183000118808BD064BDB6839B1426818605A60F0
:10184000136043600420FFF74BBF4FF0FF30704739
:10185000982300200368984206D01A6802605060FE
:1018600099611846FFF72CBF7047000038B5044651
:101870000D462068844200D138BD036823605C6057
:101880008561FFF71DFFF4E710B503689C68A2426D
:101890000CD85C688A600B604C6021605960996864
:1018A0008A1A9A604FF0FF33836010BD1B68121BC9
:1018B000ECE700000A2938BF0A2170B504460D463E
:1018C0000A26601901F092FA01F07EFA041BA54283
:1018D00003D8751C2E460446F3E70A2E04D9BDE84A
:1018E0007040012001F0C8BA70BD0000F8B5144B7B
:1018F0000D46D96103F1100141600A2A196982601D
:1019000038BF0A22016048601861A818144601F027
:101910005FFA0A2701F058FA431BA342064606D392
:101920007C1C281901F062FA27463546F2E70A2F97
:1019300004D9BDE8F840012001F09EBAF8BD00BF0F
:1019400098230020F8B506460D4601F03DFA0F4AEF
:10195000134653F8107F9F4206D12A46014630466F
:10196000BDE8F840FFF7C2BFD169BB68441A2C1923
:1019700028BF2C46A34202D92946FFF79BFF2246E7
:1019800031460348BDE8F840FFF77EBF98230020AA
:10199000A823002010B4C0E9032300235DF8044B02
:1019A0004361FFF7CFBF000010B5194C236998427F
:1019B0000DD0D0E90032816813605A609A680A44F9
:1019C0009A60002303604FF0FF33A36110BD2346EC
:1019D000026843F8102F53600022026022699A4285
:1019E00003D1BDE8104001F0FBB9936881680B4456
:1019F000936001F0E9F92269E1699268441AA24210
:101A0000E4D91144BDE81040091AFFF753BF00BFE5
:101A1000982300202DE9F047DFF8BC8008F110077B
:101A20002C4ED8F8105001F0CFF9D8F81C40AA6815
:101A3000031B9A423ED81444D5E900324FF0000906
:101A4000C8F81C4013605A60C5F80090D8F81030F0
:101A5000B34201D101F0C4F989F31188D5E903310A
:101A600028469847302383F311886B69002BD8D020
:101A700001F0AAF96A69A0EB04094A4582460DD231
:101A8000022001F0F9F90022D8F81030B34208D151
:101A900051462846BDE8F047FFF728BF121A2244F6
:101AA000F2E712EB090938BF4A4629463846FFF7E4
:101AB000EBFEB5E7D8F81030B34208D01444211A31
:101AC000C8F81C00A960BDE8F047FFF7F3BEBDE809
:101AD000F08700BFA8230020982300200020704733
:101AE000FEE70000704700004FF0FF307047000035
:101AF00002290CD0032904D00129074818BF00206F
:101B00007047032A05D8054800EBC2007047044817
:101B100070470020704700BFC43500082022002015
:101B20007835000870B59AB00546084601A91446F4
:101B300000F0C2F801A8FFF7BFF8431C5B00C5E93D
:101B400000340022237003236370C6B201AB023459
:101B50001046D1B28E4204F1020401D81AB070BD11
:101B600013F8011B04F8021C04F8010C0132F0E721
:101B700008B5302383F311880348FFF759FA00238F
:101B800083F3118808BD00BF0826002090F8443078
:101B900003F01F02012A07D190F845200B2A03D138
:101BA0000023C0E90E3315E003F06003202B08D1B9
:101BB000B0F848302BB990F84520212A03D81F2AC5
:101BC00004D8FFF717BA222AEBD0FAE7034A826358
:101BD0000722C26303640120704700BF182200205F
:101BE00007B5052917D8DFE801F0191603191920E0
:101BF000302383F31188104A01900121FFF7BAFACC
:101C000001980E4A0221FFF7B5FA0D48FFF7DCF9FB
:101C1000002383F3118803B05DF804FB302383F3C2
:101C200011880748FFF7A6F9F2E7302383F31188FC
:101C30000348FFF7BDF9EBE7183500083C3500080D
:101C40000826002038B50C4D0C4C0D492A4604F1ED
:101C50000800FFF767FF05F1CA0204F11000094907
:101C6000FFF760FF05F5CA7204F118000649BDE8E8
:101C70003840FFF757BF00BFD02A002020220020A5
:101C8000F8340008023500080D35000870B5044628
:101C900008460D46FFF710F8C6B220460134037817
:101CA0000BB9184670BD32462946FEF7F1FF0028F1
:101CB000F3D10120F6E700002DE9F84F05460C4668
:101CC000FEF7FAFF2B49C6B22846FFF7DFFF08B13F
:101CD0000536F6B228492846FFF7D8FF08B1103676
:101CE000F6B2632E0DD8DFF88C80DFF88C90234F8E
:101CF000DFF890A0DFF890B02E7846B92670BDE8E6
:101D0000F88F29462046BDE8F84F01F09BBB252EF1
:101D10002BD1072241462846FEF7BAFF58B9DBF817
:101D200000302360DBF804306360DBF80830A36028
:101D300007350C34E0E7082249462846FEF7A8FF9D
:101D400098B90F4BA21C197809090232C95D02F833
:101D5000041C13F8011B01F00F015345C95D02F883
:101D6000031CF0D118340835C6E704F8016B0135BF
:101D7000C2E700BFE43500080D350008F93500085A
:101D8000107AFF1F1C7AFF1FEC350008BFF34F8F3E
:101D9000024AD368DB03FCD4704700BF003C02401A
:101DA00008B5094B1B7873B9FFF7F0FF074B1A69A9
:101DB000002ABFBF064A5A6002F188325A601A6888
:101DC00022F480621A6008BD2E2D0020003C0240E3
:101DD0002301674508B50B4B1B7893B9FFF7D6FF76
:101DE000094B1A6942F000421A611A6842F48052A3
:101DF0001A601A6822F480521A601A6842F48062EB
:101E00001A6008BD2E2D0020003C02400B28F0B5C2
:101E100016D80C4C0C4923787BB90C4D0E460C237C
:101E20004FF0006255F8047B46F8042B013B13F099
:101E3000FF033A44F6D10123237051F82000F0BD8E
:101E40000020FCE7602D0020302D00200C3600081B
:101E5000014B53F8200070470C3600080C207047E7
:101E60000B2810B5044601D9002010BDFFF7CEFFA6
:101E7000064B53F824301844C21A0BB90120F4E77A
:101E800012680132F0D1043BF6E700BF0C360008BF
:101E90000B2810B5044621D8FFF778FFFFF780FF25
:101EA0000F4AF323D360C300DBB243F4007343F063
:101EB00002031361136943F480331361FFF766FF74
:101EC000FFF7A4FF074B53F8241000F0D9F8FFF7F1
:101ED00081FF2046BDE81040FFF7C2BF002010BDC3
:101EE000003C02400C360008F8B512F0010314461D
:101EF00042D18218B2F1016F57D82D4B1B6813F0F5
:101F0000010352D02B4DFFF74BFFF323EB60FFF79C
:101F10003DFF40F20127032C15D824F00104661878
:101F2000244C401A40F20117B142236900EB01052D
:101F300024D123F001032361FFF74CFF0120F8BDFA
:101F4000043C0430E7E78307E7D12B6923F44073AF
:101F50002B612B693B432B6151F8046B0660BFF387
:101F60004F8FFFF713FF03689E42E9D02B6923F0E0
:101F700001032B61FFF72EFF0020E0E723F44073FD
:101F8000236123693B4323610B882B80BFF34F8F71
:101F9000FFF7FCFE2D8831F8023BADB2AB42C3D057
:101FA000236923F001032361E4E71846C7E700BF74
:101FB00000380240003C0240084908B50B7828B1BF
:101FC0001BB9FFF7EDFE01230B7008BD002BFCD001
:101FD000BDE808400870FFF7FDBE00BF2E2D0020B1
:101FE00010B50244064BD2B2904200D110BD441C41
:101FF00000B253F8200041F8040BE0B2F4E700BF50
:10200000502800400F4B30B51C6F240407D41C6FC0
:1020100044F400741C671C6F44F400441C670A4CB1
:10202000236843F4807323600244084BD2B2904289
:1020300000D130BD441C00B251F8045B43F820507D
:10204000E0B2F4E700380240007000405028004041
:1020500007B5012201A90020FFF7C2FF019803B0D4
:102060005DF804FB13B50446FFF7F2FFA04205D06C
:10207000012201A900200194FFF7C4FF02B010BDA6
:1020800070470000034B1A681AB9034AD2F8742843
:102090001A607047642D00200030024008B5FFF739
:1020A000F1FF024B1868C0F3407008BD642D00209A
:1020B00070470000FEE700000A4B0B480B4A9042B5
:1020C0000BD30B4BDA1C121AC11E22F003028B42F7
:1020D00038BF00220021FEF7F7BD53F8041B40F87B
:1020E000041BECE7B8370008602E0020602E0020AB
:1020F000602E002070B5D0E915439E6800224FF095
:10210000FF3504EB42135101D3F800090028BEBF8C
:10211000D3F8000940F08040C3F80009D3F8000B61
:102120000028BEBFD3F8000B40F08040C3F8000B7E
:10213000013263189642C3F80859C3F8085BE0D22D
:102140004FF00113C4F81C3870BD0000890141F044
:102150002001016103699B06FCD41220FFF716BB26
:1021600010B5054C2046FEF7E5FF4FF0A043636530
:10217000024BA36510BD00BF682D0020603600082B
:1021800070B50378012B054650D12A4B446D984217
:102190001BD1294B5A6B42F080025A635A6D42F0B0
:1021A00080025A655A6D5A6942F080025A615A6932
:1021B00022F080025A610E2143205B6900F022FC6C
:1021C0001E4BE3601E4BC4F800380023C4F8003EE9
:1021D000C02323606E6D4FF40413A3633369002B97
:1021E000FCDA012333610C20FFF7D0FA3369DB07F7
:1021F000FCD41220FFF7CAFA3369002BFCDA002660
:10220000A6602846FFF776FF6B68C4F81068DB68A5
:10221000C4F81468C4F81C684BB90A4BA3614FF0AA
:10222000FF336361A36843F00103A36070BD064BF5
:10223000F4E700BF682D0020003802404014004041
:1022400003002002003C30C0083C30C0F8B5446DAB
:10225000054600212046FFF779FFA96D00234FF0C6
:1022600001128F68C4F834384FF00066C4F81C2897
:102270004FF0FF3004EB431201339F42C2F8006974
:10228000C2F8006BC2F80809C2F8080BF2D20B685A
:102290006A6DEB65636210231361166916F0100610
:1022A000FBD11220FFF772FAD4F8003823F4FE6352
:1022B000C4F80038A36943F4402343F01003A3613A
:1022C0000923C4F81038C4F814380A4BEB604FF0F7
:1022D000C043C4F8103B084BC4F8003BC4F8106975
:1022E000C4F80039EB6D03F1100243F48013EA6582
:1022F000A362F8BD3C36000840800010426D90F8A3
:102300004E10D2F8003823F4FE6343EA0113C2F8FA
:10231000003870472DE9F84300EB8103456DDA681A
:10232000166806F00306731E022B05EB41130C46DC
:1023300080460FFA81F94FEA41104FF00001C3F8CF
:10234000101B4FF0010104F1100398BFB60401FA0D
:1023500003F391698EBF334E06F1805606F50046B1
:1023600000293AD0578A04F15801490137436F5088
:10237000D5F81C180B43C5F81C382B180021C3F8DE
:10238000101953690127611EA7409BB3138A928BD2
:102390009B08012A88BF5343D8F85C20981842EA6A
:1023A000034301F1400205EB8202C8F85C002146BC
:1023B00053602846FFF7CAFE08EB8900C3681B8AF2
:1023C00043EA8453483464011E432E51D5F81C3827
:1023D0001F43C5F81C78BDE8F88305EB4917D7F80B
:1023E000001B21F40041C7F8001BD5F81C1821EA96
:1023F0000303C0E704F13F0305EB83030A4A5A6075
:1024000028462146FFF7A2FE05EB4910D0F8003917
:1024100023F40043C0F80039D5F81C3823EA070735
:10242000D7E700BF0080001000040002826D126830
:10243000C265FFF75FBE00005831436D49015B582C
:1024400013F4004004D013F4001F0CBF022001203D
:10245000704700004831436D49015B5813F4004058
:1024600004D013F4001F0CBF0220012070470000AD
:1024700000EB8101CB68196A0B6813604B685360ED
:102480007047000000EB810330B5DD68AA6913686E
:10249000D36019B9402B84BF402313606B8A146842
:1024A000426D1C44013CB4FBF3F46343033323F05B
:1024B000030302EB411043EAC44343F0C043C0F8B6
:1024C000103B2B6803F00303012B09B20ED1D2F8A5
:1024D000083802EB411013F4807FD0F8003B14BFA2
:1024E00043F0805343F00053C0F8003B02EB41122D
:1024F000D2F8003B43F00443C2F8003B30BD00007B
:102500002DE9F041244D6E6D06EB40130446D3F8DF
:10251000087BC3F8087B38070AD5D6F814381907A2
:1025200006D505EB84032146DB6828465B6898479F
:10253000FA071FD5D6F81438DB071BD505EB840343
:10254000D968CCB98B69488A5A68B2FBF0F600FBAF
:1025500016228AB91868DA6890420DD2121AC3E9B5
:102560000024302383F311880B482146FFF78AFFAC
:1025700084F31188BDE8F081012303FA04F26B892A
:1025800023EA02036B81CB68002BF3D0214602487B
:10259000BDE8F041184700BF682D002000EB810323
:1025A00070B5DD68436D6C692668E6604A0156BB0C
:1025B0001A444FF40020C2F810092A6802F00302FE
:1025C000012A0AB20ED1D3F8080803EB421410F422
:1025D000807FD4F8000914BF40F0805040F00050D4
:1025E000C4F8000903EB4212D2F8000940F004409D
:1025F000C2F80009D3F83408012202FA01F10143BC
:10260000C3F8341870BD19B9402E84BF4020206033
:1026100020682E8A8419013CB4FBF6F440EAC440D9
:1026200040F000501A44C6E72DE9F8433B4D6E6D6B
:1026300006EB40130446D3F80889C3F8088918F05C
:10264000010F4FEA40171AD0D6F81038DB0716D51D
:1026500005EB8003D9684B691868DA68904230D27C
:10266000121A4FF000091A60C3F80490302383F364
:10267000118821462846FFF791FF89F3118818F049
:10268000800F1CD0D6F834380126A640334216D02D
:1026900005EB84036D6DD3F80CC0DCF81420013415
:1026A000E4B2D2F800E005EB04342F4451687145E0
:1026B00015D3D5F8343823EA0606C5F83468BDE8E2
:1026C000F883012303FA04F22B8923EA02032B8106
:1026D0008B68002BD3D0214628469847CFE7BCF81B
:1026E0001000AEEB0103834228BF0346D7F8180958
:1026F00080B2B3EB800FE2D89068A0F1040959F8DA
:10270000048FC4F80080A0EB09089844B8F1040FC6
:10271000F5D818440B4490605360C7E7682D00203B
:102720002DE9F74FA24C656D6E69AB691E4016F43A
:1027300080586E6107D02046FEF764FD03B0BDE807
:10274000F04F00F047BC002E12DAD5F8003E984852
:102750009B071EBFD5F8003E23F00303C5F8003EDB
:10276000D5F8043823F00103C5F80438FEF774FDEA
:10277000370505D58E48FFF7BDFC8D48FEF75AFD9D
:10278000B0040CD5D5F8083813F0060FEB6823F425
:1027900070530CBF43F4105343F4A053EB60310764
:1027A0001BD56368DB681BB9AB6923F00803AB6119
:1027B0002378052B0CD1D5F8003E7D489A071EBF23
:1027C000D5F8003E23F00303C5F8003EFEF744FDB4
:1027D0006368DB680BB176489847F30274D4B7029C
:1027E00027D5D4F85490DFF8C8B100274FF0010A7C
:1027F00009EB4712D2F8003B03F44023B3F5802FD6
:1028000011D1D2F8003B002B0DDA62890AFA07F3E6
:1028100022EA0303638104EB8703DB68DB6813B1FF
:10282000394658469847A36D01379B68FFB29F42CF
:10283000DED9F00617D5676D3A6AC2F30A1002F0C6
:102840000F0302F4F012B2F5802F00F08580B2F58C
:10285000402F08D104EB83030022DB681B6A07F5D5
:10286000805790426AD13003D5F8184813D5E10358
:1028700002D50020FFF744FEA20302D50120FFF796
:102880003FFE630302D50220FFF73AFE270302D57D
:102890000320FFF735FE75037FF550AFE00702D543
:1028A0000020FFF7C1FEA10702D50120FFF7BCFE03
:1028B000620702D50220FFF7B7FE23077FF53EAF80
:1028C0000320FFF7B1FE39E7636DDFF8E4A0019361
:1028D00000274FF00109A36D9B685FFA87FB9B45BA
:1028E0003FF67DAF019B03EB4B13D3F8001901F4C6
:1028F0004021B1F5802F1FD1D3F8001900291BDA30
:10290000D3F8001941F09041C3F80019D3F8001929
:102910000029FBDB5946606DFFF718FC218909FA95
:102920000BF321EA0303238104EB8B03DB689B6831
:1029300013B15946504698470137CCE7910708BF75
:10294000D7F80080072A98BF03F8018B02F1010233
:1029500098BF4FEA182884E7023304EB830207F597
:1029600080575268D2F818C0DCF80820DCE9001C57
:10297000A1EB0C0C002188420AD104EB83046368AC
:102980009B699A6802449A605A6802445A606AE7EE
:1029900011F0030F08BFD7F800808C4588BF02F8FC
:1029A000018B01F1010188BF4FEA1828E3E700BF5E
:1029B000682D0020436D03EB4111D1F8003B43F437
:1029C0000013C1F8003B7047436D03EB4111D1F890
:1029D000003943F40013C1F800397047436D03EB2D
:1029E0004111D1F8003B23F40013C1F8003B7047BC
:1029F000436D03EB4111D1F8003923F40013C1F802
:102A00000039704700F1604303F561430901C9B221
:102A100083F80013012200F01F039A4043099B0032
:102A200003F1604303F56143C3F880211A607047E6
:102A300030B5039C0172043304FB0325C0E906533F
:102A4000049B03630021059BC160C0E90000C0E94D
:102A50000422C0E90842C0E90A11436330BD000006
:102A6000416A0022C0E90411C0E90A22C2606FF085
:102A70000101FEF7FBBE0000D0E90432934201D110
:102A8000C2680AB9181D70470020704703691960B1
:102A9000C2680132C260C269134482690361934211
:102AA00024BF436A03610021FEF7D4BE38B5044653
:102AB0000D46E3683BB16269131D1268A3621344BB
:102AC000E362002007E0237A33B929462046FEF767
:102AD000B1FE0028EDDA38BD6FF00100FBE7000021
:102AE000C368C269013BC36043691344826943619F
:102AF000934224BF436A436100238362036B03B1A3
:102B00001847704770B53023044683F31188866AEE
:102B10003EB9FFF7CBFF054618B186F3118828466A
:102B200070BDA36AE26A13F8015BA362934202D309
:102B30002046FFF7D5FF002383F31188EFE700005D
:102B40002DE9F84F04460E46174698464FF03009D7
:102B500089F311880025AA46D4F828B0BBF1000FEC
:102B600009D141462046FFF7A1FF20B18BF3118820
:102B70002846BDE8F88FD4E90A12A7EB050B521AD4
:102B8000934528BF9346BBF1400F1BD9334601F153
:102B9000400251F8040B43F8040B9142F9D1A36AA7
:102BA00040334036A3624035D4E90A239A4202D327
:102BB0002046FFF795FF8AF31188BD42D8D289F3EA
:102BC0001188C9E730465A46FEF758F8A36A5B44B5
:102BD0005E44A3625D44E7E710B5029C01720433D2
:102BE00003FB0421C0E906130023C0E90A33039B59
:102BF0000363049BC460C0E90000C0E90422C0E98B
:102C00000842436310BD0000026AC260426AC0E924
:102C100004220022C0E90A226FF00101FEF726BE5D
:102C2000D0E904239A4201D1C26822B9184650F86B
:102C3000043B0B60704700231846FAE7C368C2697B
:102C40000133C3604369134482694361934224BFE3
:102C5000436A43610021FEF7FDBD000038B504461C
:102C60000D46E3683BB123691A1DA262E269134471
:102C7000E362002007E0237A33B929462046FEF7B5
:102C8000D9FD0028EDDA38BD6FF00100FBE7000048
:102C900003691960C268013AC260C269134482695B
:102CA0000361934224BF436A036100238362036B81
:102CB00003B118477047000070B530230D46044635
:102CC000114683F31188866A2EB9FFF7C7FF10B14A
:102CD00086F3118870BDA36A1D70A36AE26A01338E
:102CE0009342A36204D3E16920460439FFF7D0FF81
:102CF000002080F31188EDE72DE9F84F04460D46DA
:102D0000904699464FF0300A8AF311880026B34660
:102D1000A76A4FB949462046FFF7A0FF20B187F3C5
:102D200011883046BDE8F88FD4E90A073A1AA8EBB3
:102D30000607974228BF1746402F1BD905F14003CD
:102D400055F8042B40F8042B9D42F9D1A36A403377
:102D5000A3624036D4E90A239A4204D3E1692046AB
:102D60000439FFF795FF8BF311884645D9D28AF3D2
:102D70001188CDE729463A46FDF780FFA36A3B4418
:102D80003D44A3623E44E5E7D0E904239A4217D1CB
:102D9000C3689BB1836A8BB1043B9B1A0ED013604E
:102DA000C368013BC360C3691A44836902619A42E4
:102DB00024BF436A036100238362012318467047DE
:102DC0000023FBE700F030B94FF08043586A7047AA
:102DD0004FF08043002258631A610222DA60704784
:102DE0004FF080430022DA60704700004FF08043CC
:102DF00058637047FEE7000070B51B4B0163002568
:102E0000044686B0586085620E4600F0BFF804F1B3
:102E10001003C4E904334FF0FF33C4E90635C4E9B5
:102E20000044A560E562FFF7CFFF2B460246C4E9E8
:102E3000082304F134010D4A256580232046FEF75E
:102E4000AFFC0123E0600A4A0375009272680192A8
:102E5000B268CDE90223074B6846CDE90435FEF799
:102E6000C7FC06B070BD00BF002600206C3600080D
:102E700071360008F52D0008024AD36A1843D06263
:102E8000704700BF982300204B6843608B688360C5
:102E9000CB68C3600B6943614B6903628B69436212
:102EA0000B6803607047000008B5264B26481A6976
:102EB00040F2FF110A431A611A6922F4FF7222F0EC
:102EC00001021A611A691A6B0A431A631A6D0A43DE
:102ED0001A651E4A1B6D1146FFF7D6FF02F11C0151
:102EE00000F58060FFF7D0FF02F1380100F5806047
:102EF000FFF7CAFF02F1540100F58060FFF7C4FF3D
:102F000002F1700100F58060FFF7BEFF02F18C0155
:102F100000F58060FFF7B8FF02F1A80100F58060BE
:102F2000FFF7B2FF02F1C40100F58060FFF7ACFFCC
:102F300002F1E00100F58060FFF7A6FFBDE8084060
:102F400000F0EEB800380240000002407836000879
:102F500008B500F059FAFEF701FCFFF793F8BDE859
:102F60000840FEF76FBE000070470000EFF30983D2
:102F700005494A6B22F001024A63683383F30988EA
:102F8000002383F31188704700EF00E0302080F3C6
:102F9000118862B60C4B0D4AD96821F4E06109042E
:102FA000090C0A43DA60D3F8FC20094942F0807228
:102FB000C3F8FC200A6842F001020A602022DA7796
:102FC00083F82200704700BF00ED00E00003FA051F
:102FD000001000E010B5302383F311880E4B5B68BE
:102FE00013F4006314D0F1EE103AEFF30984683C57
:102FF0004FF08073E361094BDB6B236684F3098830
:10300000FEF78CFB10B1064BA36110BD054BFBE72F
:1030100083F31188F9E700BF00ED00E000EF00E066
:103020002F030008320300080F4B1A6C42F0010214
:103030001A641A6E42F001021A660C4A1B6E9368FB
:1030400043F0010393604FF0804353229A624FF0A4
:10305000FF32DA6200229A615A63DA605A60012212
:103060005A611A60704700BF00380240002004E037
:103070004FF0804208B51169D3680B40D9B2C943FB
:103080009B07116107D5302383F31188FEF77CFB82
:10309000002383F3118808BD1F4B1A696FEAC252DF
:1030A0006FEAD2521A611A69C2F308021A614FF02C
:1030B000FF301A695A69586100215A6959615A6981
:1030C0001A6A62F080521A621A6A02F080521A6218
:1030D0001A6A5A6A58625A6A59625A6A1A6C42F0F3
:1030E00080521A641A6E42F080521A661A6E0B4AA7
:1030F000106840F480701060186F00F44070B0F5F4
:10310000007F1EBF4FF4803018671967536823F49F
:103110000073536000F054B9003802400070004062
:10312000334B4FF080521A64324A4FF440411160E1
:103130001A6842F001021A601A689107FCD59A6871
:1031400022F003029A602A4B9A6812F00C02FBD11B
:10315000196801F0F90119609A601A6842F4803226
:103160001A601A689203FCD55A6F42F001025A673E
:103170001F4B5A6F9007FCD51F4A5A601A6842F0DD
:1031800080721A601B4A53685904FCD5184B1A68A0
:103190009201FCD5194A9A60194B1A68194B9A4248
:1031A000194B21D1194A1168194A91421CD140F298
:1031B00005121A60144A136803F00F03052BFAD1A5
:1031C0000B4B9A6842F002029A609A6802F00C0275
:1031D000082AFAD15A6C42F480425A645A6E42F478
:1031E00080425A665B6E704740F20572E1E700BFAD
:1031F00000380240007000400854400700948838AE
:10320000002004E011640020003C024000ED00E0DA
:1032100041C20F41074A08B5536903F001035361E6
:1032200023B1054A13680BB150689847BDE80840C0
:10323000FFF7D0BE003C0140E02D0020074A08B552
:10324000536903F00203536123B1054A93680BB13C
:10325000D0689847BDE80840FFF7BCBE003C01407D
:10326000E02D0020074A08B5536903F004035361B9
:1032700023B1054A13690BB150699847BDE808406E
:10328000FFF7A8BE003C0140E02D0020074A08B52A
:10329000536903F00803536123B1054A93690BB1E5
:1032A000D0699847BDE80840FFF794BE003C014054
:1032B000E02D0020074A08B5536903F0100353615D
:1032C00023B1054A136A0BB1506A9847BDE808401C
:1032D000FFF780BE003C0140E02D0020164B10B5EA
:1032E0005C6904F478725A61A30604D5134A936AA0
:1032F0000BB1D06A9847600604D5104A136B0BB126
:10330000506B9847210604D50C4A936B0BB1D06BD8
:103310009847E20504D5094A136C0BB1506C9847E5
:10332000A30504D5054A936C0BB1D06C9847BDE852
:103330001040FFF74FBE00BF003C0140E02D0020D1
:10334000194B10B55C6904F47C425A61620504D5DE
:10335000164A136D0BB1506D9847230504D5134AD7
:10336000936D0BB1D06D9847E00404D50F4A136EEE
:103370000BB1506E9847A10404D50C4A936E0BB163
:10338000D06E9847620404D5084A136F0BB1506F92
:103390009847230404D5054A936F0BB1D06F984723
:1033A000BDE81040FFF716BE003C0140E02D0020B4
:1033B00008B5FFF75DFEBDE80840FFF70BBE000053
:1033C000062108B50846FFF71DFB06210720FFF779
:1033D00019FB06210820FFF715FB06210920FFF73E
:1033E00011FB06210A20FFF70DFB06211720FFF72E
:1033F00009FB06212820FFF705FBBDE8084007214F
:103400001C20FFF7FFBA000008B5FFF745FE00F0EB
:103410000BF8FDF78DFEFDF765FDFFF7A5FDBDE897
:103420000840FFF7CFBC00000023054A19460133CE
:10343000102BC2E9001102F10802F8D1704700BF59
:10344000E02D0020034611F8012B03F8012B002A80
:10345000F9D1704753544D3332463F3F3F005354E8
:103460004D3332463430780053544D333246343283
:10347000780053544D3332463434365858000000E7
:10348000012033000010410001105A0003105900C0
:10349000071031000000000054340008130400003D
:1034A0005E3400081904000068340008210400009C
:1034B0007234000800000000610E00084D0E000884
:1034C000890E0008750E0008810E00086D0E0008B8
:1034D000590E0008450E0008950E00080000000077
:1034E000010000000000000063300000E834000824
:1034F000F0230020002600204172647550696C6F33
:10350000740025424F415244252D424C002553451D
:103510005249414C2500000002000000000000005C
:103520007D100008E910000840004000A02A00209B
:10353000B02A00200200000000000000030000008C
:10354000000000002D110008000000001000000025
:10355000C02A002000000000010000000000000060
:10356000682D002001010200E11B0008F11A00088B
:103570008D1B0008711B0008430000008035000807
:1035800009024300020100C03209040000010202E6
:103590000100052400100105240100010424020299
:1035A0000524060001070582030800FF0904010045
:1035B000020A000000070501024000000705810221
:1035C0004000000012000000CC350008120110017C
:1035D00002000040091241570002010203010000ED
:1035E0000403090425424F4152442500466F786583
:1035F0006572463430357632003031323334353608
:10360000373839414243444546000000004000003D
:1036100000400000004000000040000000000100E9
:103620000000020000000200000002000000020092
:103630000000020000000200000002000000000084
:103640007112000829150008D51500084000400037
:10365000C82D0020C82D002001000000D82D00201A
:103660008000000040010000030000006D61696EF1
:103670000069646C65000000000180060000000025
:10368000AAAAAAAA00010000FFDF000000000000B3
:1036900000A00A000000000100000000AAAAAAAAD7
:1036A00000000001FFFF000000000000000000001B
:1036B0000000001000000000AAAAAAAA0000001042
:1036C000FFFF0000000000000000000000000000FC
:1036D00000000000AAAAAAAA00000000FFFF000044
:1036E00000000000000000000000000000000000DA
:1036F000AAAAAAAA00000000FFFF00000000000024
:10370000000000000000000000000000AAAAAAAA11
:1037100000000000FFFF00000000000000000000AB
:103720000000000000000000AAAAAAAA00000000F1
:10373000FFFF00000000000000000000000000008B
:10374000000000000A00000000000000030000006C
:103750000000000000000000000000000000000069
:103760000000000000000000000000000000000059
:1037700000000000000000008504000000000000C0
:1037800000400F0000000000FF009600000000084D
:10379000009600000000080004000000E03500086A
:1037A0000000000000000000000000000000000019
:1037B0000000000000000000FFFFFFFFFFFFFFFF11
:1037C000FFFFFFFFFFFFFFFFFFFFFFFFFFFFFFFF09
:1037D000FFFFFFFFFFFFFFFFFFFFFFFFFFFFFFFFF9
:1037E000FFFFFFFFFFFFFFFFFFFFFFFFFFFFFFFFE9
:1037F000FFFFFFFFFFFFFFFFFFFFFFFFFFFFFFFFD9
:10C000000006002099D20008E16C09083D6C09087F
:10C01000A96C09083D6C0908756C09089BD20008D9
:10C020009BD200089BD200089BD20008E57D0B083C
:10C030009BD200089BD200089BD200089BD200082C
:10C040009BD200089BD200089BD200089BD200081C
:10C050009BD200089BD2000801900B0829900B0886
:10C0600051900B0879900B08A1900B08313C0B08FC
:10C07000593C0B08853C0B08B13C0B08DD3C0B0818
:10C08000053D0B08313D0B08B53B0B089BD2000862
:10C090009BD200089BD200089BD20008C9900B08D5
:10C0A00015920B0819920B082D920B0831920B0870
:10C0B00035920B0849920B085D920B08BD420B08A4
:10C0C00065440B089BD200089BD200089BD2000855
:10C0D0009BD200089D910B08B1910B08C5910B08EC
:10C0E0002D910B089BD200089BD2000881920B086F
:10C0F00085920B0899920B089D920B085D3D0B08E9
:10C100009BD200089BD2000871920B089BD20008BA
:10C11000D9910B08ED910B089BD200089BD2000827
:10C12000893D0B08B13D0B08DD3D0B08093E0B08AE
:10C13000353E0B089BD200089BD200089BD200081A
:10C140009BD200089BD200089BD2000811850B08E7
:10C150005D3E0B08893E0B08B53E0B0801920B08AB
:10C160009BD200089BD200089BD200089BD20008FB
:10C170009BD200089BD200089BD200089BD20008EB
:10C180009BD200089BD200089BD200089BD20008DB
:10C190009BD200089BD200089BD200089BD20008CB
:10C1A0009BD200089BD200089BD200089BD20008BB
:10C1B0009BD200089BD200089BD200089BD20008AB
:10C1C0009BD200089BD200089BD200089BD200089B
:10C1D0009BD200089BD200089BD200089BD200088B
:10C1E00009F500081D2501082DAC010835FA0108E4
:10C1F000897B020855F003083D780508457E05084F
:10C2000069E90508CD38060891400608C9430608C3
:10C2100081A406081DC30608E958070885C7070852
:10C22000A965090801570A086DB80A0885DE0A08D9
:10C23000D1E90A0875170B083D1D0B080000000026
:10C2400081F0004102E000BF83F0004330B54FEAC7
:10C2500041044FEA430594EA050F08BF90EA020F34
:10C260001FBF54EA000C55EA020C7FEA645C7FEAC7
:10C27000655C00F0E2804FEA5454D4EB5555B8BFEA
:10C280006D420CDD2C4480EA020281EA030382EA5B
:10C29000000083EA010180EA020281EA0303362DED
:10C2A00088BF30BD11F0004F4FEA01314FF4801CC0
:10C2B0004CEA113102D0404261EB410113F0004FD2
:10C2C0004FEA03334CEA133302D0524263EB430389
:10C2D00094EA050F00F0A780A4F10104D5F1200E27
:10C2E0000DDB02FA0EFC22FA05F2801841F1000182
:10C2F00003FA0EF2801843FA05F359410EE0A5F156
:10C3000020050EF1200E012A03FA0EFC28BF4CF086
:10C31000020C43FA05F3C01851EBE37101F000453C
:10C3200007D54FF0000EDCF1000C7EEB00006EEB49
:10C330000101B1F5801F1BD3B1F5001F0CD34908D3
:10C340005FEA30004FEA3C0C04F101044FEA44522A
:10C3500012F5800F80F09A80BCF1004F08BF5FEAB1
:10C36000500C50F1000041EB045141EA050130BD91
:10C370005FEA4C0C404141EB0101013C28BFB1F5A3
:10C38000801FE9D291F0000F04BF01460020B1FAEE
:10C3900081F308BF2033A3F10B03B3F120020CDAC1
:10C3A0000C3208DD02F1140CC2F10C0201FA0CF09F
:10C3B00021FA02F10CE002F11402D8BFC2F1200C04
:10C3C00001FA02F120FA0CFCDCBF41EA0C019040BA
:10C3D000E41AA2BF01EB0451294330BD6FEA040403
:10C3E0001F3C1CDA0C340EDC04F11404C4F12002EE
:10C3F00020FA04F001FA02F340EA030021FA04F300
:10C4000045EA030130BDC4F10C04C4F1200220FA56
:10C4100002F001FA04F340EA0300294630BD21FA94
:10C4200004F0294630BD94F0000F83F4801306BF5A
:10C4300081F480110134013D4EE77FEA645C18BF4E
:10C440007FEA655C29D094EA050F08BF90EA020FE5
:10C4500005D054EA000C04BF1946104630BD91EADD
:10C46000030F1EBF0021002030BD5FEA545C05D1E0
:10C470004000494128BF41F0004130BD14F580041F
:10C480003CBF01F5801130BD01F0004545F0FE4193
:10C4900041F470014FF0000030BD7FEA645C1ABFC8
:10C4A000194610467FEA655C1CBF0B46024650EAFF
:10C4B000013406BF52EA033591EA030F41F400212B
:10C4C00030BD00BF90F0000F04BF0021704730B5B1
:10C4D0004FF4806404F132044FF000054FF0000186
:10C4E00050E700BF90F0000F04BF0021704730B547
:10C4F0004FF4806404F1320410F0004548BF40421C
:10C500004FF000013EE700BF42004FEAE2014FEA70
:10C5100031014FEA02701FBF12F07F4393F07F4F4B
:10C5200081F06051704732F07F4208BF704793F04E
:10C530007F4F04BF41F40021704730B54FF4607461
:10C5400001F0004521F000411CE700BF50EA010264
:10C5500008BF704730B54FF000050AE050EA01020D
:10C5600008BF704730B511F0004502D5404261EB7D
:10C5700041014FF4806404F132045FEA915C3FF4BE
:10C58000D8AE4FF003025FEADC0C18BF03325FEA5B
:10C59000DC0C18BF033202EBDC02C2F1200300FA0C
:10C5A00003FC20FA02F001FA03FE40EA0E0021FA31
:10C5B00002F11444BDE600BF70B54FF0FF0C4CF41F
:10C5C000E06C1CEA11541DBF1CEA135594EA0C0FD1
:10C5D00095EA0C0F00F0DEF82C4481EA030621EA0C
:10C5E0004C5123EA4C5350EA013518BF52EA033547
:10C5F00041F4801143F4801338D0A0FB02CE4FF0F9
:10C600000005E1FB02E506F00042E0FB03E54FF028
:10C610000006E1FB03569CF0000F18BF4EF0010E20
:10C62000A4F1FF04B6F5007F64F5407404D25FEA1C
:10C630004E0E6D4146EB060642EAC62141EA5551CF
:10C640004FEAC52040EA5E504FEACE2EB4F1FD0C11
:10C6500088BFBCF5E06F1ED8BEF1004F08BF5FEA8F
:10C66000500E50F1000041EB045170BD06F0004641
:10C6700046EA010140EA020081EA0301B4EB5C04EE
:10C68000C2BFD4EB0C0541EA045170BD41F48011E6
:10C690004FF0000E013C00F3AB8014F1360FDEBF0B
:10C6A000002001F0004170BDC4F10004203C35DAE7
:10C6B0000C341BDC04F11404C4F1200500FA05F36A
:10C6C00020FA04F001FA05F240EA020001F000420B
:10C6D00021F0004110EBD37021FA04F642EB060181
:10C6E0005EEA430E08BF20EAD37070BDC4F10C04AB
:10C6F000C4F1200500FA04F320FA05F001FA04F26F
:10C7000040EA020001F0004110EBD37041F100015A
:10C710005EEA430E08BF20EAD37070BDC4F1200565
:10C7200000FA05F24EEA020E20FA04F301FA05F2CD
:10C7300043EA020321FA04F001F0004121FA04F275
:10C7400020EA020000EBD3705EEA430E08BF20EA45
:10C75000D37070BD94F0000F0FD101F0004640007F
:10C7600041EB010111F4801F08BF013CF7D041EA01
:10C77000060195F0000F18BF704703F00046520005
:10C7800043EB030313F4801F08BF013DF7D043EAD6
:10C790000603704794EA0C0F0CEA135518BF95EA8C
:10C7A0000C0F0CD050EA410618BF52EA4306D1D113
:10C7B00081EA030101F000414FF0000070BD50EA32
:10C7C000410606BF1046194652EA430619D094EABC
:10C7D0000C0F02D150EA013613D195EA0C0F05D1A6
:10C7E00052EA03361CBF104619460AD181EA0301FA
:10C7F00001F0004141F0FE4141F470014FF00000B2
:10C8000070BD41F0FE4141F4780170BD70B54FF04C
:10C81000FF0C4CF4E06C1CEA11541DBF1CEA1355CC
:10C8200094EA0C0F95EA0C0F00F0A7F8A4EB0504AE
:10C8300081EA030E52EA03354FEA013100F08880A5
:10C840004FEA03334FF0805545EA131343EA12636E
:10C850004FEA022245EA111545EA10654FEA002623
:10C860000EF000419D4208BF964244F1FD0404F5DC
:10C87000407402D25B084FEA3202B61A65EB030538
:10C880005B084FEA32024FF480104FF4002CB6EBF5
:10C89000020E75EB030E22BFB61A754640EA0C0075
:10C8A0005B084FEA3202B6EB020E75EB030E22BFB5
:10C8B000B61A754640EA5C005B084FEA3202B6EBF6
:10C8C000020E75EB030E22BFB61A754640EA9C00B5
:10C8D0005B084FEA3202B6EB020E75EB030E22BF85
:10C8E000B61A754640EADC0055EA060E18D04FEA43
:10C8F000051545EA16754FEA06164FEAC30343EAE3
:10C9000052734FEAC2025FEA1C1CC0D111F4801FAF
:10C910000BD141EA00014FF000004FF0004CB6E7A8
:10C9200011F4801F04BF01430020B4F1FD0C88BF47
:10C93000BCF5E06F3FF6AFAEB5EB030C04BFB6EB52
:10C94000020C5FEA500C50F1000041EB045170BD45
:10C950000EF0004E4EEA113114EB5C04C2BFD4EB72
:10C960000C0541EA045170BD41F480114FF0000EF6
:10C97000013C90E645EA060E8DE60CEA135594EA72
:10C980000C0F08BF95EA0C0F3FF43BAF94EA0C0F75
:10C990000AD150EA01347FF434AF95EA0C0F7FF4EA
:10C9A00025AF104619462CE795EA0C0F06D152EA3E
:10C9B00003353FF4FDAE1046194622E750EA410622
:10C9C00018BF52EA43067FF4C5AE50EA41047FF433
:10C9D0000DAF52EA43057FF4EBAE12E74FF0FF3C98
:10C9E00006E000BF4FF0010C02E000BF4FF0010C69
:10C9F0004DF804CD4FEA410C7FEA6C5C4FEA430CE2
:10CA000018BF7FEA6C5C1BD001B050EA410C0CBF30
:10CA100052EA430C91EA030F02BF90EA020F002092
:10CA2000704710F1000F91EA030F58BF994208BFF9
:10CA300090422CBFD8176FEAE37040F001007047B6
:10CA40004FEA410C7FEA6C5C02D150EA013C07D10D
:10CA50004FEA430C7FEA6C5CD6D152EA033CD3D058
:10CA60005DF8040B704700BF8446104662468C4652
:10CA70001946634600E000BF01B5FFF7B7FF002885
:10CA800048BF10F1000F01BD4DF808EDFFF7F4FFAE
:10CA90000CBF012000205DF808FB00BF4DF808ED39
:10CAA000FFF7EAFF34BF012000205DF808FB00BF5C
:10CAB0004DF808EDFFF7E0FF94BF012000205DF87E
:10CAC00008FB00BF4DF808EDFFF7CEFF94BF012033
:10CAD00000205DF808FB00BF4DF808EDFFF7C4FF2C
:10CAE00034BF012000205DF808FB00BF4FEA410C75
:10CAF0007FEA6C5C02D150EA013C0AD14FEA430C58
:10CB00007FEA6C5C02D152EA033C02D14FF0000094
:10CB100070474FF0010070474FEA410212F50012D2
:10CB200015D211D56FF47873B3EB625212D94FEA74
:10CB3000C12343F0004343EA505311F0004F23FA5E
:10CB400002F018BF404270474FF00000704750EAB3
:10CB5000013005D111F0004008BF6FF00040704770
:10CB60004FF00000704700BF4A0011D212F50012CA
:10CB700011D20DD56FF47873B3EB62520ED44FEA35
:10CB8000C12343F0004343EA505323FA02F07047B5
:10CB90004FF00000704750EA013002D14FF0FF30F3
:10CBA00070474FF0000070474FEA4102B2F1E04396
:10CBB00024BFB3F5001CDCF1FE5C0DD901F0004C84
:10CBC0004FEAC0024CEA5070B2F1004F40EB8300D4
:10CBD00008BF20F00100704711F0804F21D113F100
:10CBE0003872BCBF01F00040704741F480114FEA39
:10CBF0005252C2F11802C2F1200C10FA0CF320FAC2
:10CC000002F018BF40F001004FEAC1234FEAD323DE
:10CC100003FA0CFC40EA0C0023FA02F34FEA430348
:10CC2000CCE77FEA625307D150EA01331EBF4FF0D1
:10CC3000FE4040F44000704701F0004040F0FE40EC
:10CC400040F40000704700BF80F0004002E000BFE9
:10CC500081F0004142001FBF5FEA410392EA030FE7
:10CC60007FEA226C7FEA236C6AD04FEA1262D2EB31
:10CC70001363C1BFD218414048404140B8BF5B4236
:10CC8000192B88BF704710F0004F40F4000020F0CF
:10CC90007F4018BF404211F0004F41F4000121F0E5
:10CCA0007F4118BF494292EA030F3FD0A2F101022F
:10CCB00041FA03FC10EB0C00C3F1200301FA03F16D
:10CCC00000F0004302D5494260EB4000B0F5000F90
:10CCD00013D3B0F1807F06D340084FEA310102F14F
:10CCE0000102FE2A51D2B1F1004F40EBC25008BF01
:10CCF00020F0010040EA03007047490040EB0000CB
:10CD0000013A28BFB0F5000FEDD2B0FA80FCACF1CB
:10CD1000080CB2EB0C0200FA0CF0AABF00EBC250F8
:10CD200052421843BCBFD0401843704792F0000FE6
:10CD300081F4000106BF80F400000132013BB5E739
:10CD40004FEA41037FEA226C18BF7FEA236C21D0AF
:10CD500092EA030F04D092F0000F08BF0846704714
:10CD600090EA010F1CBF0020704712F07F4F04D1E2
:10CD7000400028BF40F00040704712F100723CBFF5
:10CD800000F50000704700F0004343F0FE4040F41F
:10CD9000000070477FEA226216BF08467FEA2363DD
:10CDA0000146420206BF5FEA412390EA010F40F4C8
:10CDB000800070474FF0000304E000BF10F0004314
:10CDC00048BF40425FEA000C08BF704743F09643FB
:10CDD00001464FF000001CE050EA010208BF704716
:10CDE0004FF000030AE000BF50EA010208BF70479D
:10CDF00011F0004302D5404261EB41015FEA010CB2
:10CE000002BF84460146002043F0B64308BFA3F1A9
:10CE10008053A3F50003BCFA8CF2083AA3EBC2538B
:10CE200010DB01FA02FC634400FA02FCC2F12002AA
:10CE3000BCF1004F20FA02F243EB020008BF20F0E1
:10CE40000100704702F1200201FA02FCC2F1200247
:10CE500050EA4C0021FA02F243EB020008BF20EA3C
:10CE6000DC7070477BB972B90029BEBF00204FF05B
:10CE7000004106E008BF00281CBF6FF000414FF0E2
:10CE8000FF3000F007BAADF1080C6DE904CE0029BF
:10CE900009DB002B1ADB00F095F8DDF804E0DDE992
:10CEA000022304B07047404261EB4101002B1BDBC1
:10CEB00000F088F8DDF804E0DDE9022304B0404228
:10CEC00061EB4101524263EB43037047524263EB13
:10CED000430300F077F8DDF804E0DDE9022304B055
:10CEE000404261EB41017047524263EB430300F063
:10CEF00069F8DDF804E0DDE9022304B0524263EB97
:10CF00004303704753B94AB9002908BF00281CBF22
:10CF10004FF0FF314FF0FF3000F0BCB9ADF1080C1D
:10CF20006DE904CE00F04EF8DDF804E0DDE90223FF
:10CF300004B07047430803F05533C01A830803F068
:10CF4000333300F03330184400EB101000F00F3092
:10CF500000EB002000EB0040000E704707EE900A47
:10CF6000F5EEC07AF1EE10FA01D400F00BB8F1EE54
:10CF7000677A08B517EE900A00F004F8404261EBBA
:10CF8000410108BDD0B5FFF7BFFA0C4B00220646A1
:10CF90000F46FFF711FBFFF7E7FD0446FFF792FA94
:10CFA000074B0022FFF708FB02460B463046394686
:10CFB000FFF74AF9FFF7D8FD2146D0BD0000F03D4C
:10CFC0000000F0412DE9F047089D04468E46002BF5
:10CFD0004DD18A42944669D9B2FA82F252B101FA2D
:10CFE00002F3C2F1200120FA01F10CFA02FC41EA3D
:10CFF000030E94404FEA1C48210CBEFBF8F61FFAC2
:10D000008CF708FB16E341EA034306FB07F199425C
:10D010000AD91CEB030306F1FF3080F01F8199420F
:10D0200040F21C81023E63445B1AA4B2B3FBF8F0E9
:10D0300008FB103344EA034400FB07F7A7420AD970
:10D040001CEB040400F1FF3380F00A81A74240F298
:10D0500007816444023840EA0640E41B00261DB103
:10D06000D4400023C5E900433146BDE8F0878B4238
:10D0700009D9002D00F0EF800026C5E900013046F7
:10D080003146BDE8F087B3FA83F6002E4AD18B42D1
:10D0900002D3824200F2F980841A61EB030301207B
:10D0A0009E46002DE0D0C5E9004EDDE702B9FFDE67
:10D0B000B2FA82F2002A40F09280A1EB0C014FEA12
:10D0C0001C471FFA8CFE0126200CB1FBF7F307FB6F
:10D0D000131140EA01410EFB03F0884208D91CEB12
:10D0E000010103F1FF3802D2884200F2CB804346AF
:10D0F000091AA4B2B1FBF7F007FB101144EA01448E
:10D100000EFB00FEA64508D91CEB040400F1FF311C
:10D1100002D2A64500F2BB800846A4EB0E0440EA0A
:10D1200003409CE7C6F12007B34022FA07FC4CEA13
:10D13000030C20FA07F401FA06F31C43F9404FEA06
:10D140001C4900FA06F3B1FBF9F8200C1FFA8CFE1B
:10D1500009FB181140EA014108FB0EF0884202FA6F
:10D1600006F20BD91CEB010108F1FF3A80F0888030
:10D17000884240F28580A8F102086144091AA4B2ED
:10D18000B1FBF9F009FB101144EA014100FB0EFE6E
:10D190008E4508D91CEB010100F1FF346CD28E459D
:10D1A0006AD90238614440EA0840A0FB0294A1EB2E
:10D1B0000E01A142C846A64656D353D05DB1B3EB8B
:10D1C000080261EB0E0101FA07F722FA06F3F140BB
:10D1D0001F43C5E9007100263146BDE8F087C2F162
:10D1E0002003D8400CFA02FC21FA03F391400143DA
:10D1F0004FEA1C471FFA8CFEB3FBF7F007FB103613
:10D200000B0C43EA064300FB0EF69E4204FA02F4BE
:10D2100008D91CEB030300F1FF382FD29E422DD911
:10D22000023863449B1B89B2B3FBF7F607FB163346
:10D2300041EA034106FB0EF38B4208D91CEB0101C6
:10D2400006F1FF3816D28B4214D9023E6144C91A46
:10D2500046EA004638E72E46284605E70646E3E656
:10D260001846F8E64B45A9D2B9EB020864EB0C0E60
:10D270000138A3E74646EAE7204694E74046D1E76F
:10D28000D0467BE7023B614432E7304609E764441D
:10D29000023842E7704700BF02E000F000F8FEE706
:10D2A00072B6374880F30888364880F309883648D4
:10D2B0003649086040F20000CCF200004EF63471AE
:10D2C000CEF200010860BFF34F8FBFF36F8F40F2C3
:10D2D0000000C0F2F0004EF68851CEF20001086066
:10D2E000BFF34F8FBFF36F8F4FF00000E1EE100AD6
:10D2F0004EF63C71CEF200010860062080F31488DF
:10D30000BFF36F8FAAF0CCFDABF016FD4FF0553098
:10D310001F491B4A91423CBF41F8040BFAE71D49E3
:10D32000184A91423CBF41F8040BFAE71A491B4ADC
:10D330001B4B9A423EBF51F8040B42F8040BF8E72E
:10D3400000201849184A91423CBF41F8040BFAE703
:10D35000AAF0AAFDABF044FD144C154DAC4203DA23
:10D3600054F8041B8847F9E702F0BEF8114C124D3F
:10D37000AC4203DA54F8041B8847F9E7AAF092BDDF
:10D38000000600200022002000C0000808ED00E098
:10D39000000000200006002070250E08002200205A
:10D3A000AC2B0020B02B0020D04E0120E0C10008A3
:10D3B0003CC200083CC200083CC200082DE9F04F06
:10D3C0002DED108AC1F80CD0C3689D46BDEC108AC3
:10D3D000BDE8F08F002383F311882846A047002082
:10D3E000A9F052FDFEE7A9F0BFFB00DFFEE7000059
:10D3F00001F0FF01102A2BDB10F0070F08D010F806
:10D40000013B013A8B422DD010F0070F42B3F6D109
:10D41000F0B441EA012141EA014122F007047FF022
:10D4200000070023F0E80256083C85EA010586EA79
:10D43000010685FA47F5A3FA87F586FA47F6A5FAB5
:10D4400087F68EB9EED1F0BC01F0FF0102F00702C1
:10D4500032B110F8013B013A83EA010313B1F8D16C
:10D460000020704701387047002D06BF354603384D
:10D47000073815F0010F07D1013015F4807F02BF86
:10D48000013015F4C03F0130F0BC0138704700BFD7
:10D4900010F8012B11F8013B012A28BF9A42F7D05E
:10D4A000D01A7047034613F8012B002AFBD1181A33
:10D4B0000138704738B50022002304460D46FFF7B7
:10D4C000EDFA28B920462946BDE8384000F00AB8F0
:10D4D000204605F1004100F005F8404261EB4101B2
:10D4E00038BD00BFD0B50C4B002206460F46FFF7F3
:10D4F00063F8FFF739FB0446FEF7E4FF074B002211
:10D50000FFF75AF802460B4630463946FEF79CFEB6
:10D51000FFF72AFB2146D0BD0000F03D0000F0419E
:10D52000036800221B6818477FB503914021054618
:10D5300078F008FF039A18B90124204604B070BDA2
:10D54000134E039296F98231002BF5D05DF0CEF99F
:10D55000437A039A53B95DF0C9F9847A039A2CB9D6
:10D560000C4B4021284678F0F5FEE6E7D6F8D03A95
:10D57000B6F98411B3F906309942DDDD064B00930C
:10D580004021064B284678F0E5FE0024D5E700BF91
:10D59000B84B002078040C0897040C0885040C088C
:10D5A000F0B50D469DB02021044678F0CBFE002852
:10D5B00000F09D804F4E96F98231ABB1D6F8D02A5B
:10D5C000B6F98431B2F90A1003F10A02914203DD7F
:10D5D00040F28D32934207DC474B2A4620212046F9
:10D5E00078F0B8FE002080E096F97131022B05D169
:10D5F000424B2A462021204678F0ACFEB6F8443152
:10D60000A3F57A739BB241F6583293420DD83C4F42
:10D6100096ED6C7AD7F83839D3ED097AB4EEE77A1B
:10D62000F1EE10FA03DD374BD7E7374BD5E796ED30
:10D630006D7AD3ED0B7AB4EEE77AF1EE10FAF2DC04
:10D64000B6F97E31002B01DC304BC6E796F810228C
:10D650000D2A06D80123934013F4215F01D02C4BEF
:10D66000BBE72C480EF0B2FD012806D1D7F84409DB
:10D670007FF05EFE98B101281AD00021602204A834
:10D680000391AEF0D1FB2449D7F84009642303AAE3
:10D690007FF070FA00BB03AB0093204B02E0204BFD
:10D6A0000093204B2A462021204678F053FE99E72C
:10D6B00096F8E43A73B11C4819214AF00DFE48B1BE
:10D6C0001948D6F85C6119214AF02CFE8642D4DD57
:10D6D000164BE5E7164BE3E71649D7F838096423FC
:10D6E00003AA7CF007F90028D5D01DB0F0BD0120B9
:10D6F000FBE700BFB84B0020A0040C08B3040C08E3
:10D70000B86B0020EB040C08DB040C0805050C08C2
:10D710001A050C08E07C002094050C0898050C08FC
:10D720005F050C083A050C08C83800207E050C0877
:10D730006F050C08AA050C0807B5044881F050F9DC
:10D7400000F0010003B05DF804FB00BFD4740020BA
:10D750002DE9F043474F0446D7F8940E0368A5B06F
:10D760001B690D469847814614F0A0FA00218046B7
:10D7700060220CA80B91AEF057FB64230BAA49461C
:10D78000404613F095FD064648B93B4A0BAB294687
:10D79000204678F0E7FF304625B0BDE8F08307F17A
:10D7A000480066F01FFBB9F1000F03D194F91E3059
:10D7B000012B0AD1314811F09FFA80B9304A29462D
:10D7C000204678F0CFFF0026E5E710F0060FE2D004
:10D7D000A7F5005011F090FA08B92A4AEFE703A91B
:10D7E000404613F09BFB28B19DF80D305B0601D538
:10D7F000254AE4E7D7ED687AF5EEC07AF1EE10FA43
:10D800004FF00003C7DD089309930A930DF1200937
:10D8100007AB019305AA06AB04A9CDF800904046DA
:10D8200013F05AFF48462EF029FCD7ED687AB4EE83
:10D83000E70AF1EE10FA01DB144AC0E79DED057A24
:10D84000F4EEC77AF1EE10FA01D8114AB7E79DED70
:10D85000047AF4EEC77AF1EE10FA01D80D4AAEE779
:10D860009DED067AF4EEC77AF1EE10FA93D80A4AE3
:10D87000A5E700BFB84B0020B0050C08B82B00206E
:10D88000B9050C08D0050C08F6050C0804060C08B0
:10D8900019060C082F060C0845060C0808B5064B9F
:10D8A00093F8AD3E9B0704D5044A78F05BFF002057
:10D8B00008BD0120FCE700BFB84B00205C060C0847
:10D8C00070B50C4C0546D4F8940E03685B690E469F
:10D8D000984710B10124204670BDA4F5005011F006
:10D8E0001DFA04460028F5D1034A3146284678F04F
:10D8F00039FFF0E7B84B00206C060C082DE9F04624
:10D90000464ED6F8B83E93F8CB509BB081468A4637
:10D9100065B9434B1B68986A03685B6B984704467C
:10D9200040B9404A5146484678F01CFF28461BB093
:10D93000BDE8F0865CF0DAFF20215DF08FFF58B182
:10D940005CF0D4FF1F215DF089FF88B3364A514651
:10D95000484678F007FF002496F88A3E03F0140347
:10D96000142B05D1314A5146484678F0FBFE00247D
:10D970005146484679F084FD002188424FF060020C
:10D9800002A808BF0C460191AEF04EFAD6F8B80EC8
:10D99000036801AA1B6864219847054680B9244A98
:10D9A00001AB5146484678F0DDFE2C462546BDE7E2
:10D9B0005CF09CFFA5215DF051FF0028C6D1CBE7AC
:10D9C000002CF3D0D9F808303BB9D9F800305146D3
:10D9D0005B6B484698470446E8E751464846FFF7E0
:10D9E000DFFD514607464846FFF758FF3840C4B2AE
:10D9F00051464846FFF798FD514604404846FFF718
:10DA00005FFF51460440484678F0D4FE514604403A
:10DA1000484679F04DFD0440C8E700BFB84B0020F0
:10DA2000E07E002080060C0897060C08B1060C0862
:10DA3000C9060C0808B5FFF761FF054A92F8881E71
:10DA400060F3041182F8881E024A907108BD00BF7D
:10DA5000B84B00209D800020F7B505460F4678F0B2
:10DA6000ADFC044678B10221284678F06BFC0646EE
:10DA700048B1154880F0B4FFC205C0F30723C0F3D6
:10DA8000002403D53446204603B0F0BD9B07F9D5EA
:10DA90000D4880F0B3FF0D4B03F6E803D3ED007A99
:10DAA000F8EEE77A30EE670ADFED097AB0EEC00AE9
:10DAB000B4EEE70AF1EE10FAE4DD064B3A46022135
:10DAC000284678F047FCDEE7D4740020B86B0020CD
:10DAD0000000C842D4060C08F8B504460F4678F09A
:10DAE00009FF10210546204678F02CFC58B120464D
:10DAF000FFF722FE064630B9044B3A461021204675
:10DB000078F028FC35462846F8BD00BFE8060C082A
:10DB100070B505460E4678F0B9FB044678B1802111
:10DB2000284678F00FFC50B1074B93F80D3443B101
:10DB3000064B32468021284678F00CFC0024204613
:10DB400070BD0446FBE700BFB85B0020FC060C0874
:10DB500038B50D4D0446D5F844097FF0E9FB01289E
:10DB600010D0D5F844097FF0E3FB022804D020460A
:10DB7000BDE8384078F08CBB04480EF027FB012844
:10DB8000F5D138BD0020FCE7B86B0020E07C002018
:10DB9000F0B5114C85B0D4F8C83A0093D4F8CC3A1B
:10DBA0000193D4F8D03A02936A46D4F8D43A039356
:10DBB00006460F4679F016FC39460546304678F0A1
:10DBC00023FC94F8883E284060F3C303C3F3C000ED
:10DBD00084F8883E05B0F0BDB84B00202DE9F8432D
:10DBE00006462648DFF8A480DFF8A4900F4666F0CA
:10DBF000F9F80446D8F8940E03681B69984705465F
:10DC000030B914F0060F03D1D8F8C83E022B09D161
:10DC10003946304678F0CAFC054618B9002489F820
:10DC200007400AE039463046FFF792FD04460028D7
:10DC3000F4D02DB9012389F807302046BDE8F883D8
:10DC40000821304678F07EFB0028F3D00C4821F004
:10DC500043FF0028EED00B4B93F8E423B02101FBE7
:10DC60000233B3F8EE21B8F972319A42E2DD064B85
:10DC70003A460821304678F06DFBCFE7004C002093
:10DC8000D82C0020B82B002010070C08B84B00201F
:10DC90009D8000202DE9F3410F46054614F006F85B
:10DCA000804613F0FDF8044640B94F4A012128464A
:10DCB00078F058FD204602B0BDE8F0814B4ED6F812
:10DCC000940E036839469B699847044658B9D6F8BC
:10DCD000940E03681B6C9847454A03460121284669
:10DCE00078F040FDE6E7AB68002BE3D01021284632
:10DCF00078F028FB10B3D8ED937A98ED920A20EED5
:10DD0000270AABF02FFEDFED3B7AB6F9443120EE67
:10DD1000270ADFED397A20EE270A07EE903AF8EE6F
:10DD2000E77AB4EEE70AF1EE10FA07DD334B012291
:10DD30001021284678F00EFB0024BBE7402128463E
:10DD400078F000FB28B3012F1CD0232F1AD0042F0A
:10DD500018D0D6F8D03A2A48B3F9083000EE103A75
:10DD6000B8EEC00A00F0BEFBB5EEC00AF1EE10FA44
:10DD70001DDD244B00930122234B4021284678F0DF
:10DD8000E9FAD9E7D6F8940E0368DB6B98470028C8
:10DD9000DFD01E4B1B68D86A0368DB6998470128EF
:10DDA000014619D11A4A284678F0DCFCC4E7D6F8B7
:10DDB000940E03685B69984730B1D6F8D03AB3F94E
:10DDC0000830002BE5DDD4E7D6F8940E03681B6815
:10DDD00098470B28DDD1F0E73946284602B0BDE868
:10DDE000F04179F04FB800BF20070C08B84B002075
:10DDF00031070C08E02E65420000C84245070C08B8
:10DE0000B82B002097040C084D070C08E07E00207A
:10DE100059070C0870B505460E46FFF799FC084BEC
:10DE20000446D87131462846FFF74AFD314600289E
:10DE3000284608BF002479F0BDF9204070BD00BF1E
:10DE40009D800020F8B54E4F3B78002B40F0958028
:10DE50004C4CD4F8B85E95F8CB5001263E7015B105
:10DE60003B702846F8BD79F0CBFB054630B9464AF1
:10DE70003870137843F001031370F2E752F0D4FBCB
:10DE8000314651F00BFDA4F5005006F07FFC3F4BEE
:10DE90001E710B2645F0DEFF013E45F079FF16F0BE
:10DEA000FF06F7D13A4800F069FF13F0FFFED0F803
:10DEB0000022C4F8E02E90F87C32DA074BD413F03D
:10DEC0006DFA52F0B1FB3C2152F0EAFA04F56A63B4
:10DED00000221A6000212E4800F0E4FF2C4810F0C8
:10DEE0000BFF01462B4884F0EDFC2B4B1B68D86AD6
:10DEF000036801211B689847D4F8B80E03689B6A31
:10DF000098470121D4F8B80E81F024FD52F08CFB23
:10DF10000646D4F8940E03681B68984794F80421C9
:10DF20000146304651F092FE194806F021FC4FF0B0
:10DF3000A1FD4FF0DDF800233B7088F007FF174B81
:10DF4000C3F85009B4F88A3E23F4087343F0200361
:10DF5000A4F88A3E85E79B07BCD431460C4804F000
:10DF6000D5FC0F4880F04AFDDFED0E7A20EE270A3F
:10DF700004F56A6383ED000AACE7002571E700BF92
:10DF8000B02B0020B84B0020BC8000209D800020DA
:10DF9000B82B002024550020E07E0020B86B002024
:10DFA000D47400200AD7233C2DE9F043374DD5F82F
:10DFB000B83E93F8CB3087B0002B64D062B1012912
:10DFC00001D0232908D195F9883E002B04DB0024D9
:10DFD000204607B0BDE8F08379F0BEFB0446002878
:10DFE000F5D013F063FE07461AF0A8FB80463846CA
:10DFF00012F068FCD8B198F92430022B17D1002612
:10E000004FF00009F1B203AA38460191CDF80C9007
:10E01000CDF81090CDF8149012F0E6FF019918B1E8
:10E0200003AA40461AF03AF80136032EEAD11848FE
:10E03000012106F015FE1648012106F047FD0021DA
:10E04000D5F8B80E81F086FC124830F0FBFC52F097
:10E05000EBFA002151F022FC0F4B1B68D86A0368D1
:10E0600000211B68984795F88A3ED5F8941E0B4806
:10E070006FF3451385F88A3E0B1A594259413C30DB
:10E0800087F084F8A4E70124A2E700BFB84B002082
:10E09000B82B002014770020E07E0020B07800200C
:10E0A00010B5064CD4F8940E03685B6A984718B113
:10E0B000D4F8B83E93F8CB0010BD00BFB84B002099
:10E0C00030B52DED028B89B00C46B0EE408AFFF7DB
:10E0D000E7FF0546002838D0B4EE488AF1EE10FA82
:10E0E0007CBFDFED1C8ADFED1C7A226863689FED40
:10E0F0001A0A68BFDFED198A029278BF68EE288A93
:10E1000002A878BF68EEA78AD4ED027A0393F1EEF5
:10E11000677ACDED047A2DF0B3FBB4EE488A002285
:10E120000123F1EE10FACDE900238DED050ACDEDC6
:10E13000060A9FED0A0A0A488DED071AF0EE680AF2
:10E1400068BF134605A90CF027F9284609B0BDECB5
:10E15000028B30BDE02E65420000C8420000000086
:10E16000847B002007B50191FFF79AFF30B1019938
:10E17000044803B05DF804EB00F0F2BA03B05DF8B8
:10E1800004FB00BFB82B0020014865F0B7BF00BFFB
:10E19000004C002008B500F5005090F8883EC3F30D
:10E1A00040128A420BD061F3451380F8883E31B1AA
:10E1B00052F03AFABDE808400F2152F071B908BD9B
:10E1C00070B500F500560546D6F8C83E8B420C46A1
:10E1D00012D0012911D0022916D059B952F024FACF
:10E1E0001B2152F05DF90D4A05F5315006212C3006
:10E1F00054F038FAC6F8C84E70BD52F015FA1A211C
:10E2000052F04EF9064AEFE7012100F04BFE52F0C2
:10E210000BFA1D2152F044F9024AE5E7C4070C0845
:10E22000D9070C08D4070C0810B500F500520C46AD
:10E2300092F8AD3E03F00101A14209D064F300035E
:10E2400082F8AD3EDB0704D405F088FE024B9C72D9
:10E2500010BD06F05BF8F9E79D80002000F5005046
:10E2600090F8AD3E61F3410380F8AD3E014B197368
:10E27000704700BF9D80002010B504465CF036FB5F
:10E2800020215DF0EBFA04F50053003893F88A2E54
:10E2900018BF012060F3820283F88A2E10BD0000AF
:10E2A00010B504464FF0E6FB04F50052436FD2F878
:10E2B000B82E04F58044D360D4F838299366D4F896
:10E2C0004029C2F8FC32D4F8380903685B6D9847DE
:10E2D000D4F838090368BDE810409B6D184700006A
:10E2E00070B52DED028B00F500550446D5F8B83E0B
:10E2F00093F8CB30002B72D095F9883E002B6EDB63
:10E3000000F5804696F8803A002B68D1D5F8940E37
:10E3100003685B699847002861D1324BD3F8940EAB
:10E3200003681B6898470B2859D0D6F840399FEDF1
:10E330002E7AD3EDDB7AF0EEE77AF4EEC77AF1EEDF
:10E3400010FA4CD5D5F8B80E443053F0A1FD034671
:10E35000DFED260A93ED000A9F20B7EE001A2AF09F
:10E3600081F8B5EEC00AF1EE10FA38DD04F59240FE
:10E370001C3080F04FFBDFED1E7AB0EEC00AB4EE29
:10E38000E70AF1EE10FA2AD504F58054D6F83809D8
:10E39000D4F8603407EE903A0368D3F89830B8EEBA
:10E3A000E78A984738EE400ADFED127AB0EEC00AED
:10E3B000B4EEE70AF1EE10FA11D5D4F8643440F265
:10E3C000E63203F2F313934209D8BDEC028BD5F881
:10E3D000B80E9FED090ABDE8704082F0A5BDBDEC06
:10E3E000028B70BDB84B002000000034000000001C
:10E3F000000070420000FA430AD7233C08B500F53C
:10E400000050D0F8B80E03681B699847F6EE007A02
:10E4100020EE270AB5EEC00AF1EE10FA48BF9FEDD4
:10E42000010A08BD0000000038B52DED028B00F593
:10E4300080450446D5F83839DFED110A93ED370AE7
:10E4400004F500547120B7EE001A2AF00BF8D4F846
:10E45000B80ED5F8405903681B69B0EE408A98475A
:10E4600038EE400ABDEC028BDFED067A05F5057546
:10E47000284620EE270ABDE8384070F069B800BF92
:10E480000000000000007A4400F5805000F597631A
:10E4900000F2C440D3ED005AD2ED007AD0ED006A0C
:10E4A00091ED006A26EEE77A67EEA57AA6EE257A68
:10E4B000E6EE267A81ED007AC2ED007A7047000020
:10E4C00000F50050B0F91C3A33B9B0F97E010028CC
:10E4D000B8BF404280B2704783EAE370A0EBE370BC
:10E4E000F8E7000070B52DED028B00F5005482B006
:10E4F00094F8AD1E11F00106054605D09FED2D0ADA
:10E5000002B0BDEC028B70BD8DED010A5CF0EEF93E
:10E51000037F002BF2D0DFED288ADFED260A9DED88
:10E52000010AB0EE681A4E2029F09CFF4FF4C87221
:10E530003146B4F98601B0EE408A29F0D1FFA4F843
:10E540008601284610F08AF9B4F9863107EE900A60
:10E55000B8EEE77A07EE903AF8EEE77A77EE676A78
:10E56000B4EEE68AF1EE10FA0DD52846FFF7A8FFC3
:10E5700007EE900A38EE668AB8EEE70A20EE088ABF
:10E5800088EE260ABCE777EE877AB4EEE78AF1EEEA
:10E5900010FAB3DDB4F97E3100EE103A38EE678A36
:10E5A000B8EEC00A78EEE77A20EE088A88EE270AED
:10E5B000A6E700BF0000000000007A44002070477A
:10E5C000002070477047000000F506501430704777
:10E5D0000048704770370C0800F50050D0F8940ED2
:10E5E00003681B6818470000034808602F2111705A
:10E5F00008221A60704700BF740B0C0800F5005029
:10E60000D0F8940E0368DB6C1847000000F500504A
:10E61000D0F8940E03689B6C1847000000F5005377
:10E6200000F59640D3F8943E20301B1A58425841CA
:10E630007047000010B500F500500C46D0F8940E5D
:10E640000368DB6D984707EE900A9FED057AF8EEB8
:10E65000677A012067EE877AC4ED007A10BD00BFAB
:10E660000AD7233C10B500F500500C46D0F8940EA4
:10E6700003689B6D984707EE900A9FED057AF8EEC8
:10E68000E77A012067EE877AC4ED007A10BD00BFFB
:10E690000AD7233C10B500F500500C46D0F8940E74
:10E6A00003681B6E9847DFED047A20EE270A0120ED
:10E6B00084ED000A10BD00BF0AD7233C5EF058BDB0
:10E6C00062F0FCBC5EF0FAB84FF01EB927F008BE4D
:10E6D00051F062BA17F014B95BF05ABD59F00ABF95
:10E6E0000FF06ABD10F0AAB906F0ECBC11F0AAB99F
:10E6F00005F08ABC05F0DCB905F002B960F0B8BAE3
:10E700000EF000BCFFF7ECBD0FF08EBE10F0F4B8B9
:10E7100003F074B80FF016BE0FF094BD5CF034B87F
:10E7200022F078BC06F09EB802F03EBC10F002B9B0
:10E7300006F07EBC04F0D6B806F0D8BD05F072B97C
:10E7400006F03EB90FF0C4BCFFF7AABD28F0E6B84A
:10E7500005F05ABE09F080BE09F07ABD09F00EBD81
:10E760001FB500F500530446D3F8940E03910368D7
:10E770005B6A984760B1DFED070A0399002304F54F
:10E780009F400093B0EE600A1A464C300BF05AFCE2
:10E7900004B010BD0000000010B52DED028B00F597
:10E7A00000530446D3F8940E03685B6AB0EE408AC7
:10E7B000984720B90024BDEC028B204610BD9FED88
:10E7C000080A04F59F4028EE000A4C300AF004FFC6
:10E7D00004460028EED003480121FFF7DBFCEAE7FE
:10E7E0000000C842B82B00200A4A92F9882E002A5D
:10E7F0000B4605DA00228A604A600A6001207047F1
:10E8000000F58040D0F83829783207CA83E807003D
:10E81000F4E700BFB84B002070B51F4B036000F554
:10E8200000530446D3F81C0E1C4AC3F86C2C08B1E4
:10E8300019F0BCF91A4B236004F5805393F82C2E81
:10E8400042B9D3F8285E2DB1284626F089FB284628
:10E8500019F0A8F904F58B50103077F0A7F804F5FB
:10E86000835018305EF05EFA04F6C44504F6644640
:10E87000B54204D0183D284625F0C8FFF8E7094BFB
:10E88000C4F8983804F6941052F0DEFF04F51060D6
:10E8900052F0DAFF204670BD300F0C0860140D08EE
:10E8A00018F50C088CBC0C0838B5484B044640F8E9
:10E8B000043B5EF07DFD04F1100016F0C3FC04F192
:10E8C00068004EF0AFFD04F5907021F02DF804F5CE
:10E8D000866015F049FA04F2545019F069F904F60B
:10E8E000980027F0A1FB04F544605EF03FFB04F5BF
:10E8F000516049F017FC04F57C6050F02FFF04F5DF
:10E90000835018305EF0F6F904F58550143017F096
:10E9100095FF04F58B50103077F034F804F58C50E7
:10E920000C304FF041F904F58F505FF0EBFE04F529
:10E9300080530025264A83F8045204F5905004F5CC
:10E94000905304331430136045F096F804F5935057
:10E950002946083011F0A6FC04F5C55018306FF0B8
:10E96000B5FE04F5E5501C3074F052F804F5EE5095
:10E97000143076F061F904F5F150183076F096FD18
:10E9800004F5F450103011F08FFA04F5FF501030F8
:10E9900070F052FB04F50150083065F0C7F804F53B
:10E9A000005304F5045083F804510A4D1C3077F0ED
:10E9B000BDFB2B6813B1084888F096F9204607493B
:10E9C00048F098F92C60204638BD00BF18F50C08B7
:10E9D000148A002078810020E8070C0840F40C0815
:10E9E00010B50FF0B5FE5BF081FF0368BDE8104085
:10E9F0005B681847FFF7F4BF10B5044606F07EF8D1
:10EA0000204610F0A3F9204603F0B6FD2046BDE8ED
:10EA1000104003F01DBF0000FFF7EEBF70B500F51A
:10EA20003B5524350446284616F0E6FA19F086FED2
:10EA300090F9213093B390F840337BB304F5005341
:10EA400004F25456D3F8B80E443053F021FA03467A
:10EA5000DFED130A93ED000A9F20B7EE001A29F0AC
:10EA600001FD94F98835012B284608BF86ED0E0A72
:10EA7000002116F087F8DFED0B7A04F2AC7494ED08
:10EA8000287A20EE270ADFED087AA7EE270A30461B
:10EA900084ED280ABDE8704019F060BD70BD00BF6C
:10EAA00000000000CDCCCC3D6666663FFFF7B6BFE8
:10EAB00010B50121044610F085F960B1114BD3F86F
:10EAC000940E03689B6A984728B9204602F07AF9A9
:10EAD000204602F087F94FF40011204610F072F939
:10EAE00018B128F095FF27F0B3F94FF480212046A4
:10EAF00010F068F928B128F08BFFBDE8104027F02E
:10EB0000B5B810BDB84B0020FFF7D2BF70B500F507
:10EB100080450446D5F838099FED540A86B06C301C
:10EB20002CF0AEFE04F5935003A908308DED030AD6
:10EB3000CDED040A8DED051A11F060FA0221204690
:10EB400010F040F970B10121204610F03BF948B9AE
:10EB5000474BD3F8940E03689B6A984710B9204638
:10EB600002F030F90121204610F02CF948B9404B51
:10EB7000D3F8940E03689B6A984710B9204602F0B8
:10EB800031F90121204610F01DF910B9204602F09C
:10EB900081F94FF40031204610F014F930B104F53A
:10EBA0000053D3F8B80E03685B6C984740212046A9
:10EBB00010F008F960B104F57C60019050F08CF918
:10EBC00004F58053019893F978300BB150F0C6FAF0
:10EBD0004FF48061204610F0F5F818B104F57C6020
:10EBE00050F014FA2021204610F0ECF858B104F54A
:10EBF0000056D6F8940E03681B699847C0B1D5F843
:10EC000040097CF0F3FE8021204610F0DBF8E0B1F3
:10EC100028F0FEFE27F04EF81021204610F0D2F822
:10EC200010B3D5F8380906B0BDE8704079F024BCBF
:10EC300020460CF0BFF80028E1D1D6F8940E036806
:10EC40005B6998470028DAD0DDE74FF48021204641
:10EC500010F0B8F80028DBD14FF40021204610F066
:10EC6000B1F80028D4D1D7E706B070BDE02E6542D8
:10EC7000B84B0020FFF74ABF10B50121044610F041
:10EC8000A1F810B1204602F005F98021204610F0CD
:10EC900099F858B14FF48021204610F093F828B924
:10ECA00028F0B6FEBDE8104026F0E0BF10BD000021
:10ECB000FFF7E2BF10B5044605F074FC204605F0EE
:10ECC000D7FA204605F0B2FC204610F027FF204678
:10ECD000BDE8104003F02CBCFFF7ECBF70B54FF659
:10ECE000FF71044610F06EF804F5005528B1D5F810
:10ECF000882E0721204602F0FDF8D5F8B83E93F89B
:10ED0000CB307BB92046FFF7B7FAD5F8B80E95F8A7
:10ED10009A21036895F810121B6A9847D5F8B80E27
:10ED200082F0CEF85DF0F4FA5DF080F8204610F045
:10ED3000F3FE95F8883E0F4A04F58044DB43D4F88F
:10ED40003859C3F3C01353712B681E6F4EF092FEF7
:10ED50004EF0FAFA2846B047D4F840494EF08AFE01
:10ED600004F505744EF0F0FA2046BDE870406FF0EF
:10ED700055BA00BF9D800020FFF7B0BF2DE9F041DC
:10ED800000F5805600F5005406F5976304F6CC684C
:10ED90001B68C8F8003006F2C44304F56D671B68B1
:10EDA0003B600546D6F8680400F58C40503029F0E9
:10EDB0002DFB04F6D863C4F8D40ED8F800201A60EE
:10EDC00004F6DC643B6823604FF6FF7128460FF0C1
:10EDD000F9FF38B1D6F8682428460921BDE8F0418A
:10EDE00002F060B8BDE8F08110B500F50053D3F82B
:10EDF000C84E002C55D093F8892ED10751D56FF30A
:10EE0000000283F8892ED3F8CC2AD3F8C81AB2F9B5
:10EE10000820012C06EE902AB1F908400BBF03F63A
:10EE2000CC6203F6D862D2ED007AD2ED007A0CBF44
:10EE300003F56D6203F6DC62D2ED005A0CBFF8EE0A
:10EE4000E66AF8EEE66A07EE104A25EEE66AB8EEE4
:10EE5000C77A00F58050A7EE276A00F5976200F2A6
:10EE6000C44067EEA67AD2ED006AE7EE257A90ED0F
:10EE7000007A27EE877AA6EE267ABDEEC77A17EEDD
:10EE8000104A0C8192ED007AD3F8CC3A67EE877A7B
:10EE900090ED007AE6EE477AFDEEE77A17EE902ADB
:10EEA0001A8110BD38B505462DED028B00F50054D2
:10EEB00071B128460FF0DAFAD4F8D43E1B1A03F2E7
:10EEC000F31340F2E63293420CD8BDEC028B38BD0E
:10EED000D4F8C83E022BF8D10FF0AAFAB0F57A7F29
:10EEE000E7D2F2E7C4F8D40E00F58C40503064232A
:10EEF00090FBF3F308EE103ADFED0B7AB8EEC88A18
:10EF000028EE278AB0EE480AAAF072FB04F6D8630E
:10EF100083ED000AB0EE480AAAF0C0FC04F6DC64F7
:10EF200084ED000AD1E700BF35FA8E3C00F593501E
:10EF30000121083012F02CBEFFF7F8BF10B50446CF
:10EF40000FF092FC102120460FF03CFF70B12046DC
:10EF500001F092FE4FF4001120460FF033FF28B964
:10EF600028F056FDBDE8104026F072BF10BD00002D
:10EF7000FFF7E4BFF8B50446254606F0DFF8224B5C
:10EF800045F83C3B214BA465C4E91734204BC4E948
:10EF90001934204BE36604F1800018F09BFA04F169
:10EFA0009C0018F097FA04F1B80018F093FA4FF6A5
:10EFB000FF76194BC4F8CC30A4F8D06004F1D4002B
:10EFC00018F088FA4FF0FF37144B1549C4F8307128
:10EFD00028461D6047F08EFEA4F87870A4F894606F
:10EFE00004F5A27018F076FA04F5B07018F072FA11
:10EFF00004F5BE7018F06EFA002384F89031C4F85E
:10F00000B4312046F8BD00BFD4620C0855E70008B3
:10F0100059E700085DE700080000FFFF6C80002052
:10F020004CCA0C0810B5044606F088F80A4B236059
:10F030000123A38704F1400018F04CFA04F15000BA
:10F0400018F048FA04F1600018F044FA04F1700076
:10F0500018F040FA204610BD7C6A0C082DE9F043F8
:10F06000044689B0FFF720FCA24B236004F506504C
:10F070003C3004F5005502F071F804F506530833EE
:10F0800004F52B57C5F8DC3A062385F8E03A4FF033
:10F090007C5805A907F12C00CDF8148052F05AFFD6
:10F0A00007F1440087F016F804F5924600231C3659
:10F0B00004F52C5785F81C3B192304A985F8283B37
:10F0C000C5F8246B07F13400CDF8108052F042FFF0
:10F0D00007F14C0086F0FEFF4FF00108182304F5FD
:10F0E0002E5004F52F5785F8703B2C3785F8648B2C
:10F0F000C5F86C6B04305DF00FFA384677F0D2F843
:10F1000006AE7D4BC5F8EC3B3146381D8DF81880B6
:10F1100048F00EFC04F53050243077F0ADF8774B12
:10F12000774FC5F8243C04F5305031463C30069703
:10F1300052F010FF04F5315031460830069752F076
:10F1400009FF04F531503146143004F53158069763
:10F1500008F12C0852F0FEFE6A4BC5F86C3C08F131
:10F16000080086F0B7FF04F5325704F53359183715
:10F1700009F13C093846143757F0B4FB4F45F9D133
:10F180000723C5F8203E0023A5F8243E4FF4CB709A
:10F1900018F006FDC5F81C0E04F53850283086F02E
:10F1A00099FF04F539502C3086F094FF564B1A68BD
:10F1B0000AB9C3F8008004F5A347544BC5F86C3C6A
:10F1C000343704F53A50C5F8947E183078F0E4FAF4
:10F1D00005F6CC634FF07E58C3F8008005F6D8657D
:10F1E0004B4B07934B4BC5F800800694009304F5F6
:10F1F0003B5096E80C004FF40071243015F07AFB78
:10F2000004F55050103068F01DFC04F5914003A93E
:10F210006C30CDF80C8052F0C3FE03A904F5924087
:10F22000CDF80C8052F096FE04F5924004F580452E
:10F230000C3018F04FF905F61C1300261E605E60B6
:10F240009E6005F6281304F592401E605E609E6085
:10F2500004F593530833C5F83439002385F855393C
:10F260004FF40041583016F0D1F804F5934058306F
:10F2700066F076FD04F59440143048F08FFC264B80
:10F28000C5F8143A04F59440244B2549283004F578
:10F290009448186008F1480847F02CFDFF2385F8D2
:10F2A000583A85F8603A1F49404647F023FD1E4A08
:10F2B000136813B11D4887F017FD1D491D48C2F89A
:10F2C000008004F59442703208604FF0140E1FFA6B
:10F2D00083FC0EFB0C010133097C0029F7D1164B8E
:10F2E000A3F800C0154BD3F80080B8F1000F29D067
:10F2F0001348E0E7300F0C0870070C08B0070C0843
:10F300000000A04060140D0894840020B00F0C0889
:10F3100051E70008200F0C08C0070C08188A0020CD
:10F32000E8200D08E4A50D08A88A0020FC070C08B9
:10F330003881002064510C0836810020F4800020C0
:10F340001D080C0804F595401A6003A9554B03935A
:10F35000043052F0FFFD04F59540243005F0EEFE38
:10F36000514BC5F8A43A04F59540643005F0E6FE2B
:10F3700004F599494D4BC5F8E43A04F5964009F176
:10F3800078092030FFF7F6FD484605F0D7FE484BD8
:10F39000C5F8F83C09F13C0084F080FB454BC5F80A
:10F3A000343D04F59D40383005F0C8FE424BC5F8A9
:10F3B000B83E04F59D407C3005F0C0FE3F4BC5F8DB
:10F3C000FC3E04F59E4085F8388F3C3005F0B6FED3
:10F3D0003B4BC5F83C3F04F59E40783005F0AEFE4F
:10F3E000384BC5F8783F05F6B47304F59F401E60AE
:10F3F0005E609E604C3005F0A1FE334BC5F8CC3FFB
:10F4000004F5A0452846C5F80880103005F096FEA2
:10F410002E4B2B612846583005F090FE2C4BAB65E7
:10F4200004F5A140143005F089FE2A4BC5F894304C
:10F4300004F5A240C5F80C61C5F810612830FFF74B
:10F44000F1FD384605F07AFE234BC5F8B43104F5DA
:10F45000A340703005F072FE204BC5F8F03104F582
:10F46000A440A5F82C824030FFF7DCFD1C4BC5F80A
:10F47000403204F5A540012385F8C932C5F8D062B1
:10F48000C5F8D462C5F8D8625C3005F057FE154B5C
:10F49000C5F8DC322046C5F81C63C5F8206309B006
:10F4A000BDE8F083CDCC4C3DD05F0C0874600C08F7
:10F4B00078630C0808640C08C4640C0864650C08C4
:10F4C00004660C089C660C083C670C08CC670C08AA
:10F4D00064680C0804690C08D86B0C08746D0C087F
:10F4E000346B0C08386E0C0838B5054B1C68236863
:10F4F0000A461D68034B01462046A847002038BD38
:10F50000E07E0020B82B002010B587F049F8064CAB
:10F51000064B18602046FFF7A1FD2046044A054926
:10F52000BDE81040A9F03EBFB82B0020E07E0020CF
:10F530000CE3002019E800080120704790F8903093
:10F540008B4286BF00EB8100D0F89400002070470A
:10F5500090F890308B4286BF00EB8100D0F8940089
:10F5600000207047FA207047014B93F84A0170471A
:10F57000B84B0020034BD3F8C80E431E58425841E5
:10F58000704700BFB84B0020034BD3F8C80E831E52
:10F5900058425841704700BFB84B0020034BD3F886
:10F5A000B80E08B180F0CEBA01487047B84B0020C1
:10F5B0009C0F0C0870B5036A2E4D43F4E0520262B2
:10F5C000426A42F4E0524262826A42F4E05282624B
:10F5D000D5F840290446E2B143F4F8430362D5F874
:10F5E00040097BF0C3FD38B1636A43F48043636232
:10F5F000A36A43F48043A362D5F840097BF0D8FEA8
:10F6000038B1636A43F400536362A36A43F400535E
:10F61000A362194B1D6845B11921284648F05CFECC
:10F6200018B1236A43F480732362144E96F8E43AC7
:10F630006BB1636A43F48073636245B11921284654
:10F6400048F082FE18B1A36A43F48073A362236A70
:10F6500043F080432362636A43F080436362D6F8D9
:10F66000B83E93F8C1301BB9A36A43F08043A3624C
:10F6700070BD00BFB86B002044810020B84B002053
:10F6800013B54FF44470CDE9002118F083FA044615
:10F6900028B1DDE9002159F07BFE024B23602046B2
:10F6A00002B010BDF0110C08002070477047000038
:10F6B0000320704708207047014B93F84C017047B6
:10F6C000B84B0020034B93F90402003818BF012007
:10F6D000704700BFB84B0020014B93F94E017047B3
:10F6E000B84B0020704700007047000008B50C4B75
:10F6F000D3F8400970B910230A4AD2F8B82E43F063
:10F70000400022B192F8CB200AB143F0C00040F093
:10F71000010008BD7BF02AFD0028ECD01823EBE7A0
:10F72000B86B0020B84B002038B5C5780B46352D96
:10F73000044628BF3525352200211846ACF074FB5D
:10F740002A4604F10C01BDE83840ACF023BB0000B0
:10F750001FB5184C94F8DE1F04F5696010F090FB9B
:10F7600078B194F8DE1F04F5696010F08BFB40B1AE
:10F7700094F8DE1F04F5696004B0BDE8104010F095
:10F7800083BB002301930293039312F08FFA01A924
:10F7900012F066F820B101A82CF070FC04B010BD86
:10F7A00021F076FC90F8C432B02202FB030090ED09
:10F7B0002F0AF3E7B83B002008B50D4BD3F8B80E7D
:10F7C000A8B1443052F064FB034693ED000ADFED2C
:10F7D000090A9F20B7EE001A28F044FEDFED067AF2
:10F7E00020EE270ABDEEC00A10EE103A18B208BD8E
:10F7F000B84B0020000000000000C8422DE9F04F87
:10F80000DFF8D880344F8DB00446042508F5005643
:10F8100017F8019BB8F9A43109F1FF3A43FA0AF34A
:10F82000D90742D5207C53F0ABFE8346207C54F0B0
:10F83000ABFD00F121039B4505D2207C0DB0BDE856
:10F84000F04F53F019B9BAF1030F2ED8DFE80AF0E0
:10F850000234393ED6F8380903689B68984700F1AE
:10F8600094035A69D3F800A0D3F804E0D868196962
:10F87000D3F818C008925A6A1B6ACDF82520CDF833
:10F88000293062222123CDE9003206900791207CA5
:10F89000CDF80CA0192303AAC221CDF810E0CDF8B1
:10F8A00014C08DF8249053F0D5FE013D15F0FF05EE
:10F8B000AED10DB0BDE8F08FD6F838090368DB682B
:10F8C000CCE7D6F8380903681B69C7E7D6F8403992
:10F8D00003F52A73C5E700BFBC120C08B84B002023
:10F8E00013B504460748019108F0FAFB30B90199B5
:10F8F000204602B0BDE8104054F06ABF042002B0B8
:10F9000010BD00BFD8760020014808F043BA00BF00
:10F91000D876002058F09CBC10B588B0044656F04C
:10F92000E3F80C4BD3F8B80E38B90B4A0621204641
:10F9300008B0BDE8104056F0BFB869461E2280F0FE
:10F9400005F9064A6B460621204656F0B5F808B080
:10F9500010BD00BFB84B0020E80F0C08465D0C0836
:10F96000034A92F8C43A013382F8C43A55F0C0B958
:10F97000B84B002007B50846019117F081FE38B159
:10F980000448019902F086FC002003B05DF804FBF6
:10F990000420FAE7EC7E0020162A10B40C4605D0AD
:10F9A000542A03D05DF8044B54F030BF0323237076
:10F9B00001205DF8044B704708B555F0CDF840F4D0
:10F9C0001C6040F00D0008BD10B5044618F0EAF8C0
:10F9D000204610BD10B50C4C94F9883E002B0FDB6F
:10F9E000D4F8940E0368DB6C984758B9D4F8940E99
:10F9F00003689B6C984700280CBF0220032010BDB1
:10FA00000120FCE70420FAE7B84B002010B44C6951
:10FA1000012C05D101465DF8044B034802F0BEBF3E
:10FA20005DF8044B55F07EB9B82B00202DE9F34169
:10FA3000B1F90430002B06460C46154635DB4FF075
:10FA40000008CDE900281A4FB1F902209FED190AEC
:10FA5000D7F8C81A4FF47A7358F0D4FE0123CDE9D1
:10FA600000539FED140AB4F90020D7F8CC1A4FF4D4
:10FA70007A73304658F0C6FE9FED0F0AB4F90420A1
:10FA8000D7F8D01A43463046CDE9005858F0BAFEB0
:10FA9000CDE900589FED070AB4F90620D7F8D41A2B
:10FAA0004FF47A73304658F0ADFE02B0BDE8F081F5
:10FAB000B84B00200000FA4400007A44044B187848
:10FAC00020B9044B93F88A0EC0F38010704700BF32
:10FAD0003C800020B84B00200C4B93F80D248AB9D1
:10FAE000A3F5805393F8AD2E92060BD193F9882E8F
:10FAF000002A09DB93F8893E13F0200F14BF04207D
:10FB0000012070470520704703207047B85B002034
:10FB100008B5074B93F99831032B03D0BDE8084093
:10FB200056F042B8034A022155F0C6FF042008BD32
:10FB3000B84B002000100C08094BD3F8082292079C
:10FB400001D454F055BE03F5005303F5116393ED52
:10FB5000000ADFED047AB8EEC00A20EE270A7047EB
:10FB6000B84B00200AD7233C10B594B0044603A834
:10FB700017F0B0FC1C4BD3F8940E036803A95B6D1F
:10FB8000984778B3002103A817F03CFD50B3247CBC
:10FB900087F0DCF8059BDDED047A0893069B09935A
:10FBA0000023F8EEE77A9FED117A0B930C930D93F7
:10FBB0000E930F931093119312934FF6F853ADF8E1
:10FBC0004C300023962267EE877A8DF84E3033232F
:10FBD000CDE90032079007AA57212046CDED0A7AD9
:10FBE00053F038FD14B010BDB84B00200AD7233CA9
:10FBF00030B52DED0A8B764C0546D4F8940E03688B
:10FC000099B05B6A984700285AD004F54054A3681D
:10FC1000062B00F2C980DFE803F00404045788AB28
:10FC200053006C489FED6C8A0AF0D4FB9FED6B0A81
:10FC30000168426883680D930BA80B910C922BF01E
:10FC40001FFEF0EE489AB0EE40CAF0EE60BAB0EE99
:10FC5000419AB0EE48AAF0EE488AF0EE48AAB0EE1B
:10FC600048BA40F6F8542D7C87F070F800231593BD
:10FC7000169301238C228DF85E303323CDE90032B8
:10FC80000B90B1EE499AF1EE688AB1EE488A0BAA60
:10FC9000552128468DED0CCACDED0DBA8DED0E9A8D
:10FCA0008DED0FBACDED10AACDED118A8DED12AA12
:10FCB000CDED139A8DED148AADF85C4053F0CAFC7B
:10FCC00019B0BDEC0A8B30BD42480AF083FB9FEDB2
:10FCD000430A0168426883680D930BA80B910C924C
:10FCE0002BF0CEFD3B48F0EE60BAB0EE419AB0EE9C
:10FCF00040CA0AF073FB9FED390A2BF0C1FD35486D
:10FD0000B0EE40BAF0EE60AAF0EE418A0AF06AFB6B
:10FD10009FED320A2BF0B4FD4FF44064B0EE40AAE0
:10FD2000F0EE609AB0EE418A9DE72A489FED2A9A4C
:10FD30000AF054FB9FED290A2BF0A2FD2548B0EEF6
:10FD400040BAF0EE60AAF0EE418A0AF04BFB9FED5C
:10FD5000230A2BF095FDF0EE49BAB0EE40AAF0EE82
:10FD6000609AB0EE418AB0EE49CA40F607447AE79D
:10FD70001848DFED198A0AF035FB9FED180A2BF0C1
:10FD80007FFDF0EE68AAB0EE40AAF0EE609AB0EE09
:10FD9000418AB0EE68BAB0EE689AF0EE68BAB0EE9A
:10FDA00068CA40F63F445EE79FED0B8A0024F0EE00
:10FDB000489AB0EE48AAF0EE488AF0EE48AAB0EEB3
:10FDC00048BAB0EE489AF0EE48BAB0EE48CA4AE7F0
:10FDD000B84B0020847B0020000000000AD7233CA1
:10FDE0002DE9F0412DED068B3B4D95F8893E9906A6
:10FDF0008CB004466AD505F500579FED380AD7F850
:10FE00003809DFED378A6C302BF03AFD8DED041A9E
:10FE100021EE281AD5F8946E8DED020ABDEEC11AB6
:10FE2000CDED030A11EE103A1DB2336894F810803C
:10FE30009B6D304660EE289A20EEA89A984707EE10
:10FE4000900AF8EEE77A304667EEA87AFDEEE77A98
:10FE500017EE903A1CB23368DB6D984707EE900AB4
:10FE6000B8EE678AD7F84039DFED1E7A93ED0FAA16
:10FE7000336828EE288A1B6EB4EEE78AF1EE10FA9A
:10FE800058BFB0EE678A30469847BCEEC88A002358
:10FE9000089318EE103AB7222AEE28AA20EE280A74
:10FEA000ADF82C301A23CDE900323E2105AA404698
:10FEB000CDED059A8DED069A8DED07AA8DED090A17
:10FEC000ADF82850ADF82A4053F0C4FB0CB0BDEC9F
:10FED000068BBDE8F08100BFB84B00209F0CB345F6
:10FEE0000AD7233C00FF7F472DE9F04F2DED028B11
:10FEF0001A4B047CD3F838398DB0D3F88480D3F80A
:10FF00008870D3F88C60D3F8905093ED258AD3F89D
:10FF100098B0D3F89CA0D3F8DC9086F017FF0023AC
:10FF20008DF82C3016222523CDE90032029002AA4A
:10FF3000532120468DED078ACDF820B0CDF824A0BE
:10FF4000CDF82890CDF80C8004970596069553F0CF
:10FF500081FB0DB0BDEC028BBDE8F08FB86B0020CB
:10FF6000054BD3F8B83E2BB193F8CA00002808BF60
:10FF70000220704702207047B84B002008B5034BA1
:10FF8000D3F8940E03681B68984708BDB84B00204F
:10FF9000024B93F8890EC0F340107047B84B002015
:10FFA00070B52C4E2DED028B0546D6F8940E91EDD2
:10FFB000018A036886B05B6A0C46984750B9BDEE6B
:10FFC000C88A18EE103ADB0704D4022006B0BDEC54
:10FFD000028B70BDD4E9040129F0FCFA0028F4D0AA
:10FFE00002A817F077FA02AA2146284658F07AFBB1
:10FFF0000028EAD0184902A817F04EFB0346002853
:020000040801F1
:10000000E3D1DFED160A00900246B0EE600A144814
:1000100002A90AF017F8D8B1D6F8940E03685B6A03
:100020009847044608B10020D0E70E480222042178
:1000300005F01AFC60B1DFED090A09480094234677
:10004000B0EE600A224602A909F0FCFF0028EAD1BE
:100050000420BBE7B84B0020C4740020000000005F
:10006000847B0020B82B002008B591F82030032BAA
:100070001CD1D1ED027A9FED0E7A91ED060A0D4B5F
:10008000F0EEE77AF4EEC77ADFED0B7AD3F8940E50
:10009000F1EE10FA4CBF0121002120EE270A0FF0EB
:1000A00095F9002814BF0020042008BD0220FCE7B9
:1000B00000000034B84B00200000C84210B52DED00
:1000C000028BD1ED007AF5EEC07AF1EE10FA82B033
:1000D0000C4604DA042002B0BDEC028B10BD9FED8B
:1000E000197AF4EEC77AF1EE10FAF3D891ED030A1B
:1000F0009FED158AF0EEC07AF4EEC87AF1EE10FAB0
:1001000019D5D4ED037A1148D4ED010A94ED000A13
:10011000F4EEC87AD4ED027AFDEEE77AF1EE10FA49
:10012000CDED017A9DF90410ACBF0122002202F04E
:1001300013F80020CFE7F7EE000A28F08FF8002828
:10014000C8D0DEE70000B44300000034EC7E00209D
:1001500091ED010AB5EEC00AF1EE10FA08B501DC26
:10016000042008BD9FED107A104BD1ED007AD3F832
:10017000940E20EE070A9FED0E7A0368F4EEC77A1C
:10018000F1EE10FA05DDDB6E98470028E8D000207C
:10019000E7E79FED087AF4EEC77AF1EE10FACCBFEC
:1001A0009B6E5B6EF0E700BF0000C842B84B0020BA
:1001B0009A9939403333F33F08B5D1ED007A9FED7A
:1001C000157AF0EEE77AF4EEC77AF1EE10FA1DD563
:1001D000D1ED017AF0EEE77AF4EEC77AF1EE10FA9B
:1001E00014D50D480222032105F03EFB80B10A48D8
:1001F0000121FDF7CFFF094890F8603B012B03D0A8
:1002000000F65C302EF074FE002000E0022008BDF5
:100210000420FCE700000034B82B0020B86B00205D
:1002200010B5D1ED007AFCEEE77A17EE903A9CB269
:10023000012C02D0022C06D04CB9064821465EF0B3
:10024000D9FD002010BD044803F04EF9F9E7042061
:10025000F8E700BFE0750020B82B00201FB5D1EDF6
:10026000017A0B7CFCEEE77ACDED027AD1ED007AD3
:100270000093FCEEE77AD1ED030ACDED037A91ED20
:10028000020A9DF808309DF80C20014602480DF046
:1002900087FE05B05DF804FBB82B002010B50A4CB2
:1002A00094F8AD3EDB070CD402220521A4F50050E2
:1002B00005F0DAFA28B902221146A4F5005005F03B
:1002C000D3FA002010BD00BFB84B002010B5D1ED0F
:1002D000007AFCEEE77A044617EE903A13F0FF033B
:1002E0000FD10F4BD3F8940E03689B6F984708B15A
:1002F000002010BD0B4A2046062155F0DDFB0420EE
:10030000F7E7012B09D1064BD3F8940E0368DB6F96
:1003100098470028ECD1044AEDE70220E9E700BF46
:10032000B84B002024100C0834100C089FED0B7AF9
:1003300001F10C03F1EC017AF4EE677AF1EE10FAB8
:100340000AD6F0EEE77AF4EEC77AF1EE10FA03DCA3
:100350009942EFD1012070470020704700007A4495
:1003600030B52DED028B8DB0002305460393049329
:10037000059311F09BFC03A911F072FA58B311F028
:1003800095FC00F55A7393E8070006AC84E8070073
:10039000DDED060A9DED070A2D7CF1EE600AB1EE57
:1003A000400AA9F047FB2046B0EE408A2BF066FEDB
:1003B000DFED0B7A089B0B93012228EE278A0C2392
:1003C000CDE90032A82109AA28468DED098A8DEDD4
:1003D0000A0A53F03FF90DB0BDEC028B30BD00BFEF
:1003E000E02E6542242938B505460FD003D81B29D5
:1003F00007D1012412E04029FBD0A1F14203012BD7
:10040000F7D92846BDE8384058F02EBD0C2152F0EF
:1004100045FB044610B12846FFF7A2FF204638BD31
:1004200038B5194C94F8AD3EDB070D460AD4D4F824
:10043000B83E93F8CB303BB90122114604F6EC30BC
:10044000FDF700FD002038BD94F9883E002B4FF0E9
:10045000020212DA0521A4F5005005F005FA002881
:10046000F0D095ED000ADFED097AD4F8940E20EE75
:10047000270A01210EF0AAFFE4E70921A4F50050A4
:1004800005F0F2F9DEE700BFB84B00200000C842DB
:1004900010B5214C94F8AD3EDB070ED4D4F8B83E2D
:1004A00093F8CB304BB194F9883E002B07DA012248
:1004B000082104F6EC30FDF777FD002010BDD1EDEA
:1004C000007A9FED167AF0EEE77AF4EEC77AF1EE55
:1004D00010FA0BD512480222112105F0C5F9A0B976
:1004E000022211460E4805F0BFF9E6E7D4F8940E53
:1004F00003681B6898470428DFD0D4F8940E03687B
:100500001B6898471428E5D1D7E7064840F6C41180
:1005100008F0C0FAD1E700BFB84B0020000000345B
:10052000B82B0020707A002070B58B8BC12B05464C
:100530000C463CD8BB2B0CD8542B6AD02ED8113B80
:1005400099B2052918D921462846BDE8704059F0CE
:1005500023BBBC3B052BF6D801A151F823F000BF0B
:100560004D0601085B06010847050108470501081B
:10057000F705010801060108052BE4D801A151F88F
:1005800023F000BF370601084705010847050108A9
:1005900047060108A905010813060108732B22D09C
:1005A000B22B24D0552BCED10222092145E04AF2AC
:1005B0001146B34237D00AD8D12B26D0B3F5967F57
:1005C00035D0D02BBFD1BDE87040FFF729BE4AF22D
:1005D0001246B34223D04AF21346B342B3D1BDE828
:1005E0007040FFF755BFBDE87040FFF767BDBDE83D
:1005F0007040FFF7ADBD2146BDE87040FFF7D0BCAD
:100600002146BDE87040FFF761BEBDE87040FFF7CE
:1006100025BE21462846BDE87040FFF725BDBDE850
:100620007040FFF7FDBEBDE87040FFF737BEBDE884
:100630007040FFF7C1BD022205210A4805F014F9F8
:1006400048B9042070BD02220621F6E702210648BF
:1006500006F06EFAF4E70020F4E70221024806F003
:1006600031FAEDE7B82B0020D876002008B591EDDF
:10067000007AF6EE007AB4EEE77AF1EE10FA06DDD3
:10068000044801220521FDF78FFC002008BD04204D
:10069000FCE700BFA457002030B52DED028BCD78CC
:1006A00093B0272D28BF27250C462722002108A814
:1006B000ABF0BAFB2A4604F10C0108A8ABF06AFBC8
:1006C000424BD3F8940E03685B6A9847002841D0E8
:1006D0009DF8465068063DD400244FF07E5329060D
:1006E000049307940694059427D504A82AF0A0FB48
:1006F000EA0701940294039405F006032ED4002B1C
:100700002ED10D9B01930E9B02930F9B03933048B8
:1007100009F046FA9DED100A044630B340F2ED4070
:10072000B7EE001AFFEE000A27F09CFE2848234689
:1007300001AA04A909F03CFA0CE0099B04930A9B66
:1007400005930B9B069304A80C9B07932AF076FB5A
:100750000028CDD113B0BDEC028B30BD062BD6D016
:1007600001211B4809F0B8F9F4E7DFED1A0A4FF44C
:100770009E60B7EE001A27F075FEF6EE000AB0EEA6
:10078000408A27F06BFDE8B9B6EE000A124BB4EED2
:10079000C08AF1EE10FAD3F8443908DD38EE400A89
:1007A00030EE008A93ED070A28EE000ABEE730EE2D
:1007B000480AD3ED087A30EE000AF0EEE77A27EE29
:1007C000C00AB3E79FED030AB0E700BFB84B0020B3
:1007D000847B002000000000B86B00202DE9F0436E
:1007E0009DB0814608460EA9FEF79EFF844BD3F8C4
:1007F000940E03685B6A984750B19DF86C30012BEA
:1008000009D0DA1F022A06D97E48012109F064F9CD
:100810001DB0BDE8F083BDF86840A20504F00706EE
:1008200004F0380704F4E07501D5002DF0D04FF046
:100830000008CDF81480CDF81880CDF81C803EBBA0
:100840009FED716A9DED107ADDED117ADDED0F6A95
:1008500027EE067A67EEC67A66EE866A083B012BBB
:10086000CDED056A8DED067ACDED077A04D867489F
:1008700006AA05A9FDF708FE9DF86C30073B022B80
:1008800006D863487EF0B6F8014605A82BF018F8A4
:10089000CDF82080CDF82480CDF82880F7B9DDEDA3
:1008A000147A129B0893F1EE677A139B099308A9B7
:1008B0004846CDED0A7AFFF739FD0028A4D09FED18
:1008C000520A08A82BF030F89DF86C30083B012B39
:1008D00004D84E4809AA08A9FDF7D6FDCDF82C800A
:1008E000CDF83080CDF83480EDB99FED476A9DEDAD
:1008F000167ADDED177ADDED156A9DF86C3027EE7E
:10090000067A67EEC67A66EE866A083B012BCDED65
:100910000B6A8DED0C7ACDED0D7A04D83B480CAA0C
:100920000BA9FDF7B1FD14F4806233D1DFED397A04
:100930009DED180A9DF86C1020EE270ADFED327A43
:100940000839012920EE270A8CBF0021012114F467
:10095000006305BFDFED2F7ADDED190ADFED2E0A0A
:1009600060EEA70A04BFDFED287A60EEA70AAEB9F1
:10097000002F35D1B3FA83F3B2FA82F25B09520940
:100980000291019300920BAB08AA05A91D4809F03A
:1009900011FA3DE79FED200A0021D8E77FB9B3FAAD
:1009A00083F35B0901200093B2FA82F3CDE90110D1
:1009B0005B0914480BAA08A909F094FC28E7002D4C
:1009C0007FF422AF0120B3FA83F3B2FA82F2CDE9C9
:1009D00000105B090B4852090BA909F02BFC17E723
:1009E000002D3FF411AFB3FA83F3B2FA82F2CDE9EE
:1009F00000165B09520905A9024809F05DFA07E7EC
:100A0000B84B0020847B00200000C842B82B002097
:100A1000D4740020E02E6542000000002DE9F0476C
:100A2000A2B08046084614A9FEF77EFE7E4BD3F89E
:100A3000940E03685B6A9847C0B1BDF88040A30577
:100A400004F0070904F4E07700D57FB10CAE30461E
:100A500016F040FDB9F1000F29D1DDE9150128F0AC
:100A6000B9FD30B97148012109F036F822B0BDE86E
:100A7000F0879DF8841009AA404657F01DFE002813
:100A8000F0D0DDED177A9FED6A7A099B009367EE4F
:100A9000877A10ADFDEEE77ADDE9151217EE903A90
:100AA000284616F037FD95E80F0086E80F00002570
:100AB00014F0380A06950795089514D1DDED1A7AD9
:100AC000189B0693F1EE677A199B079306A9404697
:100AD000CDED087AFFF72AFC0028C3D09FED540A19
:100AE00006A82AF021FF09950A950B959FB99FED5D
:100AF000506A9DED1C7ADDED1D7ADDED1B6A27EE57
:100B0000067A67EEC67A66EE866A8DED0A7ACDEDD4
:100B1000096ACDED0B7A14F4806805BFDFED457AE4
:100B20009DED1E0A9FED440A20EE270A04BFDFED6B
:100B3000407A20EE270A14F4006405BFDFED3D7A09
:100B4000DDED1F0ADFED3C0A60EEA70A04BFDFED12
:100B5000387A60EEA70AB9F1000F31D1BAF1000F6F
:100B600052D13046CDED050A8DED040A16F0E2FCB7
:100B700003289DED040ADDED050A3FF473AF10A9CB
:100B80003046CDED050A8DED040A109511951295AC
:100B900016F030FE00283FF465AFB4FA84F464091F
:100BA000B8FA88F3DDED050A9DED040ACDF804A03E
:100BB00000945B0906AA10A91C4809F06BF955E7D7
:100BC000BAF1000F0FD10123B4FA84F4CDE901A3E7
:100BD0006409B8FA88F3154800945B0909AA06A9C4
:100BE00009F080FB42E7002F7FF43CAF0123CDE901
:100BF0000073B8FA88F2B4FA84F30C485B0952091E
:100C000009A909F017FB31E7002F3FF42BAFB4FA25
:100C100084F3B8FA88F2CDF800905B0952093146A6
:100C2000024809F00FFA21E7B84B0020847B00202E
:100C30000000C842E02E65420000000010B44B7A6C
:100C40008C7ACA7A43EA042343EA0243542B07D03E
:100C5000562B09D0522B0BD15DF8044BFFF71CBD6E
:100C60005DF8044BFFF7BABD5DF8044BFFF7D6BE45
:100C70005DF8044B57F028BE2DE9F0432DED028BB3
:100C800000F500560446D6F8940EDFED4B8A036853
:100C900091B05B69984704F580490027002840F02F
:100CA0008780D9F84039D3EDDE7A93EDD88AFDEE0E
:100CB000E77A28EE288A17EE903A1DB204F52D58EF
:100CC00008F1340801A940460DF032FF18B94FF081
:100CD000ABFC3A4B01933722002102A8ABF0A4F8F9
:100CE000A3238DF8083095238DF8093086F036F867
:100CF000D9F83839CDF80B00D6F8B80ED3F8DC2087
:100D0000D3F8E030CDF80F104430CDF81320CDF8F3
:100D1000173051F0BDF80346DFED290A93ED000AC4
:100D2000B7EE001A9F2027F09DFB10EE103AD6F880
:100D3000B80ECDF81B3003681B69984710EE103AC7
:100D400004F59246CDF81F301C3618EE103A3046A6
:100D5000CDF823307DF052FE20EE280A404610EEFA
:100D6000103ACDF82730D9F8E838CDF82B30019B70
:100D7000CDF82F300DF0FEFE10EE103A3046CDF8D3
:100D80003330CDF83770ADF83B507DF043FEBDEE0B
:100D9000C00A372210EE103A02A904F57C60ADF8C3
:100DA0003D304EF093FD11B0BDEC028BBDE8F083F9
:100DB00008EE107A002581E70AD7233C2292CA7FE9
:100DC0000000000010B500F58044D4F8380976F032
:100DD000FDFCD4F84019D4F83809BDE8104076F08D
:100DE0005BBD000070B54FF4805104460DF0EAFF82
:100DF00000284ED004F5804604F57C65D6F8380905
:100E000003689B689847692100F1940228464EF0D8
:100E1000F5FBD6F838090368DB6898476A2100F1CA
:100E2000940228464EF0EAFBD6F8380903681B699D
:100E300098476B2100F1940228464EF0DFFBD6F86C
:100E400040296C21284602F52A724EF0D7FB20215A
:100E500020460DF0B7FFE0B104F50053D3F8940E2F
:100E600003681B69984778B1D6F840292846903224
:100E70006E214EF0C3FBD6F840292846BC32BDE8AF
:100E800070406F214EF0BABB204609F093FF002856
:100E9000EAD170BD08B510F009FFBDE8084010F0B8
:100EA00091BC00007FB50E464FF6FF710446154613
:100EB0000DF088FFE0B1102200216846AAF0B4FFCF
:100EC000A3238DF8003095238DF8013003238DF88E
:100ED000023085F043FF1022CDF80300CDF8071053
:100EE00004F57C6069468DF80B6003954EF06EFD4D
:100EF00004B070BD7FB50E464FF6FF71044615462F
:100F00000DF060FFE0B1102200216846AAF08CFFCE
:100F1000A3238DF8003095238DF8013004238DF83C
:100F2000023085F01BFF1022CDF80300CDF807102A
:100F300004F57C6069468DF80B6003954EF046FD24
:100F400004B070BD30B52DED048B87B004460D465E
:100F5000182200216846B0EE409AF0EE608AB0EEAA
:100F6000418AAAF061FFA3238DF8003095238DF804
:100F7000013006238DF8023085F0F0FE1822CDF8FE
:100F80000300CDF8071004F57C6069468DF80B501E
:100F90008DED039ACDED048A8DED058A4EF096FC19
:100FA00007B0BDEC048B30BD10B54FF48011044682
:100FB0000DF008FF30B104F593500830BDE8104043
:100FC0000FF0F6B810BD00002DE9F0438FB01446C5
:100FD000054689463122002101A8DDE916769846AA
:100FE000AAF022FFA3238DF8043095238DF8053055
:100FF00008238DF8063085F0B1FE236804936368FA
:101000000593A36806933B68CDF81D307B68CDF847
:101010002130BB68CDF825303368CDF829307368AE
:10102000CDF80700CDF80B10CDF82D303122B36884
:101030008DF80F9001A905F57C608DF81C80CDF826
:1010400031304EF043FC0FB0BDE8F08370B52DEDAC
:10105000068B8CB0144605460E462C22002101A8B2
:10106000B0EE409AF0EE608AB0EE418AB0EE61AA2E
:10107000F0EE429AAAF0D8FEA3238DF8043095230F
:101080008DF805300B238DF8063085F067FEDFED17
:101090001A7A94ED007ACDF8070027EE277A29EE28
:1010A000279A8DED077A94ED017ACDF80B1027EE93
:1010B000277A68EEA78A8DED087A94ED027A8DF88A
:1010C0000F6028EE278A67EE277A2C2201A905F502
:1010D0007C608DED049ACDED058A8DED068ACDED0F
:1010E000097A8DED0AAACDED0B9A4EF0EFFB0CB00C
:1010F000BDEC068B70BD00BFE02E6542A02070479E
:1011000070B5144B88B004466946D3F8B80E04F5A0
:101110007C6504F500561E227EF018FD6A460E49D5
:1011200028464EF06FFDD6F8940E03681B6898476A
:1011300096F80421014628464EF088FD04F59350A8
:10114000083010F0F1FF04F590701FF00BF808B0B4
:1011500070BD00BFB84B0020465D0C082A4B2B4ADF
:1011600070B54360002343618361C361C363284B4F
:10117000426303644FF08042264B4364044682631B
:10118000583059F033FA244E244BA365A825601932
:1011900059F0E2FB66513035B5F56A7FF7D104F5B9
:1011A0006A705AF095FF002104F5F66081F0BEF8F0
:1011B0001B4BC4F864389FED1B1ADFED1B0A9FED33
:1011C0001B0A04F6780077F0F3F89FED161A9FEDEE
:1011D000180AF0EE410A04F5096077F0E9F89FED8E
:1011E000111A9FED130AF0EE410A04F6A80077F0F9
:1011F000DFF820460F4945F07DFD20460E4945F0B9
:1012000079FD204670BD00BFF83700200000C841BE
:101210000AD7233C0000E040B05A0C08C45A0C081E
:10122000EC780020000000009A99993E0000B44339
:1012300000804A43744E0C08D4500C0870B54C4DD5
:101240004C49ADF50E7DD02206465AA8AAF0A2FD63
:101250000FCD0EAC0FC40FCD0FC40FCD0FC495E84A
:101260000F0084E80F0000245AAB18190021B7EED4
:10127000000A103445F00CF8D02CF5D13E4B0FCBC2
:1012800002AC84E80F0001A9204644F0B5FF90B1FC
:101290009DF90430DFED396AE06807EE103AB8EEE8
:1012A000C77AF0EE007AE7EE267AB7EE000A80EE13
:1012B000270A46F0C7F800240EAB18190021103495
:1012C000B7EE000A44F0E4FF402CF5D12C499022FF
:1012D00036A8AAF05FFD0022092136A845F084F85F
:1012E00096F97469D6B9274D0FCD1EAC0FC40FCD3A
:1012F0000FC40FCD0FC495E80F0084E80F003246ED
:1013000004211EA845F070F89FED1F0A1F4846F003
:1013100099F81F48B7EE000A46F094F81D4C9FED6F
:101320001E0A0FCC06AD0FC594E80F0085E80F002C
:10133000002106A844F0ACFF9FED170A00212846C3
:1013400044F0A6FF04F1100160221EA8AAF022FDBD
:1013500000241EAB18190021B7EE000A103444F027
:1013600097FF602CF5D15AF0C7FC0DF50E7D70BDCE
:101370000C010C083C000C084C010C08CDCCCC3DF9
:101380005C010C08EC010C08000000005C4D0C082E
:101390006B4D0C082C020C08000034422DE9F0477C
:1013A00090B00DF106011D205AF098FD002800F0C4
:1013B0009E809DF80630614A0133DBB211210BA8F3
:1013C0008DF8063084F0ACFE00220DF107010BA869
:1013D00044F098FC9DF80630594A112105460BA8A7
:1013E00084F09EFE00220DF107010BA844F08AFC58
:1013F0009DF80630534A112106460BA884F090FE52
:1014000000220DF107010BA844F07CFC9DF806308A
:101410004D4A03F03F03112107460BA884F080FEDC
:1014200000220DF107010BA844F06CFC8046002D52
:101430005DD0002E5BD0002F59D0002857D0284611
:1014400044F078FE002852D1304644F073FE002864
:101450004DD1384644F06EFE002848D1404644F055
:1014600069FE002843D1394C94E80F000DF10C0CB3
:1014700010348CE80F0094E80F000DF11C0989E886
:101480000F0002A9604644F0B7FE98B3BDF80840CB
:1014900002A9484644F0B0FE00284AD0BDF8083002
:1014A00054BB23B340F2E2449C420FFA84FA0FFA91
:1014B00083F927D80DF10A013046ADF80A9046F0BD
:1014C000B7FA0DF10A012846ADF80AA046F0B0FAC5
:1014D0000DF10A013846ADF80AA046F0A9FA00233A
:1014E0000DF10A014046ADF80A3046F0BBFA10B0E3
:1014F000BDE8F0870024CBE740F2D662002B08BF9E
:101500001346D1E70DF10A013046ADF80AA046F0C6
:101510008FFA0DF10A012846ADF80A9046F088FAD4
:101520000DF10A013846ADF80A9046F081FA012320
:10153000D6E7002CDBD040F2D663B5E77C4D0C0833
:10154000884D0C08944D0C08A14D0C08AC020C08F9
:1015500037B500F505517822083104464CF0AEFD50
:1015600000220C21244844F03FFF2046FFF716FFDD
:1015700004F505500022B7EE000A02211C3044F0A9
:10158000BBFF012504F501511C4A009500230831D9
:10159000452044F02DFF1A4A1368D90705D419498C
:1015A000156004F5FF5310330B6004F50650154920
:1015B00001223C30012544F06DFF134A00950023C1
:1015C00004F57C61FD2044F013FF104B1A68D2072C
:1015D00005D40F4A1D6004F58C540C3414600C487B
:1015E000012144F073FF45F08BFD0A4A138843F054
:1015F0000103138003B030BDB44D0C083CA00D08AE
:10160000E47E002000220020B4FB0C08E87E0020CD
:101610000C220020288100200F299DBF302303FBCE
:101620000100503000207047014B93F98F01704743
:10163000B84B0020024B93F8AD0E00F0010070474C
:10164000B84B0020044BB3F85431DB075ABF006994
:10165000C0F3401000207047B84B0020014BD3F876
:10166000D40A7047B84B002008B503689B689847B8
:1016700030B9044B93F9AC0EB0FA80F0400908BDC4
:101680000020FCE7B84B002038B50D1E2DDB174CB1
:1016900094F8E02AEBB29A4227D3D4F8DC3A01223C
:1016A000595DA4F5005004F0DFF8F0B159F01EF9CF
:1016B00003215AF0D3F8C0B959F018F90D215AF0A6
:1016C000CDF890B994F97431EB40DB075CBF94F925
:1016D0008E11E940A4F5005048BF0221BDE8384012
:1016E00058BF01F00101FCF76BBD38BDB84B0020BD
:1016F000022A10B50C4605D1BDE810400948352234
:1017000004F0B2B8084BD3F8940E03681B689847EE
:10171000A04205D159F0EAF8BDE8104059F070B880
:1017200010BD00BFB82B0020B84B002029B1022902
:1017300007D1044BC3F88C1E7047024B0122C3F83B
:101740008C2E7047B84B002031B1022907D1044BD1
:10175000012283F8902E7047014B83F8901E70474A
:10176000B84B002010B500F50053DFED186AD3F830
:10177000CC2AD3F8C83AB2F90820B3F908309FED63
:10178000147A07EE902AF8EEE77A0446C7EEA60A26
:1017900000F593500121083007EE903AF8EEE77A11
:1017A00060EE870A87EEA60A20EE070A10F01CFBFF
:1017B0004EF03AFF26214EF073FE04F53150054AF3
:1017C000BDE8104006212C3050F04CBF0000C8424C
:1017D00035FA8E3C80580C0800F58042002382F8D0
:1017E0005439044A00F5315013720621024A2C3054
:1017F00050F038BF9D8000208C580C08F8B500F5DB
:101800008045044695F85419002955D02B4B2C4A95
:10181000D3F8940E904204D1D3F8B83E93F8CB306D
:1018200023B92046BDE8F840FFF7D6BF254E95F80E
:10183000557904F50053012093F9882E3072C7BB07
:10184000002A39DB85F855090139C9B285F85419E0
:10185000D3F8CC2AD3F8C83AB2F90820DFED1A6AD7
:10186000B3F908309FED197A07EE902AF8EEE77A7F
:10187000B1FA81F1C7EEA60A04F593504909083080
:1018800007EE903AF8EEE77A60EE870A87EEA60A4E
:1018900020EE070A10F0A8FA95F8543963B904F558
:1018A000315033720A4ABDE8F84006212C3050F01E
:1018B000D9BE002AC8DAB4E7F8BD00BFB84B002093
:1018C0006C7D00209D80002000007A4535FA8E3C1A
:1018D000A0580C086D2900F3E380012901DC59F0C0
:1018E0000BBE8B1E6B2BFAD80FF2040C5CF823F0A6
:1018F000FF1A0108F91A0108FF1A0108FF1A010866
:10190000DF180108FF1A0108DF180108DF180108B5
:10191000F91A0108DF180108FF1A0108F91A01086D
:10192000F91A0108DF180108FF1A0108FF1A010857
:10193000FF1A0108DF180108DF180108F91A010869
:10194000FF1A0108F91A0108DF180108F91A01083D
:10195000F91A0108DF180108DF180108DF1801086B
:10196000DF180108DF180108F91A0108FF1A010839
:10197000DF180108DF180108DF180108FF1A010845
:10198000DF180108F91A0108DF180108DF1801083B
:10199000FF1A0108F91A0108DF180108DF18010809
:1019A000DF180108FF1A0108FF1A0108FF1A0108D1
:1019B000DF180108DF180108FF1A0108DF18010805
:1019C000DF180108FF1A0108FF1A0108FF1A0108B1
:1019D000DF180108DF180108FF1A0108FF1A0108C3
:1019E000DF180108DF180108DF180108DF180108F7
:1019F000DF180108DF180108FF1A0108FF1A0108A3
:101A0000FF1A0108FF1A0108FF1A0108FF1A01084E
:101A1000DF180108F91A0108F91A0108DF1801088E
:101A2000DF180108DF180108DF180108DF180108B6
:101A3000DF180108FF1A0108F91A0108DF18010868
:101A4000DF180108DF180108DF180108DF18010896
:101A5000DF180108DF180108DF180108DF18010886
:101A6000DF180108DF180108DF180108DF18010876
:101A7000DF180108FF1A0108DF180108DF18010844
:101A8000DF180108DF180108DF180108DF18010856
:101A9000DF180108DF180108DF180108F91A01082A
:101AA000A12921DC96297FF71AAFA1F197030A2B10
:101AB0003FF615AF0FF2040C5CF823F0FF1A010893
:101AC000FF1A0108DF180108FF1A0108DF180108D2
:101AD000DF180108DF180108DF180108F91A0108EA
:101AE000F91A0108FF1A0108B42908D0DB2903D02C
:101AF000B2297FF4F4AE7047002359F0CFBC704791
:101B000070B563298AB000F3D180012904DC0AB0E2
:101B1000BDE8704059F092BA8B1E612BF7D801A432
:101B200054F823F0231D0108371D0108571D010833
:101B30005F1D01080F1B01088F1D01080F1B010805
:101B40000F1B01083D1E01080F1B01080F1B010898
:101B5000451D0108631E01080F1B0108391E0108FD
:101B60009D1E0108AB1E01080F1B01080F1B010879
:101B7000BB1E0108C91E0108D71E01080F1B010862
:101B8000F91E01080B1F01080F1B01080F1B01089C
:101B90000F1B01080F1B01080F1B01081D1F010867
:101BA000371F01080F1B01080F1B01080F1B01083D
:101BB0003B1F01080F1B01080F1B01080F1B010829
:101BC0000F1B01083F1F01080F1B01080F1B010815
:101BD0000F1B01080F1B01080F1B01080F1B010839
:101BE0000F1B01080F1B01080F1B01084F1F0108E5
:101BF0000F1B01080F1B0108AF1E0108B31E0108CF
:101C0000B71E01080F1B01080F1B01080F1B01085D
:101C10000F1B01080F1B01080F1B01080F1B0108F8
:101C20000F1B01080F1B01080F1B0108431F0108B0
:101C3000471F01084B1F01080F1B0108531F010814
:101C4000571F01080F1B0108991F01085B1F01089E
:101C50000F1B01080F1B01080F1B01080F1B0108B8
:101C60000F1B01080F1B01080F1B0108FB1F0108B8
:101C70000F1B01080F1B01080F1B01080F1B010898
:101C80000F1B01080F1B01080F1B01080F1B010888
:101C90000F1B01080F1B01080F1B01080F1B010878
:101CA0000F1B01080F1B0108112001089F291DDCD3
:101CB00096297FF72CAFA1F19703082B3FF627AFAA
:101CC00001A454F823F000BF1520010819200108D1
:101CD0000F1B01082D2001080F1B01080F1B010815
:101CE0000F1B01080F1B010809200108B42900F08F
:101CF000D780DB2917D0B2297FF409AF002A00F082
:101D00007581022A0FD1AD4BD3F8940E03689B6FF7
:101D1000984740B957F01EFBA94A042150F0A2FC95
:101D200001E0022A01D001242EE035220E21A5482F
:101D300003F09AFDF7E7111E18BF0121A148FCF737
:101D40003FFAF0E7012A04D0022A14BF0021022141
:101D5000F4E71146F2E70621FFF7CAFCE3E7022A9F
:101D6000E1D1964DD5F8940E0368DB6A9847044696
:101D70000028D8D0D5F8D03AB3F90830002BD2D10A
:101D8000A5F50050FFF7EEFC20460AB070BD022A10
:101D9000C9D18A4D8C4BD5F8942E9A42C3D0D5F830
:101DA000B83E93F8CB30002BBDD005F50054B4F904
:101DB000903B2BB9D5F8D03AB3F90830002BB2D00C
:101DC0001C22002103A805AEAAF02EF8304615F01B
:101DD00081FBB4F9903B93B91623ADF80E30D4F8DB
:101DE00010397A48642BB8BF642303A906932AF0FC
:101DF000F1FC20B14EF018FC27214EF051FB04F607
:101E00000C1494E80F0086E80F00D5F8D03A6F481C
:101E1000B3F90830002BCCBF1023152303A9ADF86C
:101E20000E302AF0D7FC00283FF47DAF4EF0FCFBCB
:101E300027214EF035FB76E703218DE7022A04D0F7
:101E40005E4B002283F8E42A6DE76148192146F0D1
:101E500043FA04460028F3D0584B012283F8E42AC1
:101E600092E7012A0BD0022A11D0002A7FF45BAF3F
:101E7000524B83F8B8214EF0D7FB2B21D9E74F4BBB
:101E8000019283F8B8214EF0CFFB2C21D1E74B4BC8
:101E900083F8B8214EF0C8FB2D21CAE70F215BE77C
:101EA0004C48114683F03AFB3DE7092154E70421F1
:101EB00052E7052150E717214EE7901E414241416C
:101EC00045485CF097FF2EE7022A7FF42CAF3D488F
:101ED00001F00AFB27E7012A06D0022A07D0002AD0
:101EE0007FF421AF1146EBE711460192E8E73A484B
:101EF00001215CF07FFFEAE7384B911ED3F83839B7
:101F00004A424A4183F820200DE7931E5942594125
:101F1000324BD3F8380977F057FB04E7274B013AE7
:101F200093F88A1E012A8CBF0022012262F3041159
:101F300083F88A1EF7E611210EE712210CE715211E
:101F40000AE7002108E7102106E7022104E7012142
:101F500002E7072100E70B21FEE6022A1F4B0ED104
:101F6000012483F8804A4EF05FFB4A214EF098FA34
:101F700057F0F0F91A4A062150F074FB04E70022EA
:101F800083F8802A4EF050FB4B214EF089FA57F02F
:101F9000E1F9144A0621C1E6012A09D0022A0AD031
:101FA000002A7FF4C0AE01210F480CF0F9FDBAE61B
:101FB00001920021F8E71146F6E700BFB84B002078
:101FC000DB580C08B82B0020D876002014770020AE
:101FD000C8380020EC780020E0750020B86B0020A5
:101FE000B8580C08C9580C082C570020184BD3F8C7
:101FF000940E0368DB6F984795E61146FFF796FB52
:10200000144803F0D7FF8EE61146FFF79DFB8AE6E2
:102010001B21A1E61C219FE6022A7FF484AE0E4814
:10202000FCF7ACFE57F096F90C4AB3E7114658F0AE
:1020300025FF0B4874F07AF9044600283FF473AE8C
:10204000034A92F88B3E43F0020382F88B3E9BE6F4
:10205000B84B00205C760020B82B0020F4580C0808
:10206000A457002010B5044604487CF0C5FC04F1D8
:102070000801BDE8104027F02BBA00BFD47400203F
:1020800038B504462DED028B11487CF0BBFC0546AB
:1020900029F05AF90F48B0EE408A0CF02DFE90B1AD
:1020A000DFED0D7AB4EEE78AF1EE10FA0BDDD5ED37
:1020B000000A95ED010AA7F0BDFCDFED087A20EEDD
:1020C000270A84ED080ABDEC028B94ED080A38BD9E
:1020D000D4740020B82B002000401C46E02E65423E
:1020E000074B93F97501022805D0032806D0003864
:1020F00018BF0120704781F001007047042070472D
:10210000B84B002003688B4216D00429C0E90013A5
:1021100002D007290ED07047084B9FED097A03F5CE
:102120008D63D3ED007AF8EEE77A67EE877AC0ED3B
:10213000087A704700238362704700BFB83B0020D5
:102140000AD7233C08B50246FFF7CAFFBDE808409E
:1021500001461046FFF7D6BF70B52DED048B04463F
:10216000F0EE408AB0EE608A0D46164684F0EEFD31
:102170009FED329ADFED329AE06176B3236843B97E
:10218000304B03F58D63D3ED007AF8EEE77AC4EDBA
:10219000097A68EE898A002DB7EE000AFFEE007A10
:1021A000B8BFB0EE670A68EE808AC4ED058A264B98
:1021B000B4EEE98AF1EE10FAD3F8380930DA76F0A5
:1021C000E1F920EE090A84ED060ABDEC048B2046F5
:1021D0000321BDE87040FFF795BF94ED090A98EE22
:1021E000890A26F0E9F8002D84ED050A0BDAB4EE31
:1021F000E90AF1EE10FADADBDFED147A30EE670A65
:1022000084ED050AD3E7D2D0DFED117AB4EEE70A08
:10221000F1EE10FACBD8DFED0D7A30EE270AEFE7BA
:1022200076F0B0F9B4EE480AF1EE10FA48BFB0EE1D
:10223000408A28EE098A84ED068AC6E70000C84273
:1022400000000034B83B0020B86B002000A00C4711
:10225000000000B410B52DED028B0446B0EE608A8C
:10226000F0EE408A84F072FDDFED090AE06168EE6D
:10227000A08A68EE200AC4ED098ABDEC028BC4ED89
:102280000A0A20460621BDE81040FFF73BBF00BF09
:102290000000C84208B54A680346084642B98A6841
:1022A00032B9C96821B9BDE808400748FFF74ABFFD
:1022B00003F1080115F09EFA28B1BDE80840024874
:1022C0000221FFF71FBF08BDEC7E002008B50721E3
:1022D000FFF718FF80ED0A0A08BD000008B5036883
:1022E000032B23D1D0ED057A9FED127AF0EEE77A39
:1022F000F4EEC77AF1EE10FA1AD50F4B90ED090AF9
:1023000003F58D63D3ED007AF8EEE77A37EEC00A75
:1023100026F052F8DFED097AB0EEC00AB4EEE70A13
:10232000F1EE10FA94BF0120002008BD0120FCE767
:102330000020FAE700000034B83B002000004843CA
:1023400030B50368023B85B00446082B6FD8DFE840
:1023500003F0050D30374D6341636300FFF782FEE4
:1023600084ED090A94ED090A05B030BD84F0EEFC55
:10237000E369DFED320AE061C31A07EE903AF8EE46
:10238000677A94ED050A67EEA07AD4ED060AF1208B
:1023900020EEA71A67EEE00A26F064F8D4ED057A7D
:1023A00077EEC07AC4ED057AD4ED097A37EE800A6B
:1023B000D6E7FFF765FEDFED227A20EE270ACFE7AA
:1023C000204B03F56E63D3ED007AF8EEE77AC0EDAB
:1023D000097AC7E71C4DD5F84C097AF0A7FC00280C
:1023E000C0D0D5F84C391B6B6362BBE784F0AEFC00
:1023F000E3699FED127AD4ED0A6AE061C31A07EE31
:10240000903AF8EE677A67EE877A94ED097AA6EE4D
:10241000A77A84ED097AA5E70B4B9FED0C0AD3F858
:1024200038096C3029F02CFA84ED091A9AE7064B2A
:10243000D3F84039D3F84433D6E700BF6F12833A5C
:102440000000C842B84B0020B86B00209F0CB34579
:102450000368092B08D8DFE803F0050A0505050520
:10246000070705100023836290ED0A0A7047044BAA
:10247000D3F84039D3F84833F5E7C36AF3E700BF30
:10248000B86B0020F8B50023214FCB6297F8AD3E22
:10249000204E13F0010F04460D462DD1D7F8940EAF
:1024A00003685B6F984738B3D7F8940E03F08EFB40
:1024B000DFED197A85ED0B0AB0EEC00AB4EEE70A3B
:1024C000F1EE10FA03D409213046FFF71BFE114844
:1024D000FFF736FF0F4884ED000AFFF7B9FF3368B6
:1024E00084ED010A0A2B0FD8DFE803F00C1010105E
:1024F0001010100C100C0C003368092BE7D10548A4
:102500000021E2E70223A3602046F8BD0123FAE799
:10251000B84B0020EC7E002000000034034B012269
:102520001A6000229A60DA601A617047EC7E00201F
:1025300013B501A904460CF07BFA04F5804320B9D9
:10254000012283F8FD2902B010BDDDED017ADFED37
:10255000096A03F51F62B8EEE77AD2ED007A67EEFA
:10256000A67AB4EEE77AF1EE10FA54BF0122002207
:10257000E7E700BF0000C8422DE9F04F2DED068BC4
:1025800000F5005700F5935997F9C6318BB0064610
:1025900000F5804409F1080933B1D7F8B83E93F843
:1025A000CB80B8F1000F0FD10021A4F8741A48466F
:1025B0000FF0E2FD94F8751A48460BB0BDEC068B9F
:1025C000BDE8F04F0FF0E2BD84F0C0FB8346D4F8C5
:1025D00040099FED978A90EDDBAA78F0C7FD07AD23
:1025E000002800F0CD80D4F8403903F55C7393E8FF
:1025F000070085E8070028468DED098A29F03EFD91
:10260000B0EE409A30460CF077FB06F5924A0AF19C
:102610001C0A002800F0B78050467CF0F3F907C888
:1026200085E8070028468DED098A29F027FDF0EEA0
:10263000409AD7F8940E03681B689847122840F018
:10264000AB80002384F8743AD7F8940E03685B6972
:10265000984728B1D7F8D03AB3F90830002B0CDCF2
:1026600097F9883E002B08DAC4F878BA50467CF017
:10267000C5F904F67C2383ED000A94F8743A5BB143
:10268000D4F8780A41F28833ABEB000B9B4540F25B
:102690009180002384F8743AD4F838099FED650AD4
:1026A0006C3029F0EDF88DED070ACDED080A8DEDBF
:1026B000091A95E8070004AB01AD9FED5F0A83E8B6
:1026C000070085E80700284629F0DAF83046B0EE22
:1026D000408AF0EE608A8DED040ACDED050A8DED9D
:1026E000061A0CF009FB002876D0DFED547AF4EEE0
:1026F000E79AF1EE10FA94BF01250025D4F84009BD
:1027000078F034FD30B1DFED4D7AB4EEE79AF1EEBA
:1027100010FA0AD9002D66D1D7F8940E03681B6809
:102720009847022866D04FF00008D4F8400978F0A6
:102730003FFE0546002876D0B5EEC0AAF1EE10FAAD
:1027400070D5DFED3F7AB4EEE7AAF1EE10FAACBF38
:102750000126002650467CF05DF966B9DFED397A36
:10276000B0EEC00AB4EEE70AF1EE10FA5DD8002D23
:1027700008BF4FF0000894F8741A84F8758A16E7B9
:10278000B0EE489A3EE730460CF088FA00287FF415
:1027900043AFDFED279A4CE7D7F8B83E93F8CB303C
:1027A000002B3FF451AF97F9883E002BBFF64CAF9A
:1027B000012347E750467CF021F904F67C23D3ED52
:1027C000007A30EE670ADFED207AB4EEE70AF1EE28
:1027D00010FA3FF75EAF5FE730460CF05FFA054650
:1027E000002882D18AE7D4F8400978F0BFFC00289D
:1027F00092D19AE7B0EE680AA6F0FAFEF0EE408AAF
:10280000B0EE480AA6F0F4FEDFED107A20EE280ABA
:10281000B4EEE70AF1EE10FACCBF4FF001084FF02A
:10282000000882E700252E4694E7B046A3E700BFE4
:10283000000000009F0CB345D30237390000FA4274
:102840000000C8C2000070420000484255CF7D3FE2
:1028500038B504460CF050FA04F59355083548B9DC
:1028600020460CF01BFA014620B92846BDE8384046
:102870000EF004BF04F50054D4F8940E03689B6C6A
:10288000984720B9D4F8940E0368DB6C984701464A
:10289000EBE7000030B5044689B0684604F593556F
:1028A00014F018FE083504A814F014FE69462846F2
:1028B0000EF09EFF98B104A928460EF0E9FF70B112
:1028C000059B019323680022DB6C694620469847EC
:1028D00028B104F5255001212C307FF0F3FF09B019
:1028E00030BD000000F5805292F8E424D2070BD4EA
:1028F00000F50052D2F8B82E92F8CB1009B1FFF7CC
:10290000C9BF03689B6C18477047000030B587B09B
:10291000044602A8019114F0DDFD04F5935002A9CC
:1029200008300EF065FF019A18B90025284607B057
:1029300030BD236802A9DB6C204698470546002875
:10294000F3D004F5255001212C307FF0BBFFEDE7DB
:10295000F0B5044685B004F59356684608360F4630
:10296000154614F0B7FD694630460EF091FF10B9D8
:10297000002005B0F0BD394630460EF0F1FD0028CC
:10298000F6D0002DF5D004F58054284694F8E434B0
:1029900043F0020384F8E434EBE700002DE9F04F44
:1029A0002DED0A8BBDB0044624220E4618A8002146
:1029B000A9F03AFA2422002121A8A9F035FA24220C
:1029C00000212AA8A9F030FA04F50055242200219C
:1029D00033A8A9F029FA0023CDE90D330F9395F818
:1029E000893E13F0080837D143F0080395F8C42A4C
:1029F000079285F8893E15F0A1FE90F9213003B3C6
:102A000090F84033EBB104F25457384615F0A6FD68
:102A1000C24694F876355FFA8AF18B421FD9384660
:102A200015F07AFD0AF1010A81460028F1D1C84A61
:102A30000221304653F040F895F8893E69F3C3030C
:102A400008E0C44A0221304653F036F895F8893E32
:102A50006FF3C30385F8893E4FF001083AE304F5AC
:102A60002F532C33012118460BEE903AFBF790F8C8
:102A7000814608B9B84ADBE720460BF069FED5F875
:102A8000D03AB3F90890B9F1000F01D0B34AD9E7B1
:102A900095F9883E002B01DBB14AC9E7204601F0D9
:102AA00075FE04F53B53243318464A460CA90CEE38
:102AB000103A12F0B7F8002814BF02230123039341
:102AC000F123CDE913398F210A23CDE90031307C80
:102AD000ADF85490032313AA4D2150F0BBFDA14B38
:102AE0009FEDA18A01225A720621A04A304652F077
:102AF000E3FF039B022B0CBF9D4A9E4A06213046F2
:102B00004FF0000952F0D8FF85F8829149463846C7
:102B100015F06EFC94F876355FFA89F18B420CD98A
:102B200013AA38468DED138A8DED148A8DED158A22
:102B300009F1010915F0DEFAECE7384615F00EFD53
:102B40004FF0000A4FF07C0B94F876255FFA8AF973
:102B50004A4519D94946384615F0BEF9C0B20BFBB3
:102B600000403CAA0C2300F2E45003FB092C07C8E8
:102B7000ACF1900C8CE807003CAA02EB890909ED46
:102B80002F8A0AF1010ADFE741F288310AA821F011
:102B900089FFD5F8B80E9FED749A03689FED76AA69
:102BA0009B6ADFED76AA9847D5F8B80E01217CF034
:102BB000D1FE734B1B680293D86A036801211B681E
:102BC000984784F0C3F8059084F0C0F8F0EE499A75
:102BD0000690002504F50059079A99F8C43A9342E3
:102BE00040F0D68094F89618384615F095FC0028E9
:102BF00000F0CE80D9F8B83E93F8CB300493002B88
:102C000000F0C68041F288310BA821F04BFF84F020
:102C10009DF8059BC01A132840F2D78084F096F8DF
:102C2000059020460BF094FD59F072FB824659F056
:102C300009FBD9F8D03AD9F8B80EB3F9083000EE4C
:102C4000103AB8EEC00A20EE0A0A7EF05DFB50464C
:102C500059F000FB384615F081FC1CEE100A12F00A
:102C6000CBF9D9F8D03ADFED400AB3F9083000EEDD
:102C7000103AB8EEC00AA22020EE0A0AB7EE001AF7
:102C800025F0F0FBB4EEE90AF1EE10FA1CEE100AA2
:102C90004FF000020CA958BFF0EE409AF0EE408AC7
:102CA00011F0C0FF08B900230C939DED0C8ADFEDF5
:102CB000357AB4EE498AF1EE10FAF4EEE78A48BFAD
:102CC000B0EE498AF1EE10FA80F28D809FED2E9AD7
:102CD000DFED2E8A4FF0000A94F876355FFA8AFB12
:102CE0005B4540F294814FF00C0918AB09FB0BF9DE
:102CF00003EB0900B0EE490A28F0C2FD59463846F8
:102D0000CDED110A8DED121A8DED100A15F0E4F8D3
:102D10007C23C0B203FB0040B0EE680A00F2E4502E
:102D200028F0AEFD3CAB13A910A899448DED130A11
:102D3000CDED140A8DED151A28F076FD0AF1010A81
:102D400009ED240A49ED230A09ED221AC4E700BF60
:102D5000F15A0C08E05A0C08EF6E0C08FF5A0C08E8
:102D6000115B0C089D800020000000001C5B0C081B
:102D7000315B0C0897040C086F12833A0000C842BC
:102D8000E07E002000000034A4707D3F0AD7233C81
:102D9000D9F8B80E03689B6A9847D9F8B80E002195
:102DA0007CF0D8FD029BD86A036800211B68984715
:102DB000002D40F05F813046C94A052152F07CFE6B
:102DC0002946384615F014FB70E1029B986A0368A7
:102DD00005215B6898470BA821F070FEB0EE498A88
:102DE000B0EE489AF6E64FF000094FF00C0B04F5F0
:102DF000B26A94F876255FFA89F39A4222D9194685
:102E00003846089315F068F8089B0BFB03F13CABC0
:102E10005A18A2F16C034FF07C0CC0B2CDE9083215
:102E20000CFB00A018AB1944543028F013FD089B8C
:102E3000099A09F1010902ED1B0AC3ED010A83EDAC
:102E4000021AD6E7039B012B4FF0000A46D19FEDF3
:102E5000A5BA9FEDA59A4FF00C0B94F876355FFA62
:102E60008AF5AB4240F286800BFB05F53CAB03EBE9
:102E70000509A9F14803089321ABB0EE680A581977
:102E800028F00EFD089B09ED120AC3ED010A83ED3F
:102E9000021A33ABB0EE4B0A581928F0F1FC2AABFA
:102EA00058198DED100AB0EE490ACDED110A8DEDDD
:102EB000121A28F0E5FC13A910A88DED130ACDED28
:102EC000140A8DED151A28F0C5FC0AF1010A09ED66
:102ED000090A49ED080A09ED071ABEE79FED819A34
:102EE0009FED81BAF0EE088A94F876355FFA8AF998
:102EF0004B4564D99DED0C0AB4EEE80AF1EE10FAE8
:102F000035DB0C2303FB09F93CAB03EB090521ABD3
:102F100003EB090028F0C4FC33AB45ED110A05EDC5
:102F2000101A05ED120A03EB0900B0EE490A28F069
:102F3000A7FC2AAB03EB09008DED100AB0EE4B0A9B
:102F4000CDED110A8DED121A28F09AFC13A910A8E4
:102F50008DED130ACDED140A8DED151A28F07AFCCB
:102F600005ED090A45ED080A05ED071A049D0AF169
:102F7000010AB9E74FF000094FF00C0A94F87635D2
:102F80005FFA89F5AB4241D933AB0AFB053029F032
:102F900075F81BEE900AF0EE408A73F0C3F907EE65
:102FA000900AB8EE677A3CABC8EE877A03EB8505EA
:102FB00009F1010967EEAA7A45ED2F7ADEE74FF0B5
:102FC000000A4FF00C0B94F876355FFA8AF94B45FE
:102FD0001DD933AB0BFB093029F050F8C8EE297A24
:102FE0000AF1010A1BEE900A67EE808A73F09AF9E3
:102FF00007EE900AB8EE677A3CABC8EE877A03EB2F
:10300000890967EEAA7A49ED2F7ADCE7049D83F0FF
:103010009DFE069BC01AB0F5FA7F27D983F096FE75
:1030200004F50053DDED0D7AD3F8D03A0C9A1B89E4
:103030001392FCEEE77A339A1492ADF85C30349A2E
:10304000159217EE903A359A1692ADF85E30F0224E
:103050001423CDE90032B121069013AA307C50F040
:10306000F9FA6BF0ADFF317C6BF0A4FE0BA821F0F8
:1030700025FDB5E60399384615F0BAF900254FF05D
:103080000C0A94F87635E9B28B4207D933AB0AFBC8
:103090000132384615F02EF80135F2E7384615F0C2
:1030A0003BF8124A0621304652F006FD104B00252F
:1030B00020465D7201F05CFB04F50650023043F0DF
:1030C000EFFE99F8893E65F3C30389F8893E0AA8A3
:1030D00021F0F4FC40463DB0BDEC0A8BBDE8F08F1A
:1030E0004DF00D08A4707D3F0AD7233C395B0C08D6
:1030F0009D8000207FB54C4BD3F8903ADB07044607
:1031000000F18F8000F50055D5F8B83E93F8C12046
:10311000002A40F0868093F8CB30002B7ED095F9C2
:10312000883E002B7ADB00F5804696F8803A002B2B
:1031300077D1D6F838099FED3D0A6C3028F0A0FB16
:10314000CDED020A60EEA00ADFED397A8DED010ABD
:10315000E0EE000A8DED031AF4EEE70AF1EE10FA44
:103160005CDCD6F838399FED337AD3ED377AF4EE5C
:10317000C77AF1EE10FA04D5D5F8B83E1B7A002BC9
:103180004CD0B5EE007AF4EEC77AF1EE10FA45D4E1
:1031900004F592401C307BF03DFCDFED277AB4EE65
:1031A000E70AF1EE10FA39D8D6F838399FED237ACC
:1031B000D3ED367A67EE877AB3EE0E7AF4EEC77AFD
:1031C000F1EE10FA2ADA1E4AB4F9A410138801337A
:1031D0009BB2138019B9B4F8A210A4F8A410B4F8E3
:1031E000A41099421DD8002616804DF01DFA012228
:1031F00019214DF075F9D5F8B80E03685B69984749
:10320000431C04F531500F4A31462C304FF02AFA56
:10321000D5F8B83E012283F8C12002E0084B002215
:103220001A8004B070BD00BFB84B00209F0CB3459E
:103230004054094A6666663F000000B4E02E6542CD
:10324000267F0020505B0C0870B52DED028B4A4B99
:10325000D3F8903A9B0784B004461FD400F580450C
:10326000DFED468AD5F8380903681B699847D0ED29
:10327000017AF4EEE87AF1EE10FA0FDB04F5005370
:1032800004F59546D3F8B82E92F8C110043649B12A
:10329000002303A9304603934EF0FCFD04B0BDECBF
:1032A000028B70BD92F8CB20002AF1D093F9883EB2
:1032B000002BEDDB95F8803A002BE9D1D5F83809E1
:1032C00003681B699847D0F8A430D5F838090393F0
:1032D00003681B69984704F58C7200F1A40130461D
:1032E0004EF046FEDDED037AB0EEC08AF0EEE77AEE
:1032F000F4EEC87AF1EE10FA03D503A930464EF089
:10330000C9FDD5F8380903681B699847D0ED040A50
:10331000F4EEE80AF1EE10FAC0DBF6EE087A60EEA1
:10332000A77AF4EEC87AF1EE10FA1DD583F00EFDFF
:10333000D5F8903A42F21072C31A9342AED9DFED3B
:10334000107AC5F8900A68EE277A04F5315417EE22
:10335000900AF9F7D9F82C34CDE90001094A002187
:1033600020464FF07FF999E79DED030A24F076FFA0
:103370000028DBD192E700BFB84B002000000034EA
:103380000000C8426C5B0C0810B5044600F5944080
:1033900028305BF041FD04F594400121BDE8104068
:1033A000483064F00BBA0000F8B500F580450446DB
:1033B00095F9283A4BB300F5005695F83C2A96F853
:1033C000883EDB43C3F3C01363F3C30200F59447A5
:1033D00000F5924085F83C2A1C307BF01BFBDFEDAA
:1033E0003E7A283720EE670A38465BF095FD95F85F
:1033F000803A53B938465BF03BFDD6F8B83E93F8B7
:10340000CB301BB9354B00221A80F8BD95F83C3AF9
:10341000DB07FAD4D6F8940E03689B6B9847002814
:10342000F0D096F9883E002BECDB2C4E33884BB95C
:10343000B5F92E3A33B1642213FB02F3D5F8102903
:103440009A42E2DB38465BF083FDD5F838399FEDD0
:10345000247AD3ED367A67EE877AB3EE0E7AF4EEFD
:10346000C77AF1EE10FA05D83388002BCDD0013B96
:103470003380CAE7B4F9A4301BB9B4F8A230A4F879
:10348000A4303388B4F8A420B4F9A40015499342B9
:103490003CBF013333803388D5F8E828012B01D1B4
:1034A0000A60B2E709689142ACDD18B9B4F8A2200D
:1034B000A4F8A420B4F8A4209A42A6D8002333800C
:1034C0004DF0B2F802220C214DF00AF82046BDE87A
:1034D000F840FFF759BF00BF0AD7233C247F0020E4
:1034E000E02E6542207F002008B500F5804292F969
:1034F000283A6BB300F5005393F9883E002B0EDA9F
:1035000000F53150134A06212C304FF0ABF84DF046
:103510008BF80322BDE808400F214CF0E1BFB2F95F
:103520002E3A8BB1D2F81029642113FB01F39A4291
:103530000ADA00F53150084A01212C304FF092F898
:103540004DF072F80222E5E7BDE80840FFF71CBF26
:1035500008BD00BF845B0C08965B0C08F0B52DED30
:10356000028B00F500555B4ED5F8B83E93F8CB3092
:103570008DB0044633B195F9883E002B02DB95F9F6
:103580009E312BB9002333800DB0BDEC028BF0BD12
:1035900000F5804797F8803A002BF3D101F05AFBF1
:1035A00000287DD1D5F8940E03689B6B98470028BE
:1035B000E8D004F591406C304EF08EFC28F05EFDB2
:1035C000F0EE087AB4EEE70AF1EE10FAF0EE408A77
:1035D000D8DA04F5805303F5966203F2B443D3EDD1
:1035E000007A92ED000A20EE270AA6F0BBF9DFED83
:1035F0003A7A20EE270AB2EE0E7AB4EEC70AF1EE5E
:1036000010FABFD9D7F8383993ED368A28EE278AD1
:10361000F3EE0E7AB4EEE78AF1EE10FAB2D904F5C1
:103620009350002309A9083009930A930B930EF0D5
:103630003BF900283DD13388B4F9A42001339BB273
:103640003380002A40D0B4F8A420B3EB420F9BDBB8
:103650004CF0EAFF01220C214CF042FF1F4B0022EC
:1036600018EE900ACDE90623F8F74EFF1C4BCDE982
:103670000401002218EE100ACDE90223F8F744FFF6
:1036800004F531542C34CDE90001164A20460021BE
:103690004EF0E8FF01220C211348FAF785FC73E78E
:1036A000D5F8940E0368DB6C984700287FF47AAF56
:1036B00068E709A828F0E2FCF2EE047AB4EEE70A23
:1036C000F1EE10FAB7DB5DE7B4F8A220A4F8A4206D
:1036D000B9E700BF1C7F0020E02E654200000840D3
:1036E00000003E40AC5B0C08A4570020F0B52DED67
:1036F000028B8BB0002307930893099305AB044614
:10370000019300F5935007AB009302AA04AB03A901
:1037100008300DF0E1FF04F50056054686F8600C10
:1037200028B9002528460BB0BDEC028BF0BD83F014
:1037300001FBD6F8643C9FED2F7AC31A07EE903A4E
:10374000F8EE677A074667EE877A04F5305006AAE6
:1037500002A93C30CDED067A4EF00AFC04F531505A
:1037600006AA03A908308DED020A4EF001FC04F50B
:10377000315006AA04A914308DED030A4EF0F8FB6F
:1037800096ED688AC6F8647CB5EEC08AF1EE10FA50
:10379000C7D9DDED080A9DED070AA5F0AFFFDDED05
:1037A000090AA5F0ABFFDDED037A38EE087AB4EE36
:1037B000C08AF1EE10FAB4EEE77A94BF0123002339
:1037C000F1EE10FA0AD80233DDED027AB4EEE78AA0
:1037D000F1EE10FA0AD8002BA3D0A3E7B4EEE78AE3
:1037E000F1EE10FA9CBF0133DBB2EDE7012B99D863
:1037F00097E700BFBD37863570B500F50055044624
:1038000095F8AD3E43F0040385F8AD3E4CF00CFF57
:10381000012211214CF064FED5F8B83E93F8CB306C
:10382000002B41D0D5F8940E03681B6898470928EF
:103830000AD1204607F0BEFA30B104F5A04010309E
:10384000BDE8704007F09EBA184BD3F8940E036899
:103850001B69984740B995F99D31032B24D1062166
:10386000204607F093FA0DE095F99D110229F6D153
:1038700095F8AD3EDB07F2D40622204601F0F4FFB6
:103880000028ECD00A4BD5F8940E01225A73036835
:103890001B6C9847034604F53150064ABDE870405A
:1038A00002212C304EF0DEBE70BD00BFB84B0020B0
:1038B0009D800020E05B0C0808B500F5005292F8EE
:1038C000AD3E590717D56FF3820382F8AD3E0A4B20
:1038D0005A7B42B1002200F531505A730221074A47
:1038E0002C304EF0BFFE4CF09FFEBDE80840002299
:1038F00011214CF0F5BD08BD9D800020045C0C0832
:10390000F0B5054685B005F593576846083713F0BE
:10391000E1FD694638460DF0BBFF80B105F5005367
:10392000D3ED687A374CF5EEC07AF1EE10FA08D88C
:10393000354A002328462380D373FFF7BDFF05B027
:10394000F0BD2846FFF7D2FE064628460BF0A6F942
:1039500010B928460BF07CF9A378002E18BF002080
:103960000343DBB2A370002BE9D06378A8BB83BB11
:1039700023780133DBB2082B237003D14EB33846D2
:103980000DF016FF2378092B02D138460DF008FF01
:103990002378092B1DD94FF4857323804CF044FE06
:1039A000022210214CF09CFD83F0D0F96368C01A0C
:1039B00047F23053984209D905F53150134A022194
:1039C0002C304EF04FFE83F0C1F960602846FFF7BF
:1039D00013FF0D4B6278DA73B1E72678002EF8D02A
:1039E000013EF6B22670002BF3D0002EF1D16670A6
:1039F0004CF01AFE324610214CF072FD2846FFF7BB
:103A00005BFFE6E7287F00209D8000201C5C0C08FF
:103A100000F5005393F8AD3E5B0701D5FFF7ECBE10
:103A20007047000073B5044600F5935001A90830B3
:103A300004F500550DF09AFCD5F8283C8342064663
:103A40000CD004F58043D3F8380976F05FF9C5F857
:103A5000286C4CF0E9FD3E214CF022FD04F5805627
:103A600095F92C1C96F9782596F8783591421BD05B
:103A7000FF2B19D004F58043D3F8380976F046F9C6
:103A800096F8783585F82C3C4CF0CEFD95F82C2C2A
:103A900018214CF025FD04F5315095F92C3C034AD2
:103AA00004212C304EF0DEFD02B070BD2C5C0C0801
:103AB0002DE9F0438FB0054683F048F900230593C4
:103AC00006930793089309930A930B930C930D9312
:103AD00005F5935804AB019308F1080803AB009374
:103AE00006460BAB08AA05A940460DF0D5FDDFED53
:103AF000477A9DED077AB4EEE77AF1EE10FA0746C1
:103B000030DB9DED0A7AB4EEE77AF1EE10FAACBF45
:103B10000124002405F50059404699F8603C002B2B
:103B200008BF00270DF0CAFD8046EFB9444699F959
:103B30002C3A012B29D164B1D9F8B83E93F8CB4087
:103B40003CB1D9F8940E03685B69984780F0010096
:103B5000C4B299F8303CCBBBCCB9C9F8346C0FB0C7
:103B6000BDE8F0830024D5E7002CDFD005F5315007
:103B700008304EF08DF990ED007AF7EE007AB4EE51
:103B8000E77AF1EE10FAD2DCD0E70024E1E7D9F8C9
:103B9000340C301AB0F57A7FE1D9C9F8383C0124E9
:103BA00005F5804389F8304CD3F8403983F80C444C
:103BB0004CF03AFD22461D214CF092FC144A05F5CA
:103BC000315002212C304EF04DFDC8E714B1C9F838
:103BD000386CC4E7D9F8380C43F69823361A9E425D
:103BE000BDD905F58043C9F8344C89F8304CD3F879
:103BF000403983F80C44C9F8384C4CF015FD224686
:103C00001D214CF06DFC034AD9E700BF00000034D1
:103C1000445C0C085E5C0C080B4B10B5012204469A
:103C20005A7283F093F804F58042D2F86C3AC31AC2
:103C3000142B08D9C2F86C0A04F590501430BDE872
:103C4000104040F0A5B810BD9D8000202DE9F7433D
:103C5000044604F5005500F50650002318300DF118
:103C600007018DF8073043F091FED5F8B80E90F9B2
:103C7000C030026883B3083BDBB2012B96692BD9B5
:103C80003221B04704F1100011F030FB1F4B04F556
:103C900031581F684FF0000908F12C08F86A0368D2
:103CA000DB69984701281CD183F050F841F2873333
:103CB000A0EB09029A42064605D9154A062140465C
:103CC0004EF0D0FCB1462046FFF7A6FFB86A036865
:103CD00003215B689847E1E79369B5F8AC11984711
:103CE000D0E70121D5F8B80E7BF034FED5F8B80E38
:103CF0000368DB6A984757F099FFF86A03681B6806
:103D0000012103B0BDE8F043184700BFE07E00206A
:103D10007C5C0C0870B5044600F531502DED028B2B
:103D2000174A184E9FED188A06212C304EF09AFC47
:103D30002046FFF78BFF2046FFF76EFF20460AF074
:103D400007FD3368986A036803215B68984758F059
:103D5000DFFA054658F076FA04F50053D3F8D02A76
:103D6000D3F8B80EB2F9082000EE102AB8EEC00A57
:103D700020EE080A7DF0C8FA284658F06BFADAE718
:103D8000A05C0C08E07E00206F12833A2DE9F0471A
:103D9000044600F531502DED028B2A4ADFF8AC9035
:103DA00006212C304EF05EFC2046FFF74FFF58F006
:103DB000AFFA04F50056054658F044FAB7EE000A8B
:103DC000D6F8B80E7DF0A0FA284658F043FA82F0F3
:103DD000BDFF41F2873A074682F0B8FFC01B50454D
:103DE000D9F8008017D99FED188A284658F02AFA8A
:103DF000B0EE480AD6F8B80E7DF086FA284658F09C
:103E000029FA2046FFF708FFD8F8280003680321A5
:103E10005B689847E9E7284658F014FAB7EE000ABD
:103E2000D6F8B80E7DF070FA284658F013FA2046FE
:103E3000FFF7F2FED8F82800036803215B68984773
:103E4000CAE700BFD05C0C0800000000E07E002044
:103E50002DE9F34100F500550446D5F8B83E93F935
:103E6000C030032B29D0354F652600F58048013E30
:103E700016F0FF060CD0D8F8683A4BB93B68986A40
:103E8000036814215B68984720460AF061FCEEE75E
:103E900004F52F5001212C30F9F77AFE95F998316D
:103EA00070B953B1092B08D08DF8070004F50650FE
:103EB0000DF10701183043F069FD02B0BDE8F08153
:103EC000032B34D8DFE803F002252D30D5F8D03AA3
:103ED000B3F9082040F2B5339A422ADD04F50650C2
:103EE00001250DF1070118308DF8075043F04EFD04
:103EF00004F53150124A02212C304EF0B3FB114B25
:103F00005D720E4B1C68A06A036805215B689847C8
:103F1000F9E7D5F8D03AB3F9082040F2B5339A4220
:103F200007DD2046FFF7F6FE2046FFF72FFF092B9F
:103F3000C3D000238DF80730B8E700BFE07E002033
:103F4000F45C0C089D80002000F531500B46024ABD
:103F500004212C304EF086BB145D0C0810B50446CD
:103F60004CF062FB002205214CF0BAFA04F5315006
:103F7000034ABDE8104004212C304EF073BB00BF53
:103F8000205D0C0813B50B464AB100F53150009284
:103F90000421054A2C304EF065FB02B010BD02B082
:103FA000BDE81040FFF7D0BF385D0C0808B500F53C
:103FB0003150064A04212C304EF054FB4CF034FBB7
:103FC000BDE80840002208214CF08ABA4C5D0C087C
:103FD00038B504460D4682F0B9FE04F500533DB9EC
:103FE000D3F8A42EC3F8A80E0AB9C3F8A40E38BD9E
:103FF000D3F8A82E801A642882BF0022C3F8A82E06
:10400000C3F8A42EF3E7000037B5044600F592404C
:104010001C307AF0E5FC04F50052C0F3803592F8CC
:104020008A3EC3F34001A9421DD065F3410304F564
:10403000315482F88A3E2C346DB14CF0F5FA0222EC
:104040000B214CF04DFA094A0221204603B0BDE88D
:1040500030404EF007BB4CF0E7FA2A460B214CF0FB
:104060003FFA034AF0E703B030BD00BF645D0C08BF
:10407000805D0C0838B50A460C460621054601F05D
:10408000F3FB28B1054A137843F00803137038BDD9
:1040900021462846BDE8384006F078BEBC800020A6
:1040A00038B50A460D461521044601F0DDFB28B15E
:1040B000094A137843F00803137038BD04F53150F2
:1040C00004212C30054A4EF0CDFA29462046BDE8A1
:1040D000384006F05BBE00BFBC800020905D0C083D
:1040E00038B50A460D461521044601F0BDFB28B13E
:1040F000094A137843F00803137038BD04F53150B2
:1041000004212C30054A4EF0ADFA29462046BDE880
:104110003840FFF7AFBF00BFBC800020B85D0C087F
:1041200038B50A460D461B21044601F09DFB28B117
:10413000094A137843F00803137038BD04F5315071
:1041400004212C30054A4EF08DFA29462046BDE860
:104150003840FFF78FBF00BFBC800020CE5D0C0849
:1041600038B50A460D461121044601F07DFB28B101
:10417000094A137843F00803137038BD04F5315031
:1041800004212C30054A4EF06DFA29462046BDE840
:10419000384006F0FBBD00BFBC800020E05D0C088D
:1041A00010B500F5005494F88A3E9A0623D4D4F84A
:1041B000940E03681B689847032808D005D8022886
:1041C0000ED194F8880EC00914E01B28F9D194F898
:1041D000880E00F0A000A0F180035842584109E089
:1041E000B4F8880E20F4FE4020F07F0080B2003842
:1041F00018BF012010BD0120FCE7000038B500F514
:104200000055044695F8AD3E184A43F0080300F502
:10421000315085F8AD3E02212C304EF023FA4CF09F
:1042200003FA012217214CF05BF92046FFF7B8FF93
:1042300040B104F52F500122BDE8384015212C3043
:10424000F9F7B2BED5F8940E03681B6898470628A4
:1042500006D104F5A2402830BDE8384007F09CBFE5
:1042600020460B21BDE83840FFF704BFF45D0C0881
:1042700070B500F500550646D5F8A42ED5F8A83E31
:104280009B1A41F28832934211D9D5F8940E0368F3
:104290001B6D9847044695F8AD3EC3F3C003A34297
:1042A00013D034B13046BDE87040FFF7A7BF0024FB
:1042B000F1E74CF0B9F9224617214CF011F995F8C5
:1042C000AD3E64F3C30385F8AD3E70BD0B46013BC4
:1042D0001146062B18D8DFE803F00406080A0C1371
:1042E000150006F053BDFFF7C5BEFFF7F9BEFFF797
:1042F000D7BE00F52F50012214212C30F9F754BEFF
:10430000FFF70EBFFFF72CBF7047000070B50446E3
:1043100004F500554CF088F9012205214CF0E0F835
:1043200095F88231072B98BF304A204694BFD65C5F
:104330000126FFF735FF68B12D4A2E492046FFF7C9
:1043400021FE04F52F50012210212C30F9F72CFE0C
:10435000002614E0D5F8940E0368DB6C9847A8B1EA
:1043600004F5405393F80D2482B193F90C34012BDA
:104370000CDC214A21492046FFF704FE0126314684
:1043800020460322BDE87040FFF7A0BFD5F8940E89
:104390000368DB6C984718B1D5F8303A190715D483
:1043A000D5F8940E03681B689847032803D1D5F805
:1043B000303ADA070DD4D5F8940E03685B6A984753
:1043C00068B90C492046FFF7BFFDD8E70A4A0949FA
:1043D000D1E70B4A07492046FFF7D4FDB8E7D5F8E7
:1043E000303A5B07EDD5074AF4E700BFDC5E0C0806
:1043F000145E0C081E5E0C08245E0C08375E0C0868
:10440000475E0C08575E0C0870B5044615464CF024
:104410000BF9012206214CF063F82046FFF7C0FE9D
:1044200098B104F52F50012207212C30F9F7BCFD7B
:10443000134A14492046FFF7A5FD002529462046CA
:104440000422BDE87040FFF741BF04F50056EDB20D
:10445000D6F8940E0368DB6C984758B1D6F8303A1A
:104460001B0707D535B1084A06492046FFF78AFDE4
:104470000125E3E703492046FFF766FDDEE700BFBD
:10448000145E0C08765E0C08245E0C08F8B5044631
:1044900004F500554CF0C8F8012208214CF020F832
:1044A00056F024F995F87131072B9CBF364AD65C3B
:1044B000D5F8B83E93F8CB7088BF02265FB9334970
:1044C0002046FFF741FD0026314620460522BDE883
:1044D000F840FFF7FBBE2046FFF762FE60B104F52F
:1044E0002F50012212212C30F9F75EFD284A27496E
:1044F0002046FFF747FDE6E7D5F8940E0368DB6C2E
:10450000984778B104F5405393F80D2452B193F9CC
:104510000C34012B06DC1F4A1F492046FFF732FDF1
:104520000126D1E7D5F8940E0368DB6C984718B1E3
:10453000D5F8303A190713D4D5F8940E03681B68E0
:104540009847032803D1D5F8303A9A070BD4D5F809
:10455000303ADB0609D40D492046FFF7F5FCB3E7F6
:104560000C4A0A49D9E70D4AC1E7D5F8940E036809
:10457000DB69984705460028EDD1094A03492046E2
:10458000FFF700FD2E469FE7E45E0C085F4A0C082B
:10459000145E0C08245E0C08705E0C087E5E0C082D
:1045A000935E0C0870B500F50055044695F971311D
:1045B000ABB3D5F8186E96B382F0C8FB05F6882326
:1045C00093ED000ADFED167A9FED161ADFED160A5D
:1045D000861B20EE270A8D2023F044FFBCEEC00A84
:1045E00010EE103A9E420CD295F8AD3E9A0716D5C1
:1045F00020460021F9F732FE2046BDE87040FFF763
:10460000D5BC0CD995F8AD3E9B0708D420460121B6
:10461000F9F724FE2046BDE87040FFF737BF70BDB4
:1046200000007A440000804F000000002DE9F341B3
:10463000074600F592401C307AF0D2F907F5005495
:10464000C0F38048019082F081FB94F8B03E43456E
:10465000454606460DD007F5315084F8B08E2C3013
:10466000002D3FD03A4B3B4AC4F8B46E02214DF0C6
:10467000F9FF94F8B03E43B394F8B13E2BBBB4F9C4
:104680009E3A9FED350A9FED351ADFED350A07EEAC
:10469000903AF8EEE77A40F2571027EE800A23F0BE
:1046A000E1FEBCEEC00AD4F8B40E10EE103A361A91
:1046B0009E420AD9012307F5315084F8B13E294AB8
:1046C000234B02212C304DF0CDFF94F99D3A002B65
:1046D00094F8AD3E0DDC6FF3451384F8AD3E02B0A7
:1046E000BDE8F0811A4B204AC4F8B48E84F8B18E2C
:1046F000BCE7C3F34012AA42F1D065F3451384F836
:10470000AD3E9B06EBD5194BD3F8940E03681B699D
:1047100098470028E3D04BF087FF01221F214BF080
:10472000DFFE3846FFF73CFD48B107F52F50012268
:1047300021212C3002B0BDE8F041F9F735BC94F8E6
:104740009D1A3222384602B0BDE8F041FFF7BEBDE7
:10475000AC5E0C08BB5E0C0800007A440000804F81
:1047600000000000D15E0C08C65E0C08B84B0020AB
:1047700008B5044B01221A7082F0DCFA024B186073
:1047800008BD00BF317F0020347F0020014B002294
:104790001A707047317F00202DE9F041044682F005
:1047A000C9FA2A4BB4F8BE201988294E9142054611
:1047B0000ED01A80274B18603378A3B100243470D0
:1047C0004BF032FF22461321BDE8F0414BF088BE8A
:1047D0003378214FDBB93B782BB11E4B1F4A1B6846
:1047E000C31A934201D8BDE8F0810123337004F568
:1047F0000053D3F8B80E90F8CB3013B103689B6A1E
:1048000098474BF011FF012213214BF069FE3B78D2
:10481000002BE8D03378002BE5D00E4A10491368FE
:10482000EB1A8B42DFD904F500541560D4F8B80EAA
:1048300090F8CB30002BD6D000217BF08BF8D4F849
:10484000B80E0368BDE8F0415B6A1847327F00206C
:10485000307F0020347F0020317F002080841E00C4
:1048600040420F002DE9F04100F500550446D5F80F
:10487000940E95F884700368DB6C9847014650B934
:1048800095F9883E002BA5BFD5F8B83E93F8CB002C
:10489000012180F0010104F5015808F108084046A3
:1048A0005FF0CEFDD5F8B83E93F8CB300646002B2E
:1048B0007BD0002865D03E4B93F9883E002B04DB6B
:1048C00002463C4940465FF095F995F94E7057B164
:1048D00095F9883E002B0EDA04F52F5001220F21A6
:1048E0002C30F9F761FB4BF09FFE3246BDE8F041FA
:1048F00009214BF0F5BDD5F8940E03685B69984724
:1049000058B195F9893E002B07DA95F8AD3EDA07E4
:1049100003D495F88430DB07DED5314640465FF09E
:10492000F5FDDFED257AB4EEE70AF1EE10FA05DDCC
:104930000A220921204600F097FFD4E7023F032F07
:1049400011D801A353F827F031490108594901084A
:10495000774901087D4901080A221521204600F007
:1049600083FF0028BFD10A220621204600F07CFFE9
:104970000028B8D1DCE70A221121F6E70A22152126
:10498000F3E797B195F884307BB9094B93F9883EEA
:10499000002B06DB04F53150084A05212C304DF080
:1049A00061FE4BF041FE0022A0E7BDE8F08100BFB0
:1049B000B84B0020EC5E0C080000C842F55E0C0805
:1049C00070B500F5005300F592451C3586B093F89C
:1049D000301C0446284679F0B1FF02A812F07AFD97
:1049E00004F5935002A908300CF002FF04F580434F
:1049F000049AC3F81429059AC3F81829284679F0AF
:104A0000EFFF82061AD5284679F0F8FF04F59245A3
:104A1000FDEEC07A0C3504F5805417EE901A022290
:104A2000284617EE906A12F05BFD94F8E434DB0739
:104A300006D401223146284612F052FD06B070BD60
:104A40000121284612F0DEFD0028F2D0F6E7000032
:104A500070B500F5804486B0B4F89C3A8B420D46A0
:104A6000164603D1D4F8983A934221D082F06EF9D9
:104A7000D4F8943AC31A132B1AD9C4F8986AA4F834
:104A80009C5AC4F8940A4BF0CFFD044682F066F9B4
:104A9000084B094A1B68CDE90453084B0193084BA6
:104AA0000093CDE90201074B074920464BF048FB34
:104AB00006B070BD387F00200C5F0C08245F0C0826
:104AC000E4340C0820180C081F5F0C0838B500F5FA
:104AD00000540D4694F8893EC3F380138B420BD0EB
:104AE00021B14BF0A1FD11214BF0DAFC94F8893E85
:104AF00065F3861384F8893E38BD0000F0B52DEDCE
:104B0000048B00F500558BB0D5F8B83E93F8CB3048
:104B1000064600F58044002B67D095F9883E002BAF
:104B200063DBD5F8940E03685B699847002861D170
:104B3000D4F838099FED430A6C3026F0A1FE0AAA8A
:104B4000CDED080A8DED091A8DED070A12E907006F
:104B500004AB01AF83E8070087E80700384626F07A
:104B6000FDFBD4F8383906F591406C30D3ED368A28
:104B7000B0EE409A4DF0B0F927F080FAD4F8403901
:104B8000D5F8940ED3EDDB9A0368DB6CB0EE408A67
:104B90009847DFED2D7AB4EEE79AF1EE10FA02DCD9
:104BA00095F8903E0BB1002838D0DFED287A68EEFA
:104BB000A78AF3EE0E7AF4EEE78AF1EE10FA2DDC16
:104BC000F0EE087AB4EEE78AF1EE10FA26DCF5EEA4
:104BD000C09AF1EE10FA21DAD4F8380903689B6F15
:104BE00098470BB0BDEC048BF0BDD4F838090368CE
:104BF0009B6F0DE0D5F8D02AD4F83809B2F9082017
:104C00000368002A03DCD5F88C2E022AF0D1DB6F72
:104C10000BB0BDEC048BBDE8F0401847D4F8385910
:104C2000DFED0B0A2B68D3F88060D4F8403940F2EE
:104C3000AB1093EDC90AB7EE001A23F013FC284617
:104C4000B047CEE79F0CB3450080BB44E02E6542E1
:104C50000000000000F5005090F8900E7047000032
:104C6000F8B500F50054064694F8883EB1EBD31F22
:104C70000D4644D0224B00221A6000293BD04BF055
:104C8000D3FC12214BF00CFC94F8883E65F3C7135B
:104C900085F0010784F8883E6AF0D2FA39466AF056
:104CA000ABFA37B194F806311BB982F04FF8C4F86B
:104CB000080184F8067115B3B4F854315B071ED5AA
:104CC000D4F8B83E93F8CB30CBB1D4F8940E036847
:104CD0005B69984798B9D4F8940E036820219B69C2
:104CE000984760B106F52F500122BDE8F8400D212C
:104CF0002C30F9F759B94BF097FC1C21C2E7F8BDED
:104D0000387F00202DE9F04F2DED0A8B00F500557E
:104D10008DB0D5F8B83E93F8CB60044600F58047D7
:104D20001EB90121FFF79CFF0BE095F9882E002AA0
:104D300065DAD5F8940E03689B6C98470646002800
:104D400041D04FF0000B95F9882EB24E002AC0F2E8
:104D50005581D6ED007AB4F9A420B8EE677A1AB975
:104D6000B4F8A220A4F8A420B4F8A430DFEDAA6A15
:104D700007EE903AF8EEE77A67EEA67AB4EEE77AB5
:104D8000F1EE10FAACBF012100212046FFF79EFE94
:104D900095F9882E002A95F8892EB8BF4BF0010BA3
:104DA000530697F8802A48BF4BF0020B0AB14BF02C
:104DB000080B3268594620460DB0BDEC0A8BBDE8A1
:104DC000F04FFFF745BED5F8B83E204693ED0C8A6C
:104DD000F9F714FBB4EEC80AF1EE10FAB1D5D5F824
:104DE000B83E93F8A130032BABD149F029FF4FF423
:104DF0008011422249F0DCFE3146204692E797F8C6
:104E000080AABAF1000F03D0824A0023136098E70A
:104E1000D7F8380993F8079003685B6F9847804686
:104E20000090D5F8940E03685B69984720B1D5F8D7
:104E30008C3E022B00F0E480B9F1000F0CBF4FF064
:104E4000000B4FF4007BB7EE00BAB8F1000F02D0B0
:104E50004BF4806B009604F5944808F148084046EE
:104E600062F0CCFC0130D7F838099FED6C0A9FED59
:104E70006CCADFED6C8A0CBF012302236C3008EE94
:104E8000103A26F0FDFC0CABCDED0A0A8DED0B1AA5
:104E90008DED090A13E907000DF10C0E0DF1180C48
:104EA0008CE807008EE80700704626F057FAD7F81E
:104EB0003829DFED5D7A92ED36AA2AEE27AAB4EE04
:104EC000CC0AF3EE0EBAF1EE10FA04F59140B4EE0E
:104ED000EBAAC8BF4BF4807B6C30F1EE10FAC8BF70
:104EE0004BF4807BF0EE40AA4CF0F6FF27F0C6F8BA
:104EF000B8EEC88A04F59240B4EEC80AF1EE10FA92
:104F000000F11C0098BF4BF0800BF0EE409A79F056
:104F100081FD68EE288AB0EEC09AB4EEE89AF1EE10
:104F200010FA204648BF4BF0400B09F0F7FC002870
:104F300046D14BF0200B0196404662F05FFC012801
:104F40004FD14BF0100BB2463249B9F1000F53D09C
:104F5000009B002B50D0F4EECCAAF1EE10FA4BDC03
:104F6000B4EEEBAAF1EE10FA46DCF4EEC89AF1EEDC
:104F700010FA41D8B4EEE89AF1EE10FA3CD5019B54
:104F8000D3B3BAF1000F37D00A68B4F9A40007EE22
:104F9000902AB8EE677A18B9B4F8A200A4F8A40071
:104FA000B4F8A43007EE903AF8EEE77A67EE8B7A21
:104FB000B4EEE77AF1EE10FA19D501320A60C2E6D2
:104FC00004F52B502C304CF063FFDFED187A90ED98
:104FD000007AB4EEE77AF1EE10FAAAD40023019336
:104FE000AAE7404662F00AFC0130ADD1A9E70121F1
:104FF0002046FFF735FEA6E60022DFE70121C4E6E2
:10500000B9F1000FB0EE08BA0CBF4FF0000B4FF42F
:10501000007B1DE7387F0020CDCC4C3E9F0CB34574
:105020000080BB440000C842E02E654200004843B7
:1050300030B500F5AD531833044693E8070089B046
:1050400002AD85E807009FED1D7ADDED047A77EE6D
:10505000877A9FED1B7ACDED047AD4ED2B7AF0EEB2
:10506000E77AF4EEC77A04F59140F1EE10FA00F118
:105070006C000BD5B4F9A23007EE903AF8EEE77A5F
:10508000F7EE006A86EEA77A84ED2B7AD4F8AC307E
:10509000019301AA29464CF091FF2046FFF732FE0A
:1050A0002046FEF781F92046FEF758FA2046FEF723
:1050B00021F82046FEF7C8F809B030BD0AE81C41C7
:1050C0000000003410B504462DED028B1D2056F073
:1050D0003DFF60B304F50053D3F8940E00F0C2FA1C
:1050E000192108EE100A04F5516043F0EBF802288C
:1050F0001AD00338012808D804F52B502C304CF076
:10510000C7FE90ED008ABDEEC88AB8EEC88A9FED52
:10511000090A28EE000ABDEC028B04F594404830E1
:10512000BDE8104062F0F0BB9FED038AEDE7BDECF7
:10513000028B10BD0AD7233C00000000134A026016
:10514000134A426002F1740181601249C16002F5A4
:10515000205101610839416124398161A2F56E61F4
:10516000C1610D49016202F55761416202F51861A2
:10517000816202F68411C16202F6881102F68C1275
:105180004263064A01638263704700BF58700C088F
:10519000004D0020FC740020F0740020D02C002072
:1051A0001C2953D8DFE801F0130F171B27232F1FEB
:1051B000522B52335252373B3E424652524A52527F
:1051C000525252524E0000F595402430704700F57F
:1051D000A3403430704700F595406430704700F5C7
:1051E00096402030704700F59D407C30704700F5B8
:1051F000A0405830704700F59F404C30704700F594
:10520000A0401030704700F5A2402830704700F5EC
:105210009E403C30704700F59E407830704700F566
:105220009940FAE700F5A1401430704700F59D4021
:105230003830704700F5A3407030704700F5A44047
:105240004030704700F5A5405C3070470020704743
:1052500073B50B6805461B6C08460C461646984706
:10526000034605F531500F4A009604212C304DF0CD
:10527000F9F94BF0D9F9236805461B682046984791
:105280000A21024628464BF02BF9074B93F8893E3A
:105290009B0641BF054A137843F00403137002B024
:1052A00070BD00BF285F0C08B84B0020BC800020F8
:1052B00038B50C4A182305460C4649F033FB78B143
:1052C00021462846FFF76CFF30B10146064A2846C2
:1052D000FFF7BEFF002038BD284649F069FAF9E71C
:1052E0000120F8E7A85F0C08485F0C0810B500F52E
:1052F0000054002384F8803B084B00F5804093F86D
:10530000881ED0F83809C90973F0ACF9D4F8940EA6
:105310000368BDE81040DB68184700BFB84B0020A9
:1053200070B50546086803685B690C4616469847E1
:1053300090B1306803685B69984768B905F5005318
:10534000D3F8B82E92F8CB2032B193F9883E002BD7
:1053500002DB2846F9F768F804480AF093F8206859
:105360000368BDE870409B68184700BFF87F0020C5
:1053700070B500F500550446D5F8940E0B4E036841
:10538000DB6998473074D5F8940E03681B6898471A
:10539000F070D5F8940E03685B6C9847014604F5ED
:1053A00090501430BDE870403EF03CBD9D80002020
:1053B00070B52DED028B244B93F8AD3EDB0782B028
:1053C00006460D461446B0EE408AF0EE608A06D5D9
:1053D00000232B60236002B0BDEC028B70BD55F042
:1053E00085FA037F002BF3D0F36A9FED181A1B6830
:1053F0009FED170AB3F9083007EE103AB36A1B683D
:10540000B3F9083007EE903AB8EEC77AF8EEE77ACB
:1054100067EE000A68EE811A27EE800A28EE011A6C
:1054200001A9684623F012FFDFED0A6A9DED007ABC
:10543000DDED017A27EE267A67EEA67A85ED007A11
:10544000C4ED007AC7E700BFB84B00200AD7233C61
:10545000530469390000C84270B52DED028B88B045
:10546000002302930393364B93F8AD3E13F0010FE4
:105470000646B0EE408A06AD02AC03D155F036FACE
:10548000037F5BB994E8030085E803009DED060AFD
:10549000DDED070A08B0BDEC028B70BDB36ADFED2D
:1054A000296A1B68B3F9083007EE903AF36A1B6863
:1054B000B3F9083007EE103AB8EEC77AF8EEE77A9B
:1054C00027EE267A67EEA67AF1EE476ACDED026AFC
:1054D000DFED1D6ACDED037AB0EEC77AB4EEE67A61
:1054E000F1EE10FA06D5F0EEE77AF4EEE67AF1EE98
:1054F00010FAC7D403AA21461448F8F7C5FFDDED1A
:10550000027A9DED037AF0EEE77AB0EEC77AF4EE18
:10551000477AF1EE10FACCBFB0EE670AB0EE470A58
:10552000204625F069FE04A88DED040ACDED050A9C
:1055300025F014FF204688EE000A25F08DFEA1E735
:10554000B84B00205304693900000034B82B002008
:10555000094B93F9882E002A0CDAB5EEC00AF1EE59
:1055600010FA07D9D3F8B83E93F8A100C31E5842E9
:105570005841704700207047B84B0020436A1B68B1
:1055800093F8CB3043B1054B93F8880E00F0A000A0
:10559000203818BF0120704701207047B84B002009
:1055A00010B5436A04461868D1B102217AF0E2F9D5
:1055B000236A9FED0C1A18680368F0EE410ADB6A53
:1055C000B0EE410A9847236A074A1868D2ED540A98
:1055D00003689FED040A5B6EBDE810400021184788
:1055E0000121E3E700000000B84B002010B5436A3A
:1055F00004461868002930D002217AF0BBF9236AEA
:10560000186872F0FFFF636A1B6893F8A130012BE2
:1056100004D8236A0121186873F08EFD6369186845
:1056200076F09AFE6369186876F0F6FE63699FED7E
:105630000C0A186877F01CF96369186877F08AF922
:10564000236A9FED071A18680368BDE81040DB6AFB
:10565000F0EE410AB0EE410A18470121CDE700BF44
:105660000000000013B5044601A90C4809F0E0F958
:1056700010B1019802B010BD6369186875F076FD2D
:1056800018B9074BD3F81009F4E7064801AA03211B
:1056900011F05CFF0028F4D0EBE700BFB82B00202E
:1056A000B86B0020C474002070B504462DED028B49
:1056B00000296AD18368B3F96258642DB8BF6425A4
:1056C000FFF7D0FFA8426268A4BF324B93F8895E0F
:1056D000B2F93430ACBFC5F380150125002BDBBF18
:1056E00063691B685B4293EDC48AC8BF07EE903ABA
:1056F000B2F93230C8BFB8EEE78A002BB8BF5B42C0
:105700009BB25B4207EE903AA368F8EEE77AB3F9F2
:105710006268F4EEC87AF1EE10FAD8BFB0EE678A8C
:105720002046642EB8BF6426FFF79CFF6369A26B16
:105730001B68D2ED001A93EDC61AD3ED0E0A311A8A
:1057400000EE101AB8EEC00A23F06EF96368B3F9E0
:105750003230002BB8BF5B429BB25B4201EE103A85
:1057600040F29720B8EEC11AF0EE480A22F07AFE15
:1057700063692946186875F09DFDBDEC028B63696D
:10578000BDE87040186877F0E5B89FED030A002582
:10579000EEE700BFB84B002000000000436A186825
:1057A00003681B691847000038B52DED028B0368AC
:1057B0000446D3F880309847236B2A481B68F0EEE4
:1057C000408AB3F9085009F049F84FF47A72041E80
:1057D0004FF000012846D8BF4FF4FA7422F080FE43
:1057E0008442B6EE000A2ADD07EE900AB8EEE77AA8
:1057F00007EE904A27EE007AF8EEE77A87EE278ADE
:105800004FF46D7038EEC00AF5EE087AB1EE400A3A
:1058100080EE270AB7EE001AFEEE000A22F022FE02
:10582000F7EE007A77EEC07A28EE000A20EE080A3A
:1058300020EE080AA7EE880ABDEC028B38BD031BD8
:1058400007EE103AC4F57A74B8EEC77A07EE904ABC
:1058500027EE007AF8EEE77A87EE278A38EE008A9C
:10586000CEE700BFB82B00202DE9F04F2DED028BC5
:1058700000F5804900F5005599F8A04A89F8A02A5A
:105880000646D5F8940E036883B01B688846174611
:10589000984740451FD11A2F85F8047107D130B9B8
:1058A00005F66425D9F838392A68C3F8FC208B4BF3
:1058B00093F8893E980606D40124204603B0BDEC37
:1058C000028BBDE8F08FBC42F6D0854A137843F0D6
:1058D00002031370F0E7022F0DD0B8F11B0F12D1A5
:1058E00006F596403946203003B0BDEC028BBDE88A
:1058F000F04F01F053B941463046FFF7D9FC04465A
:105900000028EAD1D9E741463046FFF749FC044672
:10591000019018B9304648F04BFFCEE7D5F8B83EB5
:1059200093F8CBB003685B699847019A06F59E43EC
:105930003C338BF0010A9A4208BF0120BBF1000FF3
:1059400008D10198036851465B689847044648BBF4
:10595000644A22E095F9883E002B80F2B18000284D
:1059600000F0AE80DFF874B1DBF8940E03685B6979
:1059700098470446002840F0A3800198FFF714FFE1
:10598000ABF50050B0EE408AF8F738FDB4EEC08AAF
:10599000F1EE10FA40F39480534A01993046FFF734
:1059A00057FC8AE706F53A5101AA14313046FFF751
:1059B000B7FC0198C5F8940E85F8047103681B685C
:1059C00098473A46014606F57C604AF03FF906F5ED
:1059D000315000212C3054F0B7F895F94E3023B1F6
:1059E00006F5015008305EF0B5FDD5F8940E036859
:1059F0001B689847C21E5042504105F6342289F870
:105A0000C809D9F838391268C3F8F82005F66422B5
:105A1000D9F838391268C3F8FC20B8F1010F02D068
:105A2000B8F10B0F06D105F64C25D9F838392A689C
:105A3000C3F8FC203046FFF79BFC284B93F8893EC7
:105A40009B063FF542AF37E795F84830002B3FF40F
:105A500078AFB5F86430D9077FF573AF95F8843027
:105A6000002B3FF46EAFD5F8B83E93F8CB30002B47
:105A70003FF467AF95F804310A2B7FF462AF95F9D4
:105A8000883E002BFFF65DAF184A01993046FFF7BC
:105A9000DFFB002411E7164809F040F90028D3D1B4
:105AA000D5F8940E03685B6998470028CCD001981C
:105AB00003685B69984704460028C5D10D4A6CE726
:105AC000019803681B6998470028E4D0084809F04A
:105AD00013F904460028DED1074A5EE7B84B0020E0
:105AE000BC8000204EEC0D08705F0C08945F0C0821
:105AF000B82B0020825F0C084E9F0D080148FFF76D
:105B0000B3BE00BFB82B002013B504468DED010ACB
:105B100061F00CFE6369A26B1B6892ED001A93EDB5
:105B20000E0AD3EDC60A01A960F08EFC9DED010AB4
:105B300002B010BD436A186803685B6A184700002A
:105B400038B5436A1C6894F8CB10054661B9204605
:105B500079F010FF6B6A1B6893F8A10018B1012857
:105B600014BF0320022038BD164803783BBBFFF763
:105B7000EFFC20BB144A92F8883E03F0A003202BD0
:105B800017D0B5EEC00AF1EE10FA10D592F88A3EA1
:105B90005B070CD40121204679F0ECFE6B6A1B6890
:105BA00093F8A130012B0CBF02200320DBE7022178
:105BB000F1E72046022179F0DDFE0420D3E7012041
:105BC000D1E700BFF87F0020B84B002010B52DEDC5
:105BD000028B134B93F8AD3EDB07044604D59FEDD3
:105BE000110ABDEC028B10BD54F080FE037F002B28
:105BF000F5D0636B186854F0A3FFA368DFED0A7A51
:105C000003F6AC0292ED008A03F50B63D3ED000AB4
:105C100028EE278A23F0D4FA28EE000AE1E700BF35
:105C2000B84B0020000000000000C8420148F8F70F
:105C300059BC00BFB82B00200148F9F7D5B800BF08
:105C4000B82B00200148FFF70FBE00BFB82B002083
:105C500070B57E4D2DED028B95F8893E8CB00026F7
:105C6000044658060496059603D56369186875F0CE
:105C7000F1F895F8AD3ED9075DD463689B899A0722
:105C80001BD573484CF004F9DFED727A90ED007A81
:105C9000B4EEE77AF1EE10FA0FDD4AF0C5FC3D21D3
:105CA0004AF0FEFB6C4809220521FFF7DDFD20B913
:105CB000092202212046FFF7C5FF636893F954309B
:105CC000CBB365489FED658AF9F78EF8E3689FEDE1
:105CD000647A1B68D3ED0A7AF4EEC87AF1EE10FA12
:105CE000B8BFF0EE477AB6EE000A27EE800A2046EB
:105CF000FFF7B2FB8DED040AB0EEC00AB4EEC80A9D
:105D0000F1EE10FACDED050A06D5F0EEE00AF4EE5C
:105D1000C80AF1EE10FA0ED495F88A3E1B0704D497
:105D20004AF082FC49214AF0BBFB95F88A3E43F0D9
:105D3000080385F88A3E95F88B3E09966FF3820337
:105D400085F88B3E60690A9609AE324604A9006860
:105D5000012375F0E9F86369186876F05DFB636903
:105D6000186875F035FCA3688DED060ACDED070ABD
:105D70008DED081AD3ED007AF5EEC07AF1EE10FA47
:105D800051DDB5F944319FED378A00EE903AF8EED7
:105D9000E00A2046CDED030AFFF764FCA368DDEDC1
:105DA000030AD3ED001A9FED2B0AB7EE002A07EE87
:105DB000900A31EE822AB8EEE71A22EE082A61EE46
:105DC000881A22F08FFADFED287A20EE270ADFED1D
:105DD000277A20EE270AA3F061FDDFED257A20EE79
:105DE000270A06A820EE088A25F0B8FAB4EEC08A81
:105DF000F1EE10FA17D5C8EE006A63699DED067AD8
:105E0000DDED077A27EE267A67EEA67A8DED067A23
:105E1000CDED077A1B68D3F88823C3F89423D3F811
:105E20008C23C3F89823236A12491C683046FCF778
:105E300029FB0B9B009396E80C0006A9204672F004
:105E400093FC0CB0BDEC028B70BD00BFB84B0020C2
:105E5000B874002000002F44B82B0020000000344C
:105E600000007A430000C8420AD7233C35FA8E3C32
:105E70000AE81C41EC7E002013B504460191FFF7AF
:105E8000E7FE0199204602B0BDE81040FFF70CBCC8
:105E90000148FEF7E5BE00BFB82B00200048704760
:105EA000245800200148F8F70BBB00BFB82B002096
:105EB00030B50F4D87B0002304466946D5F8400938
:105EC00000930193029375F09BFBD5F8400902A95A
:105ED00075F0EAFB009B0393019B04930222029B53
:105EE000059303A9204611F001FE204607B030BDFE
:105EF000B86B0020002070470020704700207047DA
:105F00000020704700207047002070470020704735
:105F10000020704700207047002070479FED010A65
:105F2000704700BF0000000000207047002070474D
:105F30000020704701207047002070470020704704
:105F400001207047002070470120704701207047F2
:105F500000207047012070470120704700207047E3
:105F600000487047C05F0C0800487047C05F0C08CD
:105F7000836893F8C038DB0706D5002380F83C30EF
:105F8000024B0222C3F88C2E01207047B84B002030
:105F900090F83C3043B9836893F8C038DB0742BFC0
:105FA000034B0122C3F88C2E002380F83C3070474D
:105FB000B84B0020012380F83C3070472DE9F043B6
:105FC0002DED0C8BF0EE409A20EE000A97B00025E4
:105FD000A0EEA00A04468946B0EE41CAF0EE60AADF
:105FE00090461F46019502950395049505950695E3
:105FF000A3F06AFEF7EE00CAB4EEEC0AF1EE10FA76
:10600000C8BFCCEE807AA36803F67C0203F5086370
:1060100092ED009A9FEDC5DAD3ED000AC4BF69EE98
:10602000A79A6AEEA7AAB0EE690A23F0C9F8A36896
:1060300029EE0D9A03F67C0203F50863D2ED008A7F
:10604000D3ED000A29EE009AB0EE6A0A23F0B8F800
:10605000A36868EE8D8A03F6940203F69803D3EDE5
:10606000000A92ED008A68EE808AB0EE4C0A23F0B6
:10607000A7F8636828EE0D8A93F9703028EE008A3D
:10608000002B00F0D980236A9FEDA90A18686C30B4
:1060900025F0F6FBB0EE60AACDED080A8DED091AE9
:1060A0008DED070A22F088F9BDEEC0BAA14940F68D
:1060B000B8321BEE100A22F003FA434207EE903A80
:1060C0006368F8EEE77A93ED1A7A67EE877AB0EEB6
:1060D0004A0ACDED017A22F06FF9FDEEC0BA40F622
:1060E000B83294491BEE900A22F0EAF94242636802
:1060F000039507EE902A93ED1B7A93F97030F8EE32
:10610000E77A022B67EE877ACDED027A6ED18A4B61
:10611000B3F944310AEE103AB8EECBBAB8EECAAAD7
:10612000236AB4EECABAF1EE10FA1A683DDDA3682C
:10613000DFED820AA16B92ED051AD1ED001A03F68C
:106140007C0393ED007A27EE0D7A3AEE4B0AC7EE08
:10615000200A22F069FCDDED017A37EE800A8DED30
:10616000010AB8EEEB0A236AB4EECA0AF1EE10FA9D
:106170001A6834DDA368A16B92ED061AD1ED001AFE
:1061800003F67C03D3ED000A20EE8DDADFED6B0A17
:106190003AEE400ACDEE200A22F046FCDDED027A0E
:1061A00037EE800A8DED020A20E0B1EE4A0AB4EE25
:1061B000C0BAF1EE10FAD4D5A368A16BDFED5F0A87
:1061C000D1ED001A92ED051A03F67C0393ED007AE7
:1061D00027EE0D7A30EE4B0AC7EE200AB9E7B1EE92
:1061E0004AAAB4EECA0AF1EE10FAC3D4236AD3F86D
:1061F00000C00CF184030FCB12AD85E80F000EAE8A
:106200000AAD86E80F0085E80F0004AB01AA294615
:10621000604672F045FF636893F97030022B16D127
:10622000DDED047A39EE279ADDED057A78EEA78A5E
:10623000DDED067A38EE278A89ED009AC8ED008AEE
:1062400087ED008A17B0BDEC0C8BBDE8F083F0EE53
:10625000E99AF0EEEAAAF4EEE9AAF1EE10FA48BFE4
:106260006D46CDED009ACDED0AAAD5ED007ADFEDB1
:10627000340AB0EECCCAF4EECC7AF1EE10FAD8BF04
:1062800035468DED0ECA95ED007ADFED2E7A87EE5C
:10629000270AAD20B7EE001A3CEEC00A22F0E2F861
:1062A000E369D3ED937A04A820EE270A25F0E8FAF3
:1062B000F0EEC07A8DED061AB0EEC91A31EE671A0B
:1062C0008DED040AB0EEC11A39EE000ACDED050AD3
:1062D000B520F1EE410A22F0C5F8B0EE409A9DEDEE
:1062E000050AB0EEE81AF0EEC07A31EE671A38EE21
:1062F000800AB0EEC11AF1EE410ABA2022F0B2F8DB
:10630000F0EE408A9DED060AB0EEC81AF0EEC07AB3
:1063100031EE671A38EE000AB0EEC11ABF20F1EE76
:10632000410A22F09FF8B0EE408A85E70000C8429B
:106330009F0CB34548F4FFFFB84B002000007A449F
:106340000000000000A08C4530B52DED028B836A63
:106350003E4D044687B0186854F0F2FBE36A1868B3
:10636000B0EE408A54F0ECFB636B8DED010A1868C7
:1063700054F0E6FB05ABB0EE401A03A92046DDED74
:10638000010A04AAB0EE480AFFF718FE636A18680B
:1063900090F8CB10002939D179F0ECFA2046FFF7BC
:1063A00003FA636A1B6893F8A1100129B0EE408AD2
:1063B0003BD0032942D051B9236A0121186873F0F8
:1063C00071FD236A186872F007F99FED218A236A2C
:1063D000A268186892F8C02803689DED030ADDEDF5
:1063E000040A9DED051A92074CBFDB6B9B6B984727
:1063F000236AD5ED540A1868036800215B6EB0EE7D
:10640000480A984707B0BDEC028B30BD95F9893E2C
:10641000002B06DBD5F88C3E022B04D190F8A1307E
:106420000BB90121B8E70221B6E7236A186873F0B7
:1064300039FD236A186872F0E5F8C6E7D9790029B2
:10644000C5D12046FFF724FDC1E700BFB84B0020AF
:1064500000000000836893ED140AB5EEC00AF1EE67
:1064600010FA01DCFFF79AB970470000704700008E
:1064700000207047012070470220704700207047BD
:1064800000207047012070470020704781F0010014
:106490007047000001207047012070470048704796
:1064A00058600C080048704764600C0838B54369B0
:1064B0000446186874F07CFF18B96369186876F0B0
:1064C000FBF8636920461D68FFF7ECFC6368B3F9CD
:1064D0003820B3F9363000EE903A434201EE102AEC
:1064E00000EE103AB8EEC11AF8EEE00AB8EEC00AB3
:1064F000284674F049FE636920461D68FFF7D2FC08
:106500006368B3F93820B3F9363000EE903A43426D
:1065100001EE102A00EE103A2846B8EEC11AF8EE45
:10652000E00AB8EEC00A74F0A9FE012038BD0000F0
:1065300030B52DED028B0446436985B01D68FFF729
:10654000B1FC6368B3F93820B3F9363000EE903A05
:10655000434201EE102A00EE103AB8EEC11AF8EEEE
:10656000E00AB8EEC00A28465B4D74F00DFE2046E6
:10657000FFF762FBB5F9443108EE103A236A186858
:1065800003689B6E9847B8EEC88AF0EE400A02AAEC
:1065900001A9B0EE480A2046FEF70AFF2046FFF7A1
:1065A00015FB236B1B68B3F90830F0EE408A00EE50
:1065B000103A2046B8EEC00AFFF738FB2046B0EE8E
:1065C000408A8DED030AFFF76DFC6368B3F936303E
:1065D00001EE103A434200EE903AB8EEC11AF8EEDE
:1065E000E00A2B20B0EE480A21F03CFF20468DED5A
:1065F000030AFFF7A5FA042813D8DFE800F0032FF9
:10660000252A4B00236A186871F0E6FF236A0021EF
:10661000186872F091FD63699FED300A186876F092
:1066200027F9236ADDED020A18689DED010A036867
:10663000B0EE681ADB6A98476369186876F08AF9E1
:1066400005B0BDEC028B30BD236A0121186872F0E1
:1066500073FD236A186871F0D5FFDCE7204D2B78B5
:1066600063B963689FED1F1ADFED1C0A93ED040AFE
:10667000452021F0F7FE284608F0ECFE20469DED6F
:10668000030AFFF741FA16488DED030A03A908F043
:106690001BFFC6E7636A0221186879F06BF9B5F948
:1066A0004431114800EE103A02AA01A9B8EEC00A1E
:1066B0005FF0FAFB20469DED030AFFF725FA0B4831
:1066C0008DED030A08F0D0F963699DED030A18689F
:1066D00074F0E0FDA5E700BFB84B0020000000000B
:1066E000F87F002000007A44907500202C5700208D
:1066F0000020704790F8B931002B14BF1B200320F5
:1067000070470000002070470120704790F890010A
:10671000062804D0A0F109035842584170470120CF
:1067200070470000012070470120704790F8B901C0
:10673000034A044B002814BF10461846704700BF98
:10674000FC600C0851B20D0890F8B901034A044BE3
:10675000002814BF10461846704700BF08610C0897
:1067600051B20D0890F890010A3818BF0120704707
:1067700090F8B9312BB9044BD3F8800A00F001002E
:1067800070470020704700BFB84B002090F8903150
:1067900023B9034B187880F0010070470020704740
:1067A000DC7F002038B590F89041012C054601D0DF
:1067B000002038BDC368186803681B699847002823
:1067C000F6D1EB681B68204683F8B848F1E7000073
:1067D000C3681B68002283F8B828012070470000B6
:1067E00070B52DED028B002380F8B931B0F8703010
:1067F000012B84B004460D4601D8002946D0636AB7
:10680000254E1B6893F8CB3073BB2448072384F8CC
:1068100090310368022B02D10021FBF773FC9FED3E
:10682000208AE368F0EE480A1868B0EE481AF0EEE5
:10683000481AB0EE480A012577F012FB84ED738AFE
:1068400084ED748A84ED758A84F8B85104F59A70E1
:1068500025F0FEFC134803F0B3FD96F88A3E6FF373
:10686000C30386F88A3E11E096F9883E002BCCDA05
:1068700004F13C0027F09EFD05460028C5D12046C6
:10688000FFF70CFB084A02214BF0ECFE284604B04F
:10689000BDEC028B70BD00BFB84B0020EC7E002029
:1068A00000000000847B002010610C0810B5044635
:1068B000064890F8603B012B03D100F65C3025F0D0
:1068C0002FFD002384F8B93110BD00BFB86B002044
:1068D00010B52DED028B094B0446D3F84409B0EEF8
:1068E000408A76F055FE9FED060A28EE008A0120C8
:1068F00084ED748ABDEC028B10BD00BFB86B002024
:106900000AD7233C10B52DED028B094B0446D3F872
:106910004409B0EE408A76F04BFE9FED060A28EE61
:10692000008A012084ED758ABDEC028B10BD00BF8A
:10693000B86B00200AD7233C10B52DED028B094B14
:106940000446D3F84409B0EE408A76F03FFE9FED4E
:10695000060A28EE008A012084ED738ABDEC028BC2
:1069600010BD00BFB86B00200AD7233CC3681B686A
:10697000186974F05FBF000038B5D0F89431044650
:106980000D461BB980F0E2F9C4F8940180F0DEF9FD
:10699000D4F89431C01A4FF47A73B0FBF3F0B4F822
:1069A0009231984209D32046FFF778FA2B88044A9F
:1069B00006214BF057FE012038BD0020FCE700BF48
:1069C0002C610C0890F89031052B05D1054BD3F8BC
:1069D0004C39D86874F0A6BEC36818680368DB68D1
:1069E000184700BFB86B002008B590F89031052B10
:1069F0000BD1094BD3F84C39D868243024F0AEFCC5
:106A0000BCEEC00A10EE100A08BDC368186803681F
:106A10009B689847F4E700BFB86B002090F890316E
:106A20008B4206D00A2B80F8901102D10148FCF766
:106A3000EFBF7047B82B002073B501231E4E80F8BE
:106A40007530D6F8943E834205460A4614D1012497
:106A500085F8B941D6F8940E019203681B689847EF
:106A6000019A0146154849F0F1F896F8893E9A06D0
:106A70001BD4204602B070BD01910321FFF7E2F85C
:106A8000019A04460028E2D185F8750049F0CCFD52
:106A90001B220A2149F024FD96F8893E9B06E8D581
:106AA000074A137843F0040303E0054A137843F0E0
:106AB00002031370DDE700BFB84B0020783B0020D5
:106AC000BC80002030B585B004460D4601466846BE
:106AD000FFF7EEF9694604F13C0028F01DFAC8B949
:106AE00049F0A2FD1B220A2149F0FAFC0D4B93F854
:106AF000893E9B0604D50C4A137843F004031370B7
:106B00002046FFF7CBF9094A04214BF0ABFD0020EA
:106B100005B030BD2946204605B0BDE83040FFF73E
:106B20008BBF00BFB84B0020BC80002040610C0828
:106B300030B585B004460D4601466846FFF7B8F902
:106B4000694604F13C0028F00BFAC8B949F06CFD25
:106B50001B220A2149F0C4FC0D4B93F8893E9B0689
:106B600004D50C4A137843F0040313702046FFF752
:106B700095F9094A04214BF075FD002005B030BDA0
:106B80002946204605B0BDE83040FFF755BF00BF9D
:106B9000B84B0020BC8000207C610C087FB5054606
:106BA0000E4605F13C0401466846FFF781F9694647
:106BB000204628F0D5F9C0B92046694628F0ACF93E
:106BC000044690B949F030FD1B220A2149F088FCA7
:106BD0000D4B93F8893E9B060FD42846FFF75EF9CC
:106BE0000A4A04214BF03EFD04E031462846FFF7F7
:106BF00023FF0446204604B070BD054A137843F0D5
:106C000004031370E9E700BFB84B0020B4610C081F
:106C1000BC80002030B5044685B00F4808F06CF801
:106C20000546B0B1072384F8903100230193029305
:106C30000393E36801A9186876F044FCE3681868D8
:106C4000036801A95B680022984704480021FBF70C
:106C500059FA284605B030BDB82B0020EC7E002044
:106C6000F0B5424FD7F81829D7F814392DED028B1B
:106C70001343D7F81029134387B005460C460CD1AF
:106C800047F0DEFF40F275124FF4801107B0BDEC03
:106C9000028BBDE8F04047F08BBF806977F0AEFE15
:106CA0002046B0EE408A10F045FC03283AD1EB684C
:106CB00001A9186876F0E2FC064698B3DDED017A8A
:106CC0006368009338EE678A294BDFED2A7A93F9DF
:106CD000883E9FED290A2948002BA8BFB0EE670A1D
:106CE00038EE008A009BBDEEC88A002118EE102AFB
:106CF0009342ACBF00930092FBF704FA6B691868EB
:106D000075F0DAFCDDED007A1D48B8EEE70A314691
:106D100008F056FE00212846FFF780FE07B0BDECC4
:106D2000028BF0BD94E80F0002AE86E80F00D7F8A2
:106D3000143904936A46D7F818390593022130466E
:106D400010F004FC78B949F06FFC0222152149F0DB
:106D5000C7FBDDED037AF8EEE77A77EE887AFDEE91
:106D6000E77ACDED007A0026AEE700BFB86B0020D1
:106D7000B84B0020000000000000C842EC7E00205C
:106D8000DC7F002030B52DED028BC36887B0044650
:106D900018680D4676F066FC00284BD194F89021D7
:106DA00000230093019302936AB93148039303A926
:106DB0000493059308F034FE28B1039B0093049BD1
:106DC0000193059B029394ED730A9FED2A8AE36871
:106DD000DDED000A9DED011ADDED021A1868B4EE32
:106DE000C80AF1EE10FAAABFDFED237A9FED230A5D
:106DF00020EE270A77F034F8D4ED747AF4EEC87AEE
:106E0000F1EE10FA07DBE3689FED1B0A186827EE26
:106E1000800A76F0BDFBD4ED757AF4EEC87AF1EE17
:106E200010FA07DBE3689FED140A186827EE800A62
:106E300076F0BEFBE3682946186876F039FF054610
:106E400088B10F4B1B68022B09D0032B03D10D4BCC
:106E500093F975311BB10A480021FBF773F9012141
:106E60002046FFF7DBFD284607B0BDEC028B30BDA6
:106E7000DC7F0020000000340000C8420000000059
:106E8000EC7E0020B84B002010B52DED028BC368BE
:106E9000DFED348A1B684269D3ED0A0A9FED328A1E
:106EA00093ED060AF4EEE80A0446F1EE10FA1068D3
:106EB000B8BFF0EE480A73F04DFFE36862691B68E3
:106EC0001068D3ED0A0A93ED060AF4EEE80AF1EE33
:106ED00010FAB8BFF0EE480A73F0B4FF636918689F
:106EE00074F044F918B96369186875F07FF9E368BC
:106EF00062691B68106893ED080A93ED0C1AD3EDD4
:106F0000070AB0EEC00A74F03FF9E36862691B68D3
:106F1000106893ED080A93ED0C1AD3ED070AB0EE52
:106F2000C00A74F0ABF96369186874F041FA18B9D3
:106F30006369186875F0C0FB00210C48FBF7E2F8A4
:106F40000B4860F079FD0B4AB2F88A3E23F4816366
:106F5000A2F88A3EBDEC028B20460221BDE810401B
:106F6000FFF75CBD0000003400007A43EC7E002097
:106F700000760020B84B002010B50C4B0446D3F827
:106F80004C0990ED0B0A90F8502000F11C0175F0AF
:106F9000E1FF07480368022B02D00821FBF7B2F893
:106FA00020460521BDE81040FFF738BDB86B002032
:106FB000EC7E0020F0B52DED028B4A4DDFED4A8AC4
:106FC000B0EE408A8FB00446D5F84C090E461746FD
:106FD00075F036FEF0EEC87AF4EEE87AF1EE10FACB
:106FE00007D49FED420AD5F84C0928EE000A75F047
:106FF0008DFED5F84C0990ED0B0AB0EEC00A0FB12A
:10700000B1EE400A75F072FE0023D5F84C090793E3
:1070100002AA07A90893099375F094FEDFED347A6C
:107020009DED027AB4EEE77AF1EE10FA56DD022217
:1070300007A90AA810F05AFD71680191304610F0B6
:1070400079FA019902460AA810F04AFAE3680AA9F7
:10705000186876F02DFE10B92648FDF7CFF8A06924
:1070600077F0CAFC02684368D5F84C09049303A979
:107070001C30039224F0A4F805A88DED050ACDED8F
:10708000060A24F06BF91C4B1B68022B1BD0D5F8A9
:107090004C391948D3ED0A7AF4EEE87AF1EE10FA99
:1070A000B8BFD3ED047AF4EEC07AF1EE10FA4FF0E7
:1070B000000110D5DFED117AB4EEE70AF1EE10FA17
:1070C00009DDFBF73FF804212046FFF7A7FC0FB0CE
:1070D000BDEC028BF0BDFBF715F8F4E72046FFF797
:1070E0004BFFF4E7B86B0020000000340000C842FA
:1070F00000009643B82B0020EC7E00200000FA43ED
:1071000008B50748D0F8803A9B0704D50121A0F5BF
:107110000050F7F73FF8BDE80840024808F0B2BA5F
:10712000B84B0020DC7F002030B589B00446FEF764
:1071300025FA30B10021204609B0BDE83040FEF705
:1071400055BA636A0221186878F014FCE36818687D
:1071500003685B69984701461048FCF739FF63698B
:10716000186875F0F7FB236A1D686369186874F086
:107170002FFA05AC20460A498DED020ACDED030A2F
:107180008DED041AFBF77EF9079B009394E80C0041
:1071900002A9284671F0E8FA09B030BDB82B0020EA
:1071A000EC7E002038B50446FEF7E8F9054628B124
:1071B00020460021BDE83840FEF718BA636A022174
:1071C000186878F0D7FB29462046BDE83840FEF71E
:1071D00053BE00000148002105F0F8BBE07C002010
:1071E00030B5174D9FED170A05F5804389B0044669
:1071F000D3F84C0975F00EFF01462846FCF7E8FE6F
:107200006369186875F0A6FB236A1D6863691868CE
:1072100074F0DEF905AC20460B498DED020ACDED88
:10722000030A8DED041AFBF72DF9079B009394E8F0
:107230000C0002A9284671F097FA09B030BD00BFD2
:10724000B82B002000000000EC7E002030B589B093
:107250000446FEF793F930B10021204609B0BDE89D
:107260003040FEF7C3B9636A0221186878F082FBE8
:10727000E368186803685B69984701461048FCF7A3
:10728000A7FE6369186875F065FB236A1D6863696A
:10729000186874F09DF905AC20460A498DED020A84
:1072A000CDED030A8DED041AFBF7ECF8079B009374
:1072B00094E80C0002A9284671F056FA09B030BDD6
:1072C000B82B0020EC7E002030B52DED028B83B072
:1072D0000446FEF753F920B9636A1B6893F8CC3073
:1072E00043B90021204603B0BDEC028BBDE830401D
:1072F000FEF77CB994F89831DA071DD4E3681D686D
:107300002B6828469B689847D5ED097A94F8983100
:10731000B4EEE70AF1EE10FA4CBF0122002262F34C
:10732000000384F8983107D4204603B0BDEC028BEB
:10733000BDE83040FFF7F8BE94F898319B0734D48D
:10734000E368DFED458A1B686269D3ED0A0A9FEDA9
:10735000438A93ED060A1068F4EEE80AF1EE10FA9B
:10736000B8BFF0EE480A73F0F5FCE36862691B6889
:107370001068D3ED0A0A93ED060AF4EEE80AF1EE7E
:1073800010FAB8BFF0EE480A73F05CFD6369186844
:1073900073F0ECFE18B96369186874F027FF94F86D
:1073A000983143F0020384F898312D4BD4F8A02192
:1073B000D3F810399B1A07EE903AB8EEE78AF1EE4F
:1073C000047AB0EEC87AB4EEE77AF1EE10FA38D566
:1073D00094F8983143F0040384F89831204684ED02
:1073E000678AFEF735FC6369A26B1B68D2ED001A51
:1073F00093EDC61AD3ED0E0AB1EE480A21F014FB44
:1074000063691B6840F2AA4093EDC31AD3EDC40A26
:1074100021F028F82046FEF777FB12488DED010A8F
:1074200007F022FB63699DED010A186873F032FFD3
:107430006369186803B0BDEC028BBDE8304075F09D
:1074400089BAD4ED677A68EE277AF5EEC07AF1EE64
:1074500010FAC3D5BCE700BF0000003400007A4337
:10746000B86B00202C57002030B52DED028B83B077
:107470000446FEF783F820B9636A1B6893F8CC30A2
:1074800043B90021204603B0BDEC028BBDE830407B
:10749000FEF7ACB86369DFED347A1B6894ED710ACE
:1074A00093EDC31AD3EDC40A20EE270A40F2C4407C
:1074B00020F0D8FF2046FEF727FB236A18680368F0
:1074C0009B6EB0EE408A9847284BB3F9443107EEE3
:1074D000903AB4F8BC316425F8EEE77A13FB05F373
:1074E000B4EEE70A07EE103A94F9BE31F1EE10FA65
:1074F000D8BFF0EE407A13FB05F39FED1D0AF8EEBE
:10750000C76A07EE103AF4EE407AB8EEC77AF1EEA9
:1075100010FA58BFB0EE670A6846CDED006A8DEDEF
:10752000017A23F06DFF236ADDED010A1868B4F8D3
:10753000C03102689DED000A126B13FB05F301EEEA
:10754000103A0121B8EEC11A90476369B0EE480ABB
:10755000186873F09FFE6369186875F0FBF903B053
:10756000BDEC028B30BD00BF0000C842B84B00200C
:1075700000007A4430B590F8B83185B00446F3B1D4
:1075800068460FF0A7FF404869460AF081F950B1FC
:1075900004F13C0027F0ACFC002384F8B83104F57A
:1075A0009A7024F055FE94F890310A2B2DD8DFE81C
:1075B00003F0294C50544C582C5C602C640000F5AE
:1075C0009A7024F045FE04F13C0590B194F84030E7
:1075D000012B0ED194F89031012B0AD1284627F0C7
:1075E000F5FA50B12046FEF759FC284A02214BF02B
:1075F00039F8284627F018FBD5E72046FEF74EFC61
:10760000234AF3E72046FFF77BFD94F844303BB96B
:1076100094F8463023B994F840309A1E53425341AF
:1076200094F8B9216AB363BB84F8B931194CD4F822
:10763000940E03681B6898472D220146A4F58250DA
:1076400005B0BDE8304048F001BB2046FFF76CFDB7
:10765000DBE72046FFF7A6FDD7E72046FFF7BAFD98
:10766000D3E72046FFF7BCFDCFE72046FFF7EEFD4E
:10767000CBE72046FFF728FEC7E72046FFF7F4FEDA
:10768000C3E705B030BD00BF203E002000620C08FB
:1076900028620C08B84B00202DE9F0412DED028B3B
:1076A000074684B008460E460FF044FF0328804684
:1076B0006D4628D1FB68186875F03AFE012822D182
:1076C0002148294607F0B4F90446B0B17B69DDEDE5
:1076D000007A1B68F8EEE77A93EDF27A77EEC77AD4
:1076E0004246FDEEE77A17EE901AC829CDED007AF2
:1076F000B8BFC82130460FF0F3FE204604B0BDEC01
:10770000028BBDE8F081114B0FCB85E80F003046AE
:107710000FF010FF014628460FF074FF04460028C2
:10772000EBD07B69DDED017A1B68B8EEE78AD3ED1B
:10773000F27A284638EE678A0FF0FCFEBDEEC88A62
:10774000024618EE101AD5E7B82B0020C4740020AA
:1077500010B543699FED126A1B68D3EDF06A93ED93
:10776000F17AD3EDF27A86B066EE866A27EE067A73
:1077700067EEC67A68460C46CDED006A8DED017A5B
:10778000CDED027A24F040F803A920468DED030ADE
:10779000CDED040A8DED051A10F0D8F906B010BD34
:1077A0000AD7233C30B5083204461D460FCA84E888
:1077B0000F00134301BFAB68A360EB68E36063682D
:1077C00085B093B920460FF0B5FE03AA01462846BE
:1077D0000FF0BCFE60B10399019120460FF0AAFEA4
:1077E0000199024620460FF07BFE204605B030BDD1
:1077F000696801912846F1E730B50B6985B0044608
:107800000BB94B6953B30023C4F8B43108310FC925
:107810006D4685E80F0029462046FFF73DFF98B9E1
:10782000124B0122D3F8101928460FF059FE48F0E8
:10783000FBFE0222152148F053FE2046FEF72EFBE8
:107840000B4A02214AF00EFF29462046FFF79AFA1A
:1078500010B90848FCF7D2FC05B030BD0123C0F8D0
:10786000B43105B0BDE83040FFF70EBBB86B002067
:107870005C620C08B82B002070B51A4B04460E460B
:107880000FCB88B06D4685E80F0020462946FFF7EC
:107890005FFFE368186875F0E5FE98B1E368186863
:1078A00003681B69984768B1E3682946186875F052
:1078B0004BFD38B947F0C4F940F295624FF480119E
:1078C00047F076F9214604A82B463246FFF76AFFB7
:1078D00004A92046FFF756FA10B90348FCF78EFCBE
:1078E00008B070BDC4740020B82B002070B5154BD3
:1078F0000C4606460FCB88B06D4685E80F0029463A
:107900003046FFF725FF2B462246314604A8FFF7F5
:1079100049FF6288A388122A4FEA132305D1227EE9
:10792000D20744BF03EB83035B00227A07EE903A51
:10793000C2F34002B8EE670A04A93046FFF73AFBEB
:1079400008B070BDC474002038B504460D46FFF77A
:1079500093FF0023C4F89431AB88A4F8923138BD6A
:107960007FB50D460446FFF787FF05F108010FC9F3
:107970006E4686E80F00134306D1234BD3F8142933
:10798000D3F818390292039304F5D07201213046DE
:107990000FF0DCFD94F8983170B923F0050343F043
:1079A000050384F898312046FEF778FA174A062135
:1079B0004AF058FE04B070BD23F0070384F89831F4
:1079C0000023C4F89C31E36862691B68106893ED7A
:1079D000080A93ED0C1AD3ED070AB0EEC00A73F053
:1079E000D3FBE36862691B68106893ED080A93EDA6
:1079F0000C1AD3ED070AB0EEC00A73F03FFC082161
:107A00002046FFF70BF8D5E7B86B002088620C081A
:107A10002DE9F0438DB06D4688461C460746134657
:107A20000A4601462846DDE91469FFF7BBFE95E8E2
:107A30000F0084E80F0007A80FF04CFDB8F80430E1
:107A4000F3B9B8F80010013105AA89B207F13C007A
:107A500026F068FCA0B1234605AA39462846FFF760
:107A6000A1FE95E80F0086E80F00BDF81630A3F1DF
:107A700052025342534189F800300DB0BDE8F08303
:107A800094E80F0086E80F000023F4E770B58B88B8
:107A900092B004460D461646002B44D10DA80FF0B7
:107AA00019FD298801310BAA89B204F13C0026F0A6
:107AB00039FC002837D0BDF82E10132903D014D874
:107AC0001039012913D833462A46214603A8FFF767
:107AD00069FE03AB214607A80BAAFFF763FEE36824
:107AE00007A9186876F024F901E0522901D012B0F4
:107AF00070BD07AD03A80FF0EDFC28460FF0EAFCBF
:107B00000DF10B03CDE90053324603AB0BA9204620
:107B1000FFF77EFFE0689DF80B3000682A4603A956
:107B200076F0DCF8E3E70120E1E7000070B5214BD7
:107B300004460E460FCB88B06D4685E80F00204600
:107B40002946FFF705FEE368186875F08BFD98B1CC
:107B5000E368186803681B69984768B1E3682946B9
:107B6000186875F0F1FB38B947F06AF840F2166210
:107B70004FF4801147F01CF8214604A82B463246EA
:107B8000FFF710FE04A92046FFF7FCF820B90A48C9
:107B9000FCF734FB08B070BD0023C4F89431B388FF
:107BA000A4F8923104AA31462046FFF76FFF00285F
:107BB000F0D1ECE7C4740020B82B0020F0B5324BB4
:107BC00004460E460FCB91B004AD85E80F00204669
:107BD0002946FFF7BDFDE368186875F043FD98B1CD
:107BE000E368186803681B69984768B1E368294629
:107BF000186875F0A9FB38B947F022F84FF4DF6236
:107C00004FF4801146F0D4FF0CAF08A80FF062FCCF
:107C100038460FF05FFC0DF10F03CDE900732A46E3
:107C200008AB31462046FFF7F3FEE0689DF80F30C1
:107C300000683A4608A976F097FB20B91348FCF78C
:107C4000DDFA11B0F0BD0023C4F89431B388A4F874
:107C5000923108AA31462046FFF718FF0028EDD0E0
:107C60000B4B1B68022B09D0032B03D1094B93F953
:107C700075311BB106480021FAF764FA012120464C
:107C8000FEF7CCFEDDE700BFC4740020B82B002057
:107C9000EC7E0020B84B002037B504460D467FF03F
:107CA00055F8C4F8A801D5ED027AF5EEC07AF1EEE8
:107CB00010FA17DD9FED137A67EE877AFCEEE77A0C
:107CC000C4ED697A2046FEF7E9F8D4F8A4214FF410
:107CD0007A73B2FBF3F30C4A062103B0BDE83040DF
:107CE0004AF0C0BC5BF0CCFE0023009395F90D2058
:107CF00095F90E3095F90C105BF05EFEC4F8A40106
:107D0000E0E700BF00007A44A0620C0810B5B1F9AA
:107D10000A30A0F8BC3191F90C3080F8BE31B1F9CD
:107D20000D30A0F8C031B1F90F3007EE903AF8EEFF
:107D3000E77A0446C0ED717A7FF008F80A21C4F8AA
:107D4000C8012046BDE81040FEF768BE38B50446BD
:107D50000D467EF0FBFFC4F8B001D5ED027A9FED31
:107D6000047A67EE877AFDEEE77AC4ED6B7A38BD68
:107D700000007A444A7C06480B46003A91F91010FC
:107D8000D3ED030A93ED020A18BF0122FAF7E4B912
:107D9000EC7E002070B51B4E0446D6F8940E0368A6
:107DA00086B01B680D469847042806D16B88102BB7
:107DB0000FD0732B20D000201CE0D6F8940E03685F
:107DC0001B6898470328F6D194F89031062BF2D11E
:107DD000ECE705F108010FC902ACDFED0B0A84E8FE
:107DE0000F00002309480093B0EE600A1A462146AE
:107DF00002F028F906B070BD20462946FFF7BAFF09
:107E00000120F7E7B84B002000000000847B002031
:107E100038B5D1F8093007EE903AF5EEC07AF1EEB8
:107E200010FA05460C4605DD0B7A022B03D01ED94D
:107E3000032B0ED038BD154B9FED150AD3F844091E
:107E400027EE800A75F0A4FBD4F80930C5F8D031CC
:107E5000F0E70E4B9FED0E0AD3F8440927EE800A97
:107E600075F0A6FBD4F80930C5F8D431E2E7074B2A
:107E70009FED070AD3F8440927EE800A75F0A6FBA8
:107E8000D4F80930C5F8CC31D4E700BFB86B002076
:107E90000000C84210B5044C237813B103485FF0CA
:107EA000C5FD207810BD00BFDC7F002000760020DB
:107EB00013B5094B01910446D3F8440903681B69C3
:107EC000984730B10199204602B0BDE81040FEF756
:107ED00053BD02B010BD00BFB86B002090F89831C0
:107EE00013F0010018BFC3F380007047094A03462E
:107EF00092F8650168B192F86421043A012A07D822
:107F00005B6A1B6893F8A100431E584258417047B2
:107F100000207047B87B002010B504467EF016FFA5
:107F2000D4F8B031C01AD4F8AC3123EAE3739842E4
:107F30004FF0000084BFC4F8AC01012010BD000068
:107F400010B503680446DB6D9847D4F8AC3123EADA
:107F5000E37398424FF000003CBFC4F8AC0101202D
:107F600010BD000008B504480321FAF7CBF8BDE8BE
:107F700008400148FAF7B2B9EC7E002070B51C4BFE
:107F80000446D3F8440903681B690E469847054622
:107F900010B90025284670BDD4F894315BB97EF045
:107FA000D5FEB4F89231C4F8940123B1114A537844
:107FB00043F0010353707EF0C9FED4F89421B4F865
:107FC0009231801A4FF47A72B0FBF2F09842E0D30B
:107FD00023B9084A537843F0010353702046FDF754
:107FE0005DFF3388044A06214AF03CFBD2E700BF1C
:107FF000B86B0020BC8000202C610C0810B590F8F4
:108000009031042B0446164B0AD1D3F84409036877
:108010001B69984718B12046FEF7AEFF002010BD3F
:108020000A79D3F84C39DFED0F6A93ED0E6A07EE4B
:10803000902A0A7E920748BF9FED0B7AF8EE677A86
:1080400048BF67EE877A86EE267AB0EEC77AB4EE3E
:10805000E77AF1EE10FAACBF01200020DFE700BFA5
:10806000B86B0020DB0FC9400000803B13B5094B03
:1080700001910446D3F8440903681B69984730B15D
:108080000199204602B0BDE81040FEF775BC02B071
:1080900010BD00BFB86B002010B504467EF056FE40
:1080A000D4F8A831C01AD4F8A43198424FF0000097
:1080B00084BFC4F8A401012010BD000038B50546F6
:1080C0000C467EF043FED5F8C831C01A23894FF420
:1080D0007A725343984294BF0020012038BD0000BB
:1080E000C368186808B190F8B808704710B5012146
:1080F00004460A4803F0EAFF28B120460321BDE800
:108100001040FEF78BBC46F09BFDBDE8104040F2EE
:108110006B124FF4801146F04BBD00BFE07C002095
:1081200090F89031022B04D0032B04D1034803F0C4
:108130009DBF012070470020704700BFE07C0020F9
:1081400038B50C4BD3F8805A90F89031032B044685
:1081500005F004050AD1084803F0A0FF94F8903117
:1081600035B110B9023B5842584138BD0020F5E7FF
:108170000120FAE7B84B0020E07C002010B50F4A40
:10818000137843F0800313700D4B93F9882E002A67
:10819000044609DBFEF73EFD70B920460822BDE823
:1081A00010400921FDF74EBDBDE8104001220E210F
:1081B00003F6EC30F5F7F8BE10BD00BFBC80002020
:1081C000B84B0020F8B5D0F8B44105465CB1012C9D
:1081D0001AD046F035FD40F643024FF4801146F0C8
:1081E000E7FC012407E0184BD3F8440903681B6936
:1081F000984710B900242046F8BD2846FEF744FEF3
:108200000123C5F8B431F6E7104F97F9883E002BEB
:10821000F0DA436A1B6893F8A160012EEAD13C3082
:1082200026F0D6F804460028E5D1D7F8B83E93F8F2
:10823000CB3033B132460D2107F6EC30F5F7B4FE02
:10824000D9E73446D7E700BFB86B0020B84B002011
:1082500038B5674BD3F8942E664B9A4204460D46C8
:1082600001D0002096E04B885D2B75D8512B2FD87C
:10827000103B9AB20F2A49D92046FDF70FFE6B88B2
:108280005D4A04214AF0EEF97DE0BC3B0D2BF3D8AA
:1082900001A252F823F000BF8783010887830108F9
:1082A00079820108798201087982010879820108BE
:1082B0007982010887830108798201088783010890
:1082C000798201087982010879820108878301088F
:1082D000523B0B2BD0D801A252F823F0D3830108D4
:1082E000798201089D830108B18301087982010820
:1082F000798201087982010879820108798201086E
:108300007982010879820108D98301080F2BB3D83B
:1083100001A252F823F000BFAB8301086382010879
:10832000B9830108BF830108CD830108B183010827
:108330009D83010879820108798201087982010808
:10834000798201087982010879820108798201081D
:1083500079820108C5830108732B46D006D8702B9B
:1083600040D0722B88D1FFF7EBFD1AE04AF2CF62C2
:10837000934234D080D8C92B0DD8BB2B85D8B23BC3
:10838000012B3FF679AF2046FDF788FD29884EF096
:108390008BFA012038BDCF2BF5D06DE72046FFF7D3
:1083A00079FD00283FF45DAFEDE7FFF7E7FDF8E763
:1083B0002046FFF707FFF4E7FFF720FEF1E7FFF79E
:1083C00077FDEEE7BDE83840FFF788BDFFF78EFD8B
:1083D000E7E7FFF74BFEE4E7FFF75EFEE1E7FFF7B5
:1083E0006DFEDEE7FFF798FDDBE7FFF7BBFDD8E7A3
:1083F000B84B0020D8760020B0620C0890F890317D
:10840000032B0BD0062B06D0012B0AD1C3681868AA
:1084100003681B681847044801F006BA034803F0D4
:10842000AFBE0020704700BF847B0020E07C0020AE
:108430008B88012B05D00B693BB94B692BB9CB68F5
:108440001BB904480021FAF761BA0248002208313A
:10845000FAF77EBAB82B002010B54B885D2B044686
:108460000A464BD8512B05D8103B99B20F291FD97A
:10847000002091E0523B0B2BFAD801A151F823F0D8
:10848000D3850108718401088D850108A385010841
:1084900071840108718401087184010871840108E4
:1084A000718401087184010871840108DB85010869
:1084B0000F2BDDD801A151F823F000BF9B850108E7
:1084C000AD850108B5850108BD850108CD85010888
:1084D000A38501088D850108718401087184010854
:1084E0007184010871840108718401087184010894
:1084F0007184010871840108C5850108B32B76D009
:1085000016D8732B70D00ED8702B6AD0722BAFD1C7
:10851000D1ED027A9FED3A7A67EE877AFDEEE77A3F
:10852000C0ED6B7A37E0B22BA2D1FFF771FC32E0DD
:10853000C92B23D8BB2B9BD9BC3B0D2B98D801A1B1
:1085400051F823F097850108978501087184010887
:108550007184010871840108718401087184010823
:10856000F585010871840108F58501087184010809
:108570007184010871840108F58501084AF2CF620F
:1085800093427FF475AFFFF7C1FB04E002F10801ED
:108590002046FEF765FB012010BD1146FFF7C6FA25
:1085A000F9E711462046FFF727F9F4E71146FFF7F0
:1085B00063F9F0E71146FFF799F9ECE71146FFF789
:1085C000C3F9E8E71146FFF7CBF9E4E7FFF78EFDC3
:1085D000E1E71146FFF7F2FADDE71146FFF75CFB32
:1085E000D9E7FFF7B3FBD6E7FFF7C4FBD3E7FFF705
:1085F0001FFFD0E7034802F10801F9F74BFECAE775
:108600000000C842EC7E0020704700007047000068
:108610007047000090F8280080F0010070470000CB
:10862000024B436040F605030381704700010204DA
:1086300090F85501704700000F20704700207047E8
:1086400000207047002070470020704700487047A6
:108650005C630C080048704768630C0808B509485B
:1086600000F50053D3F8D03AB3F9083000EE103AD1
:10867000B8EEC00AF5F736FFBDE808400248FDF73E
:1086800043BA00BFB82B0020B078002010B51448C2
:108690002DED028B1C4600F5005300F58040B3F928
:1086A0004431D0F8380908EE103A036882B09B6E66
:1086B000CDE900219847B8EEC88AF0EE400ADDE91E
:1086C0000021B0EE480A0748FCF772FE0548FDF7A6
:1086D0007DFA84ED000A02B0BDEC028B10BD00BF34
:1086E000B82B0020B0780020F8B51C4D05F50054DB
:1086F00005F580462846D6F84079F5F7E1FEB4F94D
:10870000803101EE103AB4F97E3100EE903A4342E6
:1087100000EE103AB8EEC11AF8EEE00AB8EEC00A60
:10872000384672F031FD2846D6F84069F5F7C8FEA4
:10873000B4F9803101EE103AB4F97E3100EE903A8E
:10874000434200EE103A3046B8EEC11ABDE8F84098
:10875000F8EEE00AB8EEC00A72F090BDB82B002027
:1087600038B5144C04F5804504F57C64D5F8380917
:1087700003689B689847692100F19402204646F0FF
:108780003DFFD5F838090368DB6898476A2100F196
:108790009402204646F032FFD5F8380903681B6979
:1087A00098476B2100F194022046BDE8384046F01E
:1087B00025BF00BFB82B0020014806F09DBA00BFBE
:1087C000B82B00203C307CF095BE000008B546F088
:1087D00037FABDE8084072224FF4801146F0E8B93C
:1087E00008B546F02DFABDE8084066224FF4801126
:1087F00046F0DEB908B546F023FABDE8084080220D
:108800004FF4801146F0D4B973B51E4E0546D6F824
:10881000940E0268126B9047044670B396F9893E35
:10882000002B2DDBD6F8B83E93F8CB402CB396F84E
:10883000883E03F0A003202B22D1D6F8940E0268C4
:1088400012689047052808D0D6F8940E026812687E
:108850009047A0F110035C425C410B4A02F61C13E6
:108860000193D6F8E83B0093D2F84039D2F8382982
:10887000214628467CF0ECFD0446204602B070BD3F
:108880000024FAE7B84B0020B86B00203C30FFF71B
:10889000BBBF000038B5114D04461148F6F7A4FAE5
:1088A00095F9883E002B14DA236A93F8A120012A57
:1088B00006D0D5F8940E0021BDE83840FCF796BEEE
:1088C0000D2105F6EC30F5F76FFB95F9883E002B8E
:1088D000EFDB2046BDE838407DF0F6B8B84B00200D
:1088E000B82B00203C30FFF7D5BF000001207047B7
:1088F0000120704701207047012070471120704708
:10890000012070470020704700207047002070470A
:1089100000487047AC640C0800487047B4640C0809
:1089200038B5436904461D68806976F06BF823F01A
:10893000A5FBDFED1B0A284672F00CFA6369A069FB
:108940001D6876F05FF823F099FBDFED150A2846E5
:1089500072F078FA6369186873F048FC6369DFEDB8
:10896000110A18689FED0E1AB0EE600A72F00CFC46
:108970006369DFED0C0A18689FED091AB0EE600A12
:1089800072F07CFC6369186872F012FD18B96369B3
:10899000186873F091FE00232364012038BD00BFE6
:1089A00000803B4400007A4370B52DED028B88B007
:1089B0000446FCF7E3FD70B120460021FCF716FEEB
:1089C00063699FED310A186808B0BDEC028BBDE801
:1089D000704073F04DBF636A0221186876F0CAFFD9
:1089E0002A4B93F8893E5B0603D56369186872F0D9
:1089F00031FA9FED258A60698DED018A8DED028A3D
:108A00008DED038A8DED048A03AA01A90068012374
:108A100072F08AFA6369186873F0FEFC236A1D68B5
:108A20002B68DE6C6369186872F0D2FD0122CDED0F
:108A3000060A8DED071A05A98DED050A2846B0EE48
:108A4000480AB0476369B0EE480A186872F022FC21
:108A50006369186873F07EFF236C8BB17EF076F942
:108A6000E36BC01A236C98420AD309480C220521F3
:108A7000FCF7FAFE20B906480C220221FCF7F4FEAE
:108A800008B0BDEC028B70BD00000000B84B0020A8
:108A9000B82B002038B504460D467EF057F9C4E9DE
:108AA0000F0538BD07207047012070470020704730
:108AB0000020704701207047004870474C650C0843
:108AC0000048704754650C0838B52DED028B002323
:108AD00080F83C30C368DFED338A1B684269D3ED10
:108AE0000A0A9FED318A93ED060AF4EEE80A04467D
:108AF000F1EE10FAB8BFF0EE480A106872F02AF9E9
:108B0000E36862691B681068D3ED0A0A93ED060AF0
:108B1000F4EEE80AF1EE10FAB8BFF0EE480A72F08F
:108B200091F9636920461D68FDF7BCF96368B3F9E4
:108B30003820B3F9363000EE903A434201EE102A65
:108B400000EE103AB8EEC11AF8EEE00AB8EEC00A2C
:108B5000284672F019FB636920461D68FDF7A2F9EB
:108B60006368B3F93820B3F9363000EE903A4342E7
:108B700001EE102A00EE103AB8EEC11AF8EEE00A43
:108B8000B8EEC00A284672F079FB084BD3F84C09BE
:108B900074F0FCF906480821F9F7B4FABDEC028B31
:108BA000012038BD0000003400007A43B86B00207B
:108BB000EC7E002030B52DED048BC3689FED898AD3
:108BC0001B684269D3ED0A7ADFED870A93ED060A46
:108BD000F4EEC87AF1EE10FA0446A8BFF0EE670A88
:108BE000106889B072F0B6F8636920461D68FDF719
:108BF00059F96368B3F93820B3F9363000EE903A8A
:108C0000434200EE103A01EE102A2846774DB8EEA6
:108C1000C11AF8EEE00AB8EEC00A72F0B5FAD5F85B
:108C20004C0974F0F5FAA5F5005393F8AD3ED90759
:108C300047D4D5F84C391A8BD20742D593ED0A9A0E
:108C4000B4EEC89AF1EE10FAB8BF93ED049AE36A55
:108C5000186851F075FFD5F84439D3ED067AA36B47
:108C600020EE270AD3ED007AF0EE498AE0EE278A5B
:108C7000B0EE490AF5EEC08AF1EE10FAD8BFDFED8A
:108C80005C8AF0EE680A1FF0E9FA28B9D5F84C09B9
:108C9000B0EE680A74F03AF8636893F95130272B04
:108CA0000FD0A36A186851F04BFFF0EEC07AF4EED3
:108CB000C87AF1EE10FAB0EE407A20D5002384F89D
:108CC0003C30236B1B68B3F9083000EE103A2046A5
:108CD000B8EEC00AFCF7AAFF2046FCF715FF2046B5
:108CE000B0EE408AFCF74AFC002848D0002120461C
:108CF00009B0BDEC048BBDE83040FCF777BCD5F87B
:108D00004C399FED3C0AD3ED0F7AD3ED0B6AA36B80
:108D100027EE800AF4EEC86AD3ED007AF1EE10FA7D
:108D200067EE277A10DB9FED341ADFED310A55200C
:108D300037EE800A1FF096FB012384F83C30D5F80B
:108D40004C0973F0D3FFBCE79FED2C7AF4EEC76AB1
:108D5000F1EE10FA05D89FED261ADFED290A592009
:108D6000E6E7F0EEE66AF4EEC86AF1EE10FAE3D553
:108D700094F83C30002B08BFB0EE670ADCE7636A6A
:108D80000221186876F0F6FD1E4805F06DFEB0EE83
:108D9000480AD5F84C0974F03DF901461A48FBF72A
:108DA00017F96369186873F0D5FD236A1D68636954
:108DB000186872F00DFC05AC204614498DED020ACE
:108DC000CDED030A8DED041AF9F75CFB079B0093C8
:108DD00094E80C0002A928466FF0C6FC09B0BDEC6F
:108DE000048B30BD0000003400007A43B86B0020D3
:108DF00000000000E02E65420000B442000000B414
:108E00000000B4C22C570020B82B0020EC7E0020BC
:108E100008B5064BD3F84C39D868243022F09EFAB6
:108E2000FCEEC07A17EE900A08BD00BFB86B0020B8
:108E3000024BD3F84C39D86872F074BCB86B002080
:108E40000B207047012070470020704701207047B9
:108E50000020704700487047EC650C0800487047D8
:108E6000F4650C080120704708B5DFED237AF4EEB5
:108E7000E70AF1EE10FA2DED028BF0EE408AB0EE2B
:108E8000608A35DDDFED1D7AF4EEE70AF1EE10FAC7
:108E90002ED5F6EE007A70EEE77ADFED196A9FEDD7
:108EA000190ADFED190AF0EEE77A87EEA67A872035
:108EB000B7EE001A30EE470A1FF0D4FADFED137A4E
:108EC0009FED131ADFED130A20EE270A8A2020EE09
:108ED000280A1FF0C7FA30EE080ABDEC028BDFED5E
:108EE0000A0ABDE808408D20B7EE001A1FF0BABA92
:108EF0009FED050AEFE700BFAC1C5A3ED578493F0D
:108F00008FC2753E9A99993F00000000FAEDEBBAC6
:108F10009A99993E9A9999BE70B57E4EB6F94431A8
:108F20002DED048B00EE903AF8EEE00A82B0044694
:108F300001AA6946B0EE600AFCF73AFAA06975F03A
:108F400061FDE369D0ED008AD3ED946AD3ED977AA1
:108F500090ED016AA3689FED701ADFED700A27EEAD
:108F6000E80A68EEA68A03F69403E6EE278A054629
:108F70003B20DFED6B7AB0EEE87AB4EEE77AF1EE03
:108F800010FA58BFB0EE677ADFED667AC7EE275A5F
:108F9000F7EE007A77EEE57A9DED007A67EE877A54
:108FA00093ED007A67EE877A9FED5F7AA6EE260A48
:108FB00087EE879A1FF056FA3C209FED571ADFED97
:108FC000570AB0EE408AB0EE680A1FF04BFA626BA7
:108FD000564B1268DFED567AB2F90820D3ED006ADD
:108FE0009FED541ADFED540A07EE102AB8EEC77A47
:108FF000F0EE408A27EE277ADFED507AA6EEA77AC8
:109000004520F4EE007AA7EE678ABAEE000A28EE51
:10901000000A83ED007A8DED000A1FF023FADDEDE2
:10902000017A9FED477A474B8DED000AF0EEE77A23
:10903000F4EEC77AF1EE10FA51D593ED007ADFED38
:10904000427A77EE277AB2EE007AF4EEC77AF1EE42
:1090500010FA58BFF0EE477AC3ED007A67EEA87AAF
:10906000CDED017A636A186890F8CB10002939D1E8
:1090700076F080FC636A1B6893F8A110012938D050
:1090800003293FD039B9236A186870F055F8236A6C
:1090900018686FF0A1FA236ADDED010A18689DEDEA
:1090A000000A0368B0EE491ADB6A9847204695ED3E
:1090B000028AFCF779FB2046F0EE400AB0EE480A3F
:1090C000FFF7D2FE236A62681868D2ED020A0368CD
:1090D00001215B6E984702B0BDEC048B70BD00228D
:1090E0001A60BFE796F9893E002BB4BF0121022127
:1090F000BEE7236A186870F01FF8236A18686FF0DB
:1091000081FAC8E7D9790029C5D12046FCF7C0FE0D
:10911000C1E700BFB84B002000000C4400000CC4A5
:109120000000FA4400409C45000034423C7F00208F
:109130000AD7233D00A08C4500A08CC58FC2753F87
:1091400000000034407F00208FC2F53C0E207047A5
:1091500000207047002070470020704700207047B3
:1091600000207047004870478C660C080048704724
:109170008C660C0870B52DED028B436A1B6893F862
:10918000CB300446FBB9052384F848302046FCF771
:109190000BFB636A02211868B0EE408A76F0EAFBA6
:1091A00094F95030E2696BB3D2F8F8515D4394F80A
:1091B0004820052A4FD8DFE812F02B005F0084001A
:1091C000B100DF001E01836A1B68B3F90830002B71
:1091D000B8BF5B429BB2B3F57A6FD4D2C36A1B6847
:1091E000B3F90830002BB8BF5B429BB2B3F57A6F7E
:1091F000C9D27DF0ABFDE36CC01A40F6C4139842AF
:10920000C1D8C3E794F95150D2F8FC215543CEE7B9
:10921000226A94F9511010689FED801A49F6404275
:109220005343514300EE103A00EE901A0268F8EEF4
:10923000E00A926BB8EEC00A9047DFED797A41F20E
:1092400093139D4238EE278A05DD94F950308BB197
:10925000012384F84830236A62681868D2ED020A54
:109260000368B0EE480ABDEC028B5B6EBDE870404F
:10927000002118470223ECE7226A9FED681A106864
:1092800049F64042534300EE103A0268B8EEC00A75
:10929000926BF0EE410A9047DFED627A38EE678A12
:1092A00005F50C55B5EEC08AF1EE10FA05F127056B
:1092B00043F2BA43D8BF9FED598A9D42CBD80423CD
:1092C000C7E7236A9FED551A186894F9513049F69B
:1092D0004042534300EE903A0268F8EEE00A926B87
:1092E000B0EE410A9047DFED4F7AE36938EE678AC6
:1092F000D3F8F831B5EEC08AF1EE10FAD8BF9FED81
:10930000478A002BB8BF5B4242F228329342A2DD6B
:1093100041F294139D429EDD03239AE7236A9FED59
:109320003F1A186894F9513049F64042534300EE11
:10933000903A0268F8EEE00A926BB0EE410A90476C
:10934000DFED387AE36938EE678AD3F8F831B5EEA5
:10935000C08A03F50C53F1EE10FA03F1270344F22F
:109360004E62D8BF9FED2D8A93423FF674AF2E4BCD
:109370009D42FFF670AFA2E7236A94ED111A1868B8
:10938000D4ED100A036894ED0F0A1B6B0021984777
:10939000DFED237A94F95020E36938EE278A1AB377
:1093A00093ED7E7AD4ED0F7AB8EEC77A77EEC77A6E
:1093B0009FED1E7AF0EEE77AF4EEC77AF1EE10FA3E
:1093C0003FF649AF0D2294F849101948FCF74CFAC2
:1093D000024618B901461648FCF746FA47F024F948
:1093E000162147F05DF836E793ED7F7AD4ED107AD9
:1093F000B8EEC77ADAE70D2294F849100C48FCF76A
:1094000033FA024618B901460948FCF72DFA47F02D
:109410000BF902220D2147F063F81CE70000000061
:10942000CDCC4C3E8FC2753E6DEEFFFF0000FA437F
:10943000B82B0020F7B5474D0446D5F8940E0368C5
:109440005B6B984718B90026304603B0F0BD95F91C
:10945000893E002B5EDBA36A1B68B3F90830002B42
:10946000B8BF5B429BB2B3F57A6FECD2636A1B68FC
:1094700093F8CB60002EE6D095F9883E002BE2DB16
:10948000D5F8940E03681B689847002784F84900B4
:1094900084F848707DF05AFCE36AE064A4F85070E8
:1094A0001B68B3F90830B3F5967F42DD012384F8D9
:1094B000513047F0B9F8152146F0F2FFB5F94431C3
:1094C00001EE103AE369B8EEC11A93ED7E0A8DED14
:1094D000011AF1EE410A5320B8EEC00ACDED000AA0
:1094E0001EF0C0FFE36984ED0F0A93ED7F0A9DED46
:1094F000011ADDED000AB8EEC00A54201EF0B2FFDA
:10950000E36984ED100AD3ED807AF8EEE77AC4EDD2
:10951000117A99E7D5F8940E03681B6898470128DB
:1095200091D0D5F8940E03681B689847002892D113
:1095300089E713F5967F01DAFF23B8E7A36A1B6872
:10954000B3F90830002BACBF0123FF2384F850305F
:10955000AFE700BFB84B00200420704701207047E0
:1095600000207047012070470048704724670C08AE
:10957000004870472C670C08012909D0232907D01F
:10958000042905D0034BD3F8840A00F0010070478A
:1095900001207047B84B0020C36B23B990F84100FD
:1095A00080F001007047002070470000034BD3F8A3
:1095B000840A80F00400C0F380007047B84B00209C
:1095C000012380F84230184670470000002380F8DD
:1095D000423001207047000070B52DED028BC3684A
:1095E0000446186890F9BB3886B0B0EE408A0BB3D9
:1095F00090F8BC68F6B173F09BFE01281AD1274899
:1096000019213EF08FFE07EE900AF8EEE77AF4EEAD
:10961000C87AF1EE10FA0DDD214BB3F9E63A07EE08
:10962000903AF8EEE77AF4EEC87AF1EE10FA18DB29
:10963000002012E01B4B0FCBFDEEC87A02AD85E88F
:109640000F0017EE901A012228460DF049FF01AADB
:10965000022128460DF07AFFE8B906B0BDEC028B76
:1096600070BDBDEEC88A8DED018A002529460E48E1
:10967000E563F8F747FD6369186873F01DF8DDEDE1
:10968000017A0A48B8EEE70A314606F099F984F8FB
:1096900041500120E1E70026E7E700BFC83800207D
:1096A000B84B0020C4740020EC7E0020DC7F00203A
:1096B00010B52DED048BC2689FED149A12684369B2
:1096C000D2ED0A0ADFED128AF4EEC90AF1EE10FAC1
:1096D0000446B8BFF0EE680A1868B0EE408A71F030
:1096E00039FBE268636912681868D2ED0A0AF4EE81
:1096F000C90AF1EE10FAB8BFF0EE680AB0EE480AF7
:1097000071F0A0FBBDEC048B012010BD0000003403
:1097100000007A4313B5C36842691B68F0EE400A43
:1097200093ED080A93ED0C1ACDED010A0446B0EE54
:10973000C00A106871F028FDE36862691B68106850
:1097400093ED080A93ED0C1ADDED010AB0EEC00AA4
:1097500071F094FD012002B010BD000010B52DED98
:10976000028BC36842691B68044693ED0C1AD3ED63
:10977000070A1068B0EE408A71F006FDE36862697E
:109780001B68106893ED0C1AD3ED070AB0EE480A77
:1097900071F074FDBDEC028B012010BD1FB5C36BD1
:1097A000022B0BD0032B1DD0012B22D1C3681868CC
:1097B0000368DB6805B05DF804EB1847806975F055
:1097C0001BF90D4B59689A6802911B68019301A916
:1097D00003921FF07DFEFDEEC07A17EE900A05B0F1
:1097E0005DF804FB4369186805B05DF804EB71F09F
:1097F00099BF0020F3E700BF787F0020C36B012BE7
:109800000AD003DC2BB19FED070A7047023B032B04
:10981000F9D84369186802E0C3681B68186972F0D8
:1098200009B800BF0000000030B5C26B012A89B042
:109830000C4604D0022A0AD0002009B030BDC3680B
:10984000186803681B6809B0BDE8304018470B4B27
:10985000586899681B680193094B02901B78039123
:10986000002B04AD18BF032201A928460EF03EF9D3
:1098700095E80F0084E80F000120DEE7787F0020E4
:10988000BC7F00207FB5C36B022B0FD0032B23D0EE
:10989000012B25D1C368186803689B689847BCEE04
:1098A000C00A10EE100A07B05DF804FB806975F07D
:1098B000A3F80D4B014658689A6804901B680393FF
:1098C00003A8059221F07CFC01A88DED010ACDEDE5
:1098D000020A21F043FDE2E7436918682430F8E703
:1098E0009FED020ADDE700BF787F00200000000046
:1098F00010B52DED028B01239FED1C8AC363C36855
:10990000044684B018688DED018AF0EE480AB0EE86
:10991000481AF0EE481AB0EE480A8DED028A8DED35
:10992000038A74F09DFAE3688DED018A8DED028A59
:109930008DED038A186801A973F0C4FDE368186807
:10994000036800225B6801A9984730B945F078F9AF
:10995000BB224FF4801145F02BF905480021F8F7A0
:10996000F1FB04B0BDEC028B10BD00BF0000000095
:10997000EC7E002030B589B00446FBF7FFFD70B1E6
:109980001D4805F013FD014618B1636A1B6893F882
:10999000CC10204609B0BDE83040FBF727BE636A13
:1099A0000221186875F0E6FFE368186803685B69D0
:1099B000984701461048FAF70BFB6369186872F084
:1099C000C9FF236A1D686369186871F001FE05AC60
:1099D00020460A498DED020ACDED030A8DED041AE9
:1099E000F8F750FD079B009394E80C0002A9284665
:1099F0006EF0BAFE09B030BDB82B0020EC7E00201E
:109A000010B52DED028BC368DFED298A1B68426912
:109A1000D3ED0A0A9FED278A93ED060AF4EEE80AD1
:109A20000446F1EE10FAB8BFF0EE480A106871F083
:109A300091F9E36862691B681068D3ED0A0A93ED37
:109A4000060AF4EEE80AF1EE10FAB8BFF0EE480AA2
:109A500071F0F8F9E36862691B68106893ED080A11
:109A600093ED0C1AD3ED070AB0EEC00A71F08CFB2F
:109A7000E36862691B68106893ED080A93ED0C1A9D
:109A8000D3ED070AB0EEC00A71F0F8FB63691868FD
:109A900072F012FE6369186872F0A8FB0648002194
:109AA000F8F750FB054B00221A70BDEC028B10BD7D
:109AB0000000003400007A43EC7E0020BC7F0020D0
:109AC0000223C363FFF79CBF0523C363FFF798BF5F
:109AD0000423C363FFF794BF10B50446FFF7F8FFF4
:109AE000074A0023936053601360064A93605360F3
:109AF0001360002384F8403084F84230012010BD08
:109B0000847F0020907F00200323C363FFF778BF8A
:109B100030B50623C363C36842691B6893ED080A26
:109B200093ED0C1AD3ED070A044685B01068B0EE29
:109B3000C00A71F029FBE36862691B68106893ED45
:109B4000080A93ED0C1AD3ED070AB0EEC00A71F0C3
:109B500095FB6369186871F02BFC18B96369186884
:109B600072F0AAFD7DF0F2F80C4D0346284601A9DB
:109B700040F8043B236A1B6800245B6F0393019445
:109B8000029420F063FF0023EC61AC616C616C62B5
:109B90002C6285F82C3005B030BD00BF487F002016
:109BA000024BD3F8840AC0F3C0007047B84B0020C2
:109BB0002DE9F0432DED028B9946C36B274C062B04
:109BC00085B080460E461746B0EE408A36D0FFF785
:109BD0009FFF96E80F00224D85E80F0097E80700E9
:109BE000103585E8070084F82D900023B9F1000FA7
:109BF00030D084ED0A8A63627DF0A8F803AB206060
:109C000002AA01A9304621F053F894ED092ADFEDAC
:109C1000157AD4ED0A1A9DED031ADDED020A9DEDC9
:109C2000010AD8F83C10104822EE272A3A46F7F7E6
:109C30000DFA05B0BDEC028BBDE8F083B9F1000F61
:109C4000C7D194F82D30002BC3D04369186872F047
:109C500033FDBEE7A36284ED098ACDE7487F00208B
:109C60004C7F00200AD7233CB82B002038B50B4D81
:109C70000446284605F006FD2B786BB194F8413078
:109C800053B90123064884F841305AF075F8BDE80D
:109C9000384004485DF0CABE38BD00BFDC7F0020FC
:109CA000004C00200076002070B52DED028B88B0AE
:109CB0000446FBF763FC054680B1294805F076FBB6
:109CC000014618B1636A1B6893F8CC10204608B0AF
:109CD000BDEC028BBDE87040FBF788BC636A9FED6A
:109CE000218A1868022175F045FE60698DED018AB0
:109CF0008DED028A8DED038A8DED048A2B4603AA31
:109D000001A9006871F010F963698DED008A186887
:109D10000368B0EE480A2A4669465B68984763695B
:109D2000186872F079FB6369186872F013FE236A91
:109D30001D682B68DE6C6369186871F049FC0122AC
:109D40008DED050ACDED060A8DED071AB0EE480A35
:109D500005A92846B04708B0BDEC028B70BD00BF16
:109D6000B82B002000000000A1B1DFED0F7A20EE3B
:109D7000270A33B1DFED0D0A0D4801220021F8F763
:109D8000EBB922B160EEA70A0948F8F763BADFED34
:109D9000070AF9E722B10648B0EE600AF8F796BA6A
:109DA0000348F8F7CFB900BF0AD7233C00000000F2
:109DB000EC7E00202DE9F0432DED028B8BB00446A4
:109DC000164606A802220F461D46B0EE408AF0EE67
:109DD000608A0DF08BFE284806A95AF08FF980465C
:109DE00058B946F021FC0522162146F079FB404681
:109DF0000BB0BDEC028BBDE8F083E36B032B02D00C
:109E00002046FFF781FE9DF858309DF854209DF8BC
:109E10005010F0EE680AB0EE480A2046FFF7A4FFA3
:109E20007CF094FF154BD7F800901860144BD7F8CE
:109E300004E0D7F808C0134AC3F80090C3F804E060
:109E4000C3F808C00023137096E807000E4F0F4EAA
:109E5000CDF80C9087E8070095E8070086E8070032
:109E6000CDE90076E16B0A48CDF810E003AACDF801
:109E700014C0F7F7A9F8BAE7004C0020447F00208F
:109E8000787F0020BC7F0020847F0020907F00200E
:109E9000B82B002010B588B00024059406940794D0
:109EA0009DF82C4002949DF82840CDE9003405AB84
:109EB000FFF780FF08B010BD2DE9F04F2DED028BAC
:109EC0008FB091469DF86C709DF868B0002F14BF5C
:109ED0000322022204460AA80D46B0EE408A9A46A2
:109EE000F0EE608A0DF002FE4D480AA95AF006F91C
:109EF000064658B946F098FB0522162146F0F0FABE
:109F000030460FB0BDEC028BBDE8F08F454AE36BE5
:109F1000D2F8842A12F0400F0DF11C082AD0012B30
:109F200002D02046FFF7E4FC5B46F0EE680A52469A
:109F3000B0EE480A49462046FFF716FFE368186866
:109F400003683A465B6829469847002304930593C3
:109F5000069307930893099304AB0093CDF804800C
:109F60003B462A46E16B3048F7F72EF8012384F888
:109F70004030C5E7022B02D02046FFF7A1FD002F9D
:109F800049D0E3684146186873F078FB40B922680D
:109F900003905268012120469047039B1E46AFE77D
:109FA000224B1B782BB963699DED070A186871F085
:109FB000B3FA52464946DFF874A0DFF884905B4656
:109FC000F0EE680AB0EE480A2046FFF7CDFE296899
:109FD0006A68AB68164D8AF80070164F29606A608F
:109FE000AB600023BB607B603B60C9F80830C9F8F8
:109FF0000430C9F800307CF0A9FE0F4B6A6829686C
:10A000001860AB680892CDE90079099307919AF836
:10A0100000304246A6E763699FED080AC6E700BF25
:10A02000004C0020B84B0020B82B0020BC7F002043
:10A03000787F0020847F0020447F00200000000003
:10A04000907F00202DE9F0472DED028B8EB0044665
:10A050006F489DF860A00E469046B0EE408A994643
:10A06000F0EE608A5AF04AF8054658B946F0DCFA34
:10A070000522162146F034FA28460EB0BDEC028BBC
:10A08000BDE8F087634BD3F8843A590648D5E36BB3
:10A09000012B02D02046FFF72BFCE36831461868FD
:10A0A00073F006FE054618B946F0BEFA0222E0E754
:10A0B00053464A46F0EE680AB0EE480A414620464A
:10A0C000FFF752FED6ED027AE16B0391F8EEE76AF4
:10A0D000D6ED037ACDED056AB8EEE77AD6ED017AD2
:10A0E0008DED067AF8EEE77A3046CDED077A0DF081
:10A0F00021FA00220BAB089209920A920B920C9261
:10A100000D920193C21E08AB009303995342534131
:10A1100005AA4148F6F758FF012384F84030ABE721
:10A120000027E068089709970A97006805AB08AA16
:10A13000314673F07DFD054600289DD0E36B022B70
:10A1400002D02046FFF7BCFC5346F0EE680A4A46B0
:10A15000B0EE480A41462046FFF706FE9DF814304F
:10A16000002B50D0E3680BA9186873F087FA80467B
:10A1700030B9236801215B682046984745467BE754
:10A18000264B1B782BB963699DED0B0A186871F09B
:10A19000C3F9234B089A1A60099ADFF89080DFF818
:10A1A00090905A60DFF874A00A9A9A609DF8143073
:10A1B0008AF80030C8F80870C8F80470C8F8007051
:10A1C000C9F80870C9F80470C9F800707CF0BEFDC9
:10A1D000D6ED027A134BE16B1860F8EEE76AD6ED24
:10A1E000037ACDED0B6AB8EEE77AD6ED017A8DED04
:10A1F0000C7ACDE90089F8EEE77A9AF80030CDEDD7
:10A200000D7A0BAA85E763699FED070ABEE700BFD9
:10A21000004C0020B84B0020B82B0020BC7F002051
:10A22000787F0020447F002000000000847F002011
:10A23000907F00202DE9F0470E4611461A46C36B69
:10A240008AB0052B9DF84C9005460DD0CDED050A42
:10A2500004928DED030A0291FFF736FCDDED050A4D
:10A26000049A9DED030A0299184C194F9DF8483045
:10A27000DFF868A0DFF868802846FFF775FD002347
:10A280000022A36063602360BB607B603B608AF850
:10A29000002096E8070088E807007CF057FD0D4B8A
:10A2A0001860B9F1000F0ED06268A36821680791A9
:10A2B00008920993CDE900789AF80030E96B0648D6
:10A2C00007AAF6F781FE0AB0BDE8F087787F002084
:10A2D000847F0020447F0020B82B0020BC7F00201A
:10A2E000907F00202DE9F0470F461946C36B8AB0D6
:10A2F000042B9DF85090054616460BD0CDED050A6F
:10A300008DED040A0391FFF7E3FBDDED050A9DEDFA
:10A31000040A03991A4C9DF84C309DF84820DFF848
:10A3200070A0DFF870802846FFF71EFD0023A360B1
:10A330006360236000238AF8003097E8070088E80C
:10A34000070096E807000F4F87E807007CF0FEFC47
:10A350000D4B1860B9F1000F0ED06268A368216838
:10A36000079108920993CDE900879AF80030E96BCC
:10A37000064807AAF6F728FE0AB0BDE8F08700BF36
:10A38000787F0020907F0020447F0020B82B0020A1
:10A39000BC7F0020847F002010B588B00024059485
:10A3A000069407949DF82C4002949DF82840CDE92E
:10A3B0000034134605AAFFF795FF08B010BD000052
:10A3C000034B00221A6000225A609A60DA607047DC
:10A3D0009C7F002000487047787F0020004870472D
:10A3E000847F002000487047907F00200A4B9FED3B
:10A3F0000B7AD3ED007AF4EEC77AF1EE10FAD8BFFB
